:100000000C94EE4B0C940F4C0C941BD40C940F4C92
:100010000C940F4C0C940F4C0C940F4C0C940F4CF4
:100020000C940F4C0C940F4C0C940F4C0C9446D623
:100030000C940F4C0C940F4C0C945BB70C940F4C1D
:100040000C940F4C0C940F4C0C940F4C0C940F4CC4
:100050000C940F4C0C940F4C0C940F4C0C940F4CB4
:100060000C940F4C0C9435D40C94C4D30C940F4CBA
:100070000C948ECD0C9430CD0C946CCD0C940F4C14
:100080000C94E6D40C940F4C0C940F4C0C940F4C25
:100090000C940F4C0C940F4C0C940F4C0C940F4C74
:1000A0000C940F4C0C940F4C0C940F4C0C9436BECB
:1000B0000C94DABE0C940F4C0C940F4C0C944CB96D
:1000C0000C940F4C0C940F4C0C940F4C0C940F4C44
:1000D0000C940F4C0C940F4C0C940F4C0C940F4C34
:1000E0000C9497A90C940F4C0C940F4C0C940F4C3F
:1000F0000C940F4C0C940F4C0C940F4C0C940F4C14
:100100000C940DBE0C94B1BE0C94E4BD0C9488BE4E
:100110000C940F4C0C940F4C0C940F4C0C940F4CF3
:100120000C940F4C0C940F4C0C940F4C0C940F4CE3
:100130000C940F4C0C94B0B80C940F4C0C940F4CC6
:100140000C940F4C0C940F4C0C940F4C0C940F4CC3
:100150000C940F4C0C940F4C0C948DA90C940F4CD8
:100160000C940F4C0C940F4C0C940F4C0C940F4CA3
:100170000C940F4C0C940F4C0C940F4C0C940F4C93
:100180000C940F4C0C940F4C0C940F4C0C940F4C83
:100190000C940F4C0C940F4C0C940F4C0C940F4C73
:1001A0000C945FBE0C9403BF0C940F4C0C940F4C3A
:1001B0000C94FEB80C940F4C0C940F4C0C940F4CF8
:1001C0000C940F4C0C940F4C0C940F4C0C940F4C43
:1001D0000C940F4C0C940F4C0C940F4C0C940F4C33
:1001E0000C940F4C0C940F4C24752E753875427579
:1001F0004D75517B517B517B517B517B5375517BAD
:10020000517B517B517B517B517B55755F75697576
:1002100073757D75517B517B517B517B517B517B3C
:100220008775517BDD75517B517B517B517B517BB8
:10023000517B517B1C76517B3879517B517B517BB3
:10024000517B517B517B517B517B3879517B517B69
:10025000517B49764E765876627664766E767976FC
:10026000517B8476517B517BC176517B517B517B95
:10027000517B517B517B517B517B517B517B517B1E
:10028000517B517B517B517BCB76517B517B517B99
:10029000517B517B517B517B517B517BD5761277C2
:1002A0004F779877A277BB77BB77C577CF77D9772A
:1002B000E377ED77F277FC7706784F7B4F7B4F7BC8
:1002C0004F7B4F7B4F7B4F7B4F7B4F7B4F7B4F7BDE
:1002D0004F7B4F7B4F7B4F7B4F7B4F7B4F7B4F7BCE
:1002E0004F7BC5774F7B4F7B4F7B4F7B4F7B4F7B4C
:1002F0004F7B4F7B4F7B4F7B4F7B4F7B4F7B4F7BAE
:100300004F7B4F7B4F7B10781A7824782E784F7B69
:100310004F7B4F7B4F7B4F7B4F7B4F7B4F7BBB7725
:10032000DC7A9D7AA17AA97A857A897A917A957A06
:10033000B57AC87AD07AD47AD87A347BAD7AA9786B
:10034000BA78CB78517B517B43781575517BDC783B
:10035000ED78FE783879AC772079517B5478517BF1
:100360000F7965783878517B517B517B7678877827
:1003700098787DBD85BD8DBD95BD9DBDA5BDADBD2F
:10038000B5BDA8C005C00DC015C01DC025C02DC07D
:1003900035C03DC045C04DC055C05DC065C06DC0D5
:1003A0008DC08DC08DC08DC08DC08DC08DC08DC0E5
:1003B0008DC08DC08DC08DC08DC08DC08DC08DC0D5
:1003C0008DC08DC08DC08DC08DC08DC08DC08DC0C5
:1003D0008DC08DC08DC08DC08DC08DC08DC08DC0B5
:1003E0008DC08DC08DC075C07DC08DC08DC08DC0CD
:1003F0008DC08DC08DC08DC08DC08DC08DC08DC095
:100400008DC08DC08DC08DC08DC08DC08DC08DC084
:100410008DC08DC08DC08DC08DC08DC08DC08DC074
:100420008DC08DC08DC08DC08DC08DC08DC08DC064
:100430008DC08DC08DC08DC08DC08DC08DC08DC054
:100440008DC08DC08DC08DC085C0084AD73B3BCEC6
:10045000016E84BCBFFDC12F3D6C74319ABD5683C3
:100460003DDA3D00C77F11BED9E4BB4C3E916BAA7B
:10047000AABE000000803F05A84CCDB2D44EB938CA
:1004800036A9020C50B9918688083CA6AAAA2ABEB1
:10049000000000803F07634236B79BD8A71A39682F
:1004A0005618AEBAAB558C1D3CB7CC5763BD6DED3D
:1004B000FD753EF6177231BF000000803F08000056
:1004C00000BE922449123EABAAAA2ABECDCCCC4C87
:1004D0003E00000080BEABAAAAAA3E00000000BFFA
:1004E000000000803F0000000000084178D3BB43BB
:1004F00087D1133D190E3CC3BD4282AD2B3E68EC43
:100500008276BED98FE1A93E4C80EFFFBE01C4FFC9
:100510007F3F0000000000000C94957A0C94ED7869
:100520000C948BB00C94135B0C94A2770C94255B09
:100530000C944F770C94E1670C9467C40C94F0AA68
:100540000C94DDCC0C9495BD0C94D35E0C94917AF4
:100550000C9434BD0C94DCAA0C94CD5F0C94A36B6A
:100560000C94AB5E0C942B5B0C9419D20C94AF5E84
:100570000C9412710C942E780C94995F0C94636C0B
:100580000C9427620C94254C0C944F7B0C948DC0DA
:100590000C945DC00C9481BC0C94CFBF0C941B4C8C
:1005A0000C94B3AB0C943C5B0C945CC50C94CF5D89
:1005B0000C94B57A0C94DF5E0C94C35B0C94EFBF83
:1005C0000C94114C0C94BA780C947B610C94FCAA9A
:1005D0000C941A830C9464850C944DC00C9487B0D1
:1005E0000C94A8C00C949F610C94DD750C94E37777
:1005F0000C949C670C94F75D0C9438790C94C35E52
:100600000C94E96C0C9421680C94CF5E0C94686790
:100610000C94B95F0C94195B0C94BE870C945B5BD3
:100620000C9458760C9463B00C94A3CF0C94366F52
:100630000C944CBD0C947FB00C9403D10C94F3BF7C
:100640000C94B55F0C940E5F0C940F790C947C5B4A
:100650000C94824F0C94CB5E0C945C5C0C94E95D22
:100660000C9425C00C94065B0C94DB5E0C94B15F7B
:100670000C94D7BB0C942E750C94D85C0C94475BEF
:100680000C94D47A0C94E6620C945D580C94D9774F
:100690000C941F5B0C9420790C9438780C94E35ED6
:1006A0000C94A9780C9462760C9485BD0C946E76AB
:1006B0000C9469750C9433670C94A55F0C941575B4
:1006C0000C9498780C9439BD0C94F3950C943E6F6F
:1006D0000C94057D0C94955B0C942D5F0C94665BDB
:1006E0000C94BE720C94D5760C94EF5E0C948983B6
:1006F0000C94644C0C9483B00C94A35E0C94DC7C3E
:100700000C94325C0C94E8AA0C94ED770C94B6B17E
:100710000C9447B00C943AD10C9465C00C94FE78BC
:100720000C9485C00C94AD7A0C94186C0C941277D0
:100730000C9410780C944E760C9449760C94EFBB84
:100740000C942DC00C94BB770C94CB780C94E3AE36
:100750000C94A5BD0C947DBD0C9479760C942B67FC
:100760000C94C55C0C9448BD0C9400AB0C94786C54
:100770000C94D5BF0C94DFAE0C94245E0C94D87A04
:100780000C9437670C9415C00C94B75E0C946DBC38
:100790000C94E4AA0C94FE5D0C9487780C94FC777E
:1007A0000C94D07A0C94C1760C9488660C94FDBCA1
:1007B0000C94F8AA0C94BD5F0C94D1CE0C94B67D29
:1007C0000C942F670C944ECA0C94955F0C94055EA4
:1007D0000C947DC00C941C760C9443780C94AB6400
:1007E0000C94754C0C946C660C949BBC0C945761E7
:1007F0000C941DC00C9454BD0C9464760C948476B7
:100800000C949D7A0C94FD600C94C87A0C940D7D28
:100810000C9424750C9410720C94FF610C948D83CD
:100820000C94A3AE0C94D55F0C947D750C94BF62B0
:100830000C949E5D0C948B7D0C941F630C9437D0AC
:100840000C94D15F0C9401620C94BF5E0C9476788A
:100850000C94E96B0C94DC780C94AC770C9455C038
:100860000C9493CA0C94DC7A0C940DC00C947FC445
:100870000C9405C00C94DFB10C94517B0C9454780B
:100880000C9453750C94017D0C9466C40C946CCC40
:100890000C94DECB0C94435E0C94857A0C94C66168
:1008A0000C94A97A0C9496620C94937B0C94CF7759
:1008B0000C946DC00C94897C0C944C620C94FB5B82
:1008C0000C949F5E0C9453610C9498770C942CBDFF
:1008D0000C94D6660C94A75E0C94A5AE0C94E15FC4
:1008E0000C9442750C94206B0C94B35E0C94A7AEE0
:1008F0000C94EC5F0C94B5BD0C9435C00C948267DD
:100900000C94C75E0C94B8C40C94D5BC0C942767A7
:100910000C9471620C94E75E0C94505B0C94715BC8
:100920000C947C720C9455750C94F2770C944D7564
:100930000C94C15F0C94465D0C94CBCC0C9475C0A8
:100940000C94E17C0C94117D0C94315B0C94247814
:100950000C94E17D0C94B5D10C94347B0C94D75E4F
:100960000C94E0AA0C9445C00C9450BD0C9465788E
:100970000C9406780C9491830C94F4AA0C9430BDDA
:100980000C94ADBD0C9464D30C9438750C946168D0
:100990000C943DC00C94A3D00C949BC40C94F152C5
:1009A0000C94F5710C94CB760C94C95F0C94897AF5
:1009B0000C94A15F0C94505F0C94BB5E0C94CA5DC8
:1009C0000C94EB5E0C94A95F0C94A17A0C94C55F17
:1009D0000C94315F0C9487750C9473750C94B66706
:1009E0000C94AC5B0C949DBD0C948DBD0C94ECAA46
:1009F0000C94C5770C941A780C9432B00C94366C25
:100A00000C945F750C94AD5F0C949D5F0C94097D04
:100A10000C94DDAE0C94955C0C94A37B0C944C7DF3
:100A20000C94F05D0C944BCC0C94E3BB5B257325CC
:100A3000735D20257320257320706F736974696F4F
:100A40006E2531382E336625730A005B25732573B6
:100A50005D202573202573206F66667365742532CB
:100A6000302E336625730A005B257325735D2025C0
:100A700073207A65726F206261636B6F66662531E1
:100A8000392E336625730A005B257325735D202597
:100A900073206C61746368206261636B6F666625A6
:100AA00031382E336625730A005B257325735D206C
:100AB0002573206C617463682076656C6F6369745C
:100AC000792531332E306625732F6D696E0A005BF0
:100AD000257325735D20257320736561726368201B
:100AE00076656C6F636974792531322E30662573B3
:100AF0002F6D696E0A005B257325735D20257320B9
:100B0000737769746368206D617825313764205B81
:100B1000303D6F66662C313D686F6D696E672C32B3
:100B20003D6C696D69742C333D6C696D69742B681B
:100B30006F6D696E675D0A005B257325735D202507
:100B40007320737769746368206D696E253137642B
:100B5000205B303D6F66662C313D686F6D696E6756
:100B60002C323D6C696D69742C333D6C696D697410
:100B70002B686F6D696E675D0A005B257325735D79
:100B8000202573207261646975732076616C7565C8
:100B90002532302E346625730A005B257325735D7C
:100BA000202573206A756E6374696F6E20646576A4
:100BB000696174696F6E2531342E3466257320287F
:100BC0006C61726765722069732066617374657207
:100BD000290A005B257325735D202573206A6572E1
:100BE0006B20686F6D696E672531362E3066257310
:100BF0002F6D696E5E33202A2031206D696C6C691F
:100C00006F6E0A005B257325735D202573206A656E
:100C1000726B206D6178696D756D2531352E30668A
:100C200025732F6D696E5E33202A2031206D696C2B
:100C30006C696F6E0A005B257325735D2025732038
:100C400074726176656C206D696E696D756D2531A4
:100C5000372E336625730A005B257325735D2025C7
:100C6000732074726176656C206D6178696D756D45
:100C70002531372E336625730A005B257325735D96
:100C80002025732076656C6F63697479206D6178B7
:100C9000696D756D2531312E306625732F6D696E46
:100CA0000A005B257325735D2025732066656564E6
:100CB00072617465206D6178696D756D2531312EB5
:100CC000306625732F6D696E0A005B257325735D91
:100CD0002025732061786973206D6F646525313834
:100CE000642025730A005B6D615D20206D696E20B4
:100CF000617263207365676D656E742531382E33BC
:100D00006625730A005B736C5D2020736F66742028
:100D10006C696D697420656E61626C652531326441
:100D20000A005B63745D202063686F7264616C20ED
:100D3000746F6C6572616E63652531372E3466257C
:100D4000730A005B6A615D20206A756E6374696F67
:100D50006E20616363656C65726174696F6E2538BE
:100D60002E306625730A005B6764695D20646566E2
:100D700061756C742067636F646520646973746166
:100D80006E6365206D6F6465253264205B303D477E
:100D900039302C313D4739315D0A005B6770615D48
:100DA0002064656661756C742067636F646520708C
:100DB00061746820636F6E74726F6C253364205B9E
:100DC000303D4736312C313D4736312E312C323DC6
:100DD0004736345D0A005B67636F5D20646566615A
:100DE000756C742067636F646520636F6F72642035
:100DF00073797374656D253364205B312D3620283B
:100E00004735342D473539295D0A005B67756E5DBE
:100E10002064656661756C742067636F6465207516
:100E20006E697473206D6F6465253564205B303D99
:100E30004732302C313D4732315D0A005B67706CC0
:100E40005D2064656661756C742067636F646520FE
:100E5000706C616E6525313064205B303D47313701
:100E60002C313D4731382C323D4731395D0A002560
:100E70006320776F726B206F66667365743A2531F5
:100E8000322E336625730A002563206D616368691D
:100E90006E6520706F736E3A2531312E336625737F
:100EA0000A00256320706F736974696F6E3A25318B
:100EB000352E336625730A00546F6F6C206E756D86
:100EC0006265722020202020202020202025640A16
:100ED00000466565642072617465206D6F64653AD3
:100EE00020202020202025730A0044697374616E3D
:100EF0006365206D6F64653A202020202020202526
:100F0000730A0050617468204D6F64653A20202098
:100F1000202020202020202025730A00506C616EA4
:100F2000653A202020202020202020202020202062
:100F30002025730A004D6F74696F6E206D6F6465B4
:100F40003A20202020202020202025730A00436FF3
:100F50006F7264696E6174652073797374656D3A3C
:100F600020202025730A00556E6974733A202020D2
:100F700020202020202020202020202025730A004F
:100F8000486F6D696E672073746174653A20202024
:100F9000202020202025730A0046656564686F6C58
:100FA000642073746174653A20202020202025730A
:100FB0000A004D6F74696F6E2073746174653A2016
:100FC0002020202020202025730A004379636C65AF
:100FD0002073746174653A20202020202020202076
:100FE00025730A00526177206D616368696E652020
:100FF00073746174653A20202025730A004D616383
:1010000068696E652073746174653A202020202021
:10101000202025730A004C696E65206E756D62652F
:10102000723A2531302E30660A00466565642072BA
:101030006174653A2531362E336625732F6D696EDE
:101040000A0056656C6F636974793A2531372E331F
:101050006625732F6D696E0A00B0107F105F104710
:101060003935202D20756E6974732D7065722D725F
:1010700065766F6C7574696F6E206D6F646500477F
:101080003934202D20756E6974732D7065722D6D45
:10109000696E757465206D6F64652028692E652EF4
:1010A000206665656472617465206D6F64652900F2
:1010B000473933202D20696E766572736520746917
:1010C0006D65206D6F646500EC10CC1047393120E0
:1010D0002D20696E6372656D656E74616C20646944
:1010E0007374616E6365206D6F64650047393020ED
:1010F0002D206162736F6C7574652064697374610F
:101100006E6365206D6F6465003D1125110F1147F9
:101110003634202D20636F6E74696E756F75732081
:101120006D6F6465004736312E31202D2065786162
:1011300063742073746F70206D6F6465004736317F
:10114000202D2065786163742070617468206D6F54
:10115000646500771168115911473139202D2059E4
:101160005A20706C616E6500473138202D20585A26
:1011700020706C616E6500473137202D2058592052
:10118000706C616E65000312F111D811B7119011E6
:10119000473830202D2063616E63656C206D6F745D
:1011A000696F6E206D6F646520286E6F6E652061BB
:1011B00063746976652900473320202D20636F759D
:1011C0006E74657220636C6F636B77697365206101
:1011D0007263206665656400473220202D20636CB1
:1011E0006F636B7769736520617263206665656400
:1011F00000473120202D206C696E65617220666584
:10120000656400473020202D206C696E6561722076
:10121000747261766572736520287365656B290049
:10122000CA12B01296127C12621248122E12473560
:1012300039202D20636F6F7264696E61746520734D
:10124000797374656D203600473538202D20636F23
:101250006F7264696E6174652073797374656D2053
:101260003500473537202D20636F6F7264696E61DA
:1012700074652073797374656D20340047353620AA
:101280002D20636F6F7264696E617465207379736A
:1012900074656D203300473535202D20636F6F72E4
:1012A00064696E6174652073797374656D203200B2
:1012B000473534202D20636F6F7264696E617465E9
:1012C0002073797374656D203100473533202D20EC
:1012D0006D616368696E6520636F6F7264696E61CA
:1012E00074652073797374656D00FD12F712F01246
:1012F000486F6D696E6700486F6D6564004E6F746E
:1013000020486F6D65640031132C13271321131CC3
:10131000131313456E6420486F6C6400486F6C644F
:1013200000446563656C00506C616E0053796E63B8
:10133000004F666600441340133B13486F6C640013
:1013400052756E0053746F70006E1364135E135702
:101350001353134A6F6700486F6D696E67005072D0
:101360006F6265004D616368696E696E67004F6604
:101370006600A4139E13981393138F13891380137D
:1013800053687574646F776E004379636C650045CC
:101390006E640053746F7000416C61726D00526531
:1013A00061647900496E697469616C697A696E6714
:1013B0000007140114FB13F613F213EE13E913E301
:1013C00013DD13D613D213C91353687574646F7782
:1013D0006E004A6F6700486F6D696E6700437963FE
:1013E0006C650050726F626500486F6C64005275E6
:1013F0006E00456E640053746F7000416C61726DD5
:1014000000526561647900496E697469616C697A3A
:10141000696E67002E141814473231202D206D6933
:101420006C6C696D65746572206D6F646500473220
:1014300030202D20696E63686573206D6F646500D0
:1014400068145D14511448145B7261646975735DAE
:10145000005B696E686962697465645D005B7374E2
:10146000616E646172645D005B64697361626C6586
:10147000645D0082147E1479142064656700206D19
:101480006D0020696E002A2A2A204E4F5449434598
:10149000202A2A2A20526573657474696E67206257
:1014A000617564207261746520746F202573005B20
:1014B000626175645D2055534220626175642072DB
:1014C00061746525313564205B313D393630302C0F
:1014D000323D31393230302C333D33383430302CDA
:1014E000343D35373630302C353D313135323030C2
:1014F0002C363D3233303430305D0A005B72786D0B
:101500005D2073657269616C205258206D6F64654F
:1015100025313564205B303D73747265616D696E91
:10152000675F6D6F64652C313D7061636B65745FDF
:101530006D6F64655D0A005B65785D2020656E6196
:10154000626C6520666C6F7720636F6E74726F6C6F
:1015500025313064205B303D6F66662C313D584F3D
:101560004E2F584F46462C323D5254532F4354531E
:101570005D0A005B65655D2020656E61626C6520BB
:101580006563686F25313864205B303D6F66662C7B
:10159000313D6F6E5D0A005B65635D20206578708C
:1015A000616E64204C4620746F2043524C46206F7D
:1015B0006E205458253664205B303D6F66662C31B2
:1015C0003D6F6E5D0A00F915F415EE15E815E2158C
:1015D000DB15D41532333034303000313135323010
:1015E0003000353736303000333834303000313960
:1015F0003230300039363030003000737973006695
:1016000062000000000702017DC661FF61AB3B9AEA
:1016100019DC437379730066760000000007030548
:101620007DC661FF61AF3BEC51783F737973006811
:1016300070000000000700097DC661E662B73B004C
:1016400000803F7379730068760000000007000D8A
:101650007DC661E17CBB3B0000004173797300698A
:1016600064000000000400117D897CFF61A73B003D
:10167000000000000000006E000000000001009F5C
:101680005E955B96629B3300000000000000006CDA
:10169000696E65000001009F5EAC5B96629B330043
:1016A0000000000000000076656C000000000205EC
:1016B0005EC35BFF61A73B00000000000000006606
:1016C00065656400000002245EFB5BFF61A73B00D0
:1016D000000000000000007374617400000000A3AB
:1016E0005E065BFF61A73B00000000000000006D8C
:1016F00061637300000000A75E135BFF61A73B00FE
:10170000000000000000006379637300000000AB7C
:101710005E195BFF61A73B00000000000000006D48
:101720006F747300000000AF5E1F5BFF61A73B009A
:1017300000000000000000686F6C6400000000B34F
:101740005E255BFF61A73B00000000000000007504
:101750006E697400000000BB5E315BFF61A73B0057
:1017600000000000000000636F6F7200000000BF07
:101770005E3C5BFF61A73B00000000000000006DC5
:101780006F6D6F00000000C35E475BFF61A73B0009
:1017900000000000000000706C616E00000000C7D7
:1017A0005E505BFF61A73B0000000000000000707E
:1017B00061746800000000CB5E5B5BFF61A73B00CB
:1017C000000000000000006469737400000000CF96
:1017D0005E665BFF61A73B00000000000000006642
:1017E000726D6F00000000D35E715BFF61A73B006C
:1017F00000000000000000746F6F6C00000000D754
:101800005E7C5BFF61A73B000000006D706F006DA8
:10181000706F7800000003E15F5C5CFF61A73B0034
:101820000000006D706F006D706F7900000003E1C3
:101830005F5C5CFF61A73B000000006D706F006D96
:10184000706F7A00000003E15F5C5CFF61A73B0002
:101850000000006D706F006D706F6100000003E1AB
:101860005F5C5CFF61A73B000000006D706F006D66
:10187000706F6200000003E15F5C5CFF61A73B00EA
:101880000000006D706F006D706F6300000003E179
:101890005F5C5CFF61A73B00000000706F7300702D
:1018A0006F737800000003D55F325CFF61A73B00D7
:1018B000000000706F7300706F737900000003D533
:1018C0005F325CFF61A73B00000000706F73007027
:1018D0006F737A00000003D55F325CFF61A73B00A5
:1018E000000000706F7300706F736100000003D51B
:1018F0005F325CFF61A73B00000000706F730070F7
:101900006F736200000003D55F325CFF61A73B008C
:10191000000000706F7300706F736300000003D5E8
:101920005F325CFF61A73B000000006F6673006FD1
:1019300066737800000003EC5F955CFF61A73B00D5
:101940000000006F6673006F66737900000003EC9F
:101950005F955CFF61A73B000000006F6673006F3E
:1019600066737A00000003EC5F955CFF61A73B00A3
:101970000000006F6673006F66736100000003EC87
:101980005F955CFF61A73B000000006F6673006F0E
:1019900066736200000003EC5F955CFF61A73B008B
:1019A0000000006F6673006F66736300000003EC55
:1019B0005F955CFF61A73B00000000686F6D0068E9
:1019C0006F6D6500000000B75E2B5BCF5DA73B002D
:1019D000000000686F6D00686F6D7800000000D532
:1019E0005F5761FF61703300000000686F6D006831
:1019F0006F6D7900000000D55F5761FF61713300A2
:101A0000000000686F6D00686F6D7A00000000D5FF
:101A10005F5761FF61723300000000686F6D0068FE
:101A20006F6D6100000000D55F5761FF6173330087
:101A3000000000686F6D00686F6D6200000000D5E7
:101A40005F5761FF61743300000000686F6D0068CC
:101A50006F6D6300000000D55F5761FF6175330053
:101A60000000007072620070726265000000006623
:101A7000C45761FF6176330000000070726200702D
:101A80007262780000000366C4C661FF61773300AC
:101A900000000070726200707262790000000366DC
:101AA000C4C661FF617B3300000000707262007089
:101AB00072627A0000000366C4C661FF617F330072
:101AC00000000070726200707262610000000366C4
:101AD000C4C661FF61833300000000707262007051
:101AE0007262620000000366C4C661FF6187330052
:101AF0000000007072620070726263000000036692
:101B0000C4C661FF618B33000000006A6F67006A22
:101B10006F67780000000066C45361E95D9533008B
:101B20000000006A6F67006A6F6779000000006656
:101B3000C45361F05D9533000000006A6F67006A6E
:101B40006F677A0000000066C45361F75D9533004B
:101B50000000006A6F67006A6F676100000000663E
:101B6000C45361FE5D953300000000707772007011
:101B70007772310000000054BD81BCFF61A73B00BB
:101B8000000000707772007077723200000000541D
:101B9000BD81BCFF61A73B00000000707772007040
:101BA0007772330000000054BD81BCFF61A73B0089
:101BB00000000070777200707772340000000054EB
:101BC000BD81BCFF61A73B00000000310000003177
:101BD0006D61000000030030BD57610162FB5900D8
:101BE0000000003100000031736100000003033485
:101BF000BDC661D7BB065A6666E63F3100000031BC
:101C000074720000000B0439BDC661E3BB0A5A00C0
:101C100000204231000000316D69000000030048DF
:101C2000BD5761EFBBFC590000004131000000319D
:101C3000706F00000003004CBD57612762005A001E
:101C400000803F3100000031706D00000003005043
:101C5000BD57616DBC015A000000403200000032E7
:101C60006D61000000030030BD576101621A5A0027
:101C700000803F3200000032736100000003033433
:101C8000BDC661D7BB255A6666E63F32000000320A
:101C900074720000000B0439BDC661E3BB295A0011
:101CA00000204232000000326D690000000300484D
:101CB000BD5761EFBB1B5A000000413200000032EB
:101CC000706F00000003004CBD576127621F5A006F
:101CD00000803F3200000032706D000000030050B1
:101CE000BD57616DBC205A00000040330000003336
:101CF0006D61000000030030BD57610162395A0078
:101D000000803F33000000337361000000030334A0
:101D1000BDC661D7BB445A6666E63F330000003358
:101D200074720000000B0439BDC661E3BB485A0061
:101D300000204233000000336D69000000030048BA
:101D4000BD5761EFBB3A5A00000041330000003339
:101D5000706F00000003004CBD576127623E5A00BF
:101D60000000003300000033706D000000030050DD
:101D7000BD57616DBC3F5A00000040340000003484
:101D80006D61000000030030BD57610162585A00C8
:101D9000000040340000003473610000000303348D
:101DA000BDC661D7BB635A6666E63F3400000034A7
:101DB00074720000000B0439BDC661E3BB675A6052
:101DC00076074034000000346D69000000030048CD
:101DD000BD5761EFBB595A00000041340000003488
:101DE000706F00000003004CBD576127625D5A0010
:101DF00000803F3400000034706D0000000300508C
:101E0000BD57616DBC5E5A0000004078000000784C
:101E1000616D0000000300505FC55CD85C2C32008F
:101E200000803F7800000078766D0000000B00997C
:101E30005FC661D666313200007A467800000078CD
:101E400066720000000B00955FC661D6662D3200F9
:101E5000007A467800000078746E0000000B03A141
:101E60005FC661D666393200000000780000007855
:101E7000746D0000000B039D5FC661D666353200AD
:101E800000914378000000786A6D0000000B00A507
:101E90005FC661465D3D3200409C45780000007899
:101EA0006A680000000B00A95FC6619E5D413200B8
:101EB000401C4678000000786A640000000B04AD06
:101EC0005FC661D66649320AD7233C7800000078A5
:101ED000736E0000000300B55F5761D5BF5031003D
:101EE00000803F780000007873780000000300B99C
:101EF0005F5761D5BF5131000000007800000078C5
:101F000073760000000B00BD5FC661D666513200DB
:101F1000803B4578000000786C760000000B00C123
:101F20005FC661D66655320000C84278000000786E
:101F30006C620000000B03C55FC661D666593200B3
:101F400000204178000000787A620000000B03C98D
:101F50005FC661D6665D32000000407900000079FE
:101F6000616D0000000300505FC55CD85C61320009
:101F700000803F7900000079766D0000000B009929
:101F80005FC661D666663200007A46790000007945
:101F900066720000000B00955FC661D66662320073
:101FA000007A467900000079746E0000000B03A1EE
:101FB0005FC661D6666E32000000007900000079CD
:101FC000746D0000000B039D5FC661D6666A320027
:101FD00000A04379000000796A6D0000000B00A5A5
:101FE0005FC661465D723200409C45790000007911
:101FF0006A680000000B00A95FC6619E5D76320032
:10200000401C4679000000796A640000000B04ADB2
:102010005FC661D6667E320AD7233C79000000791C
:10202000736E0000000300B55F5761D5BF523100E9
:1020300000803F790000007973780000000300B948
:102040005F5761D5BF53310000000079000000796F
:1020500073760000000B00BD5FC661D66686320055
:10206000803B4579000000796C760000000B00C1D0
:102070005FC661D6668A320000C8427900000079E6
:102080006C620000000B03C55FC661D6668E32002D
:1020900000204179000000797A620000000B03C93A
:1020A0005FC661D6669232000000407A0000007A76
:1020B000616D0000000300505FC55CD85C96320083
:1020C00000803F7A0000007A766D0000000B0099D6
:1020D0005FC661D6669B3200007A447A0000007ABF
:1020E00066720000000B00955FC661D666973200ED
:1020F000007A447A0000007A746E0000000B03A19D
:102100005FC661D666A3320000F0C27A0000007A92
:10211000746D0000000B039D5FC661D6669F3200A0
:102120000000007A0000007A6A6D0000000B00A534
:102130005FC661465DA732000048427A0000007A1F
:102140006A680000000B00A95FC6619E5DAB3200AB
:10215000007A447A0000007A6A640000000B04AD43
:102160005FC661D666B3320AD7233C7A0000007A94
:10217000736E0000000300B55F5761D5BF54310096
:102180000000007A0000007A73780000000300B9B4
:102190005F5761D5BF55310000803F7A0000007A5B
:1021A00073760000000B00BD5FC661D666BB3200CF
:1021B000007A447A0000007A6C760000000B00C1BF
:1021C0005FC661D666BF320000C8427A0000007A5E
:1021D0006C620000000B03C55FC661D666C33200A7
:1021E0000020417A0000007A7A620000000B03C9E7
:1021F0005FC661D666C732000040406100000061E2
:10220000616D0000000300505FC55CD85CCB3200FC
:102210000040406100000061766D000000030099FD
:102220005FC661E662D0320080CA4661000000618C
:1022300066720000000300955FC661E662CC320062
:10224000804A466100000061746E0000000303A133
:102250005FC661D666D832000080BF6100000061B1
:10226000746D00000003039D5FC661E662D4320016
:102270000080BF61000000616A6D0000000300A5DE
:102280005FC661465DDC3200349E4861000000613B
:102290006A680000000300A95FC6619E5DE032002D
:1022A000349E4861000000616A640000000304ADD0
:1022B0005FC661E662E832CDCCCC3D6100000061D2
:1022C00072610000000B03B15FC661E662EC32DFB1
:1022D000C3A9406100000061736E0000000300B5F7
:1022E0005F5761D5BF56310000803F61000000613B
:1022F00073780000000300B95F5761D5BF57310004
:10230000000000610000006173760000000300BD62
:102310005FC661E662F0320000FA446100000061CD
:102320006C760000000300C15FC661E662F4320013
:1023300000FA4461000000616C620000000303C504
:102340005FC661E662F8320000A0406100000061F3
:102350007A620000000303C95FC661E662FC3200D6
:102360000000406200000062616D00000003005048
:102370005FC55CD85C0033000000006200000062B2
:10238000766D0000000300995FC661E662053300C8
:102390000061456200000062667200000003009563
:1023A0005FC661E6620133000061456200000062C1
:1023B000746E0000000303A15FC661D6660D330092
:1023C0000080BF6200000062746D00000003039D86
:1023D0005FC661E6620933000080BF6200000062F0
:1023E0006A6D0000000300A55FC661465D11330001
:1023F00000A04162000000626A640000000300ADBA
:102400005FC661E6621D330AD7233C6200000062AA
:1024100072610000000B03B15FC661E66221330008
:1024200000803F6300000063616D00000003005006
:102430005FC55CD85C3533000000006300000063BA
:10244000766D0000000300995FC661E6623A3300D2
:1024500000614563000000636672000000030095A0
:102460005FC661E6623633000061456300000063C9
:10247000746E0000000303A15FC661D6664233009C
:102480000080BF6300000063746D00000003039DC3
:102490005FC661E6623E33000080BF6300000063F8
:1024A0006A6D0000000300A55FC661465D4633000B
:1024B00000A04163000000636A640000000300ADF7
:1024C0005FC661E66252330AD7233C6300000063B3
:1024D00072610000000B03B15FC661E66256330013
:1024E00000803F703100007031667271000300DCC3
:1024F000AAC661E662D7580000C842703100007079
:102500003163736C000300E0AAC661E662DB580029
:10251000007A44703100007031637368000300E496
:10252000AAC661E662DF580000FA4470310000700C
:102530003163706C000303E8AAC661E662E35800E9
:1025400000003E703100007031637068000303ECDE
:10255000AAC661E662E758CDCC4C3E7031000070EF
:102560003177736C000300F0AAC661E662EB580095
:10257000007A44703100007031777368000300F412
:10258000AAC661E662EF580000FA4470310000709C
:102590003177706C000303F8AAC661E662F3580055
:1025A00000003E703100007031777068000303FC5A
:1025B000AAC661E662F758CDCC4C3E70310000707F
:1025C00031706F6600030300ABC661E662FB58CD55
:1025D000CCCC3D673534006735347800000B03CD33
:1025E0005FC661D6669C3100000000673534006725
:1025F00035347900000B03CD5FC661D666A031008B
:10260000000000673534006735347A00000B03CDD5
:102610005FC661D666A431000000006735340067EC
:1026200035346100000B03CD5FC661D666A831006A
:10263000000000673534006735346200000B03CDBD
:102640005FC661D666AC31000000006735340067B4
:1026500035346300000B03CD5FC661D666B0310030
:10266000000000673535006735357800000B03CD75
:102670005FC661D666B43100001143673535006727
:1026800035357900000B03CD5FC661D666B83100E1
:10269000002043673535006735357A00000B03CDE0
:1026A0005FC661D666BC3100000000673535006743
:1026B00035356100000B03CD5FC661D666C03100C1
:1026C000000000673535006735356200000B03CD2B
:1026D0005FC661D666C4310000000067353500670B
:1026E00035356300000B03CD5FC661D666C8310087
:1026F000000000673536006735367800000B03CDE3
:102700005FC661D666CC31000000006735360067D1
:1027100035367900000B03CD5FC661D666D0310037
:10272000000000673536006735367A00000B03CDB0
:102730005FC661D666D43100000000673536006799
:1027400035366100000B03CD5FC661D666D8310017
:10275000000000673536006735366200000B03CD98
:102760005FC661D666DC3100000000673536006761
:1027700035366300000B03CD5FC661D666E03100DD
:10278000000000673537006735377800000B03CD50
:102790005FC661D666E43100000000673537006728
:1027A00035377900000B03CD5FC661D666E831008E
:1027B000000000673537006735377A00000B03CD1E
:1027C0005FC661D666EC31000000006735370067F0
:1027D00035376100000B03CD5FC661D666F031006E
:1027E000000000673537006735376200000B03CD06
:1027F0005FC661D666F431000000006735370067B8
:1028000035376300000B03CD5FC661D666F8310033
:10281000000000673538006735387800000B03CDBD
:102820005FC661D666FC310000000067353800677E
:1028300035387900000B03CD5FC661D666003200E3
:10284000000000673538006735387A00000B03CD8B
:102850005FC661D666043200000000673538006745
:1028600035386100000B03CD5FC661D666083200C3
:10287000000000673538006735386200000B03CD73
:102880005FC661D6660C320000000067353800670D
:1028900035386300000B03CD5FC661D66610320089
:1028A000000000673539006735397800000B03CD2B
:1028B0005FC661D6661432000000006735390067D4
:1028C00035397900000B03CD5FC661D6661832003A
:1028D000000000673539006735397A00000B03CDF9
:1028E0005FC661D6661C320000000067353900679C
:1028F00035396100000B03CD5FC661D6662032001A
:10290000000000673539006735396200000B03CDE0
:102910005FC661D666243200000000673539006763
:1029200035396300000B03CD5FC661D666283200DF
:10293000000000673932006739327800000103CDAA
:102940005FC661FF610D3400000000673932006727
:1029500039327900000103CD5FC661FF6111340097
:10296000000000673932006739327A00000103CD78
:102970005FC661FF611534000000006739320067EF
:1029800039326100000103CD5FC661FF6119340077
:10299000000000673932006739326200000103CD60
:1029A0005FC661FF611D34000000006739320067B7
:1029B00039326300000103CD5FC661FF612134003D
:1029C000000000673238006732387800000103D118
:1029D0005FC661FF61253400000000673238006780
:1029E00032387900000103D15FC661FF61293400EC
:1029F000000000673238006732387A00000103D1E6
:102A00005FC661FF612D3400000000673238006747
:102A100032386100000103D15FC661FF61313400CB
:102A2000000000673238006732386200000103D1CD
:102A30005FC661FF6135340000000067323800670F
:102A400032386300000103D15FC661FF6139340091
:102A5000000000673330006733307800000103D195
:102A60005FC661FF613D34000000006733300067DE
:102A700033307900000103D15FC661FF614134004A
:102A8000000000673330006733307A00000103D163
:102A90005FC661FF614534000000006733300067A6
:102AA00033306100000103D15FC661FF614934002A
:102AB000000000673330006733306200000103D14B
:102AC0005FC661FF614D340000000067333000676E
:102AD00033306300000103D15FC661FF61513400F0
:102AE0000000006A6964006A6964610000000066B1
:102AF000C49F61BF62D13B000000006A6964006A44
:102B00006964620000000066C49F61BF62D53B003B
:102B10000000006A6964006A69646300000000667E
:102B2000C49F61BF62D93B000000006A6964006A0B
:102B30006964640000000066C49F61BF62DD3B0001
:102B4000000000737973006A61000000000F00EF5D
:102B50005EC661D6666A310024F4497379730063F6
:102B600074000000000F040E5FC661D6666E310A65
:102B7000D7233C73797300736C0000000007002DAD
:102B80005F57610162723100000000737973007356
:102B900074000000000700EFBF5761CFBF45310050
:102BA00000803F737973006D740000000007022CF1
:102BB000BDC6619BBCF75900000040000000006DDD
:102BC0006500000000000067C4FDBCFDBCA73B0021
:102BD000000000000000006D6400000000000067BD
:102BE000C4D5BCD5BCA73B00000000737973006559
:102BF0006A000000000700898357612762C33B0019
:102C000000803F737973006A760000000007008D32
:102C10008357611A83693E0000A040737973006A8C
:102C2000730000000007009183576127626B3E002C
:102C300000803F7379730074760000000007005C29
:102C4000C5576127626A5B0000803F73797300712A
:102C5000760000000007008BB057617162305900A8
:102C6000000000737973007376000000000700E332
:102C7000AE57614C623D590000803F737973007319
:102C800069000000000700DFAE7B61A7AE3E59007F
:102C9000007A437379730065630000000007002722
:102CA000675761E167BA2900000000737973006516
:102CB000650000000007002B6757616168BB2900B1
:102CC0000000007379730065780000000007002F92
:102CD0006757612168BC290000803F7379730072D7
:102CE000786D0000000700336757612762BD290037
:102CF00000803F73797300626175640000040037DF
:102D00006757618866B8290000A040000000007382
:102D100072000000000000DDAEA3AEA5AEA73B0030
:102D20000000000000000071720000000000007F41
:102D3000B032B0FF61A73B0000000000000000714E
:102D40006900000000000083B047B0FF61A73B00AE
:102D500000000000000000716F000000000000870C
:102D6000B063B0FF61A73B000000000000000065F9
:102D70007200000000000066C4B3ABFF61A73B0017
:102D80000000000000000071660000000000006606
:102D9000C45361CA5DA73B00000000000000007240
:102DA000780000000000009BC46C66FF61A73B0038
:102DB000000000000000006D736700000000006765
:102DC000C45361FF61A73B000000000000000063E6
:102DD0006C65617200000066C4F152F152A73B00BD
:102DE00000000000000000746573740000000066BD
:102DF000C48B7DF3BFA73B0000000000000000640F
:102E00006566610000000066C4B67DFD60A73B00FA
:102E100000000000000000626F6F74000000006698
:102E2000C4E17DDC7CA73B000000000000000068DE
:102E3000656C700000000066C44C7DFF61A73B001C
:102E400000000000000000680000000000000066B4
:102E5000C44C7DFF61A73B000000007379730067DD
:102E6000706C0000000700DB5E57614C628031002F
:102E70000000007379730067756E0000000700DFC3
:102E80005E5761276281310000803F73797300676C
:102E9000636F0000000700E35E576101627F31004D
:102EA00000803F737973006770610000000700E7DE
:102EB0005E57614C62823100000040737973006795
:102EC00064690000000700EB5E57612762833100F0
:102ED00000000000000000676300000000000066C2
:102EE000C4937BA37BA73B00000000000000006DA3
:102EF00061000000000B04315FC661D6667731CDFA
:102F0000CCCC3D0000000066640000000003007FA0
:102F1000C4576127626A3E00000000756461007555
:102F2000646130000003009BC49F61BF62633B008B
:102F30000000007564610075646131000003009B4E
:102F4000C49F61BF62673B0000000075646100754B
:102F5000646132000003009BC49F61BF626B3B0051
:102F60000000007564610075646133000003009B1C
:102F7000C49F61BF626F3B00000000756462007512
:102F8000646230000003009BC49F61BF62733B001A
:102F90000000007564620075646231000003009BEC
:102FA000C49F61BF62773B000000007564620075DA
:102FB000646232000003009BC49F61BF627B3B00E0
:102FC0000000007564620075646233000003009BBA
:102FD000C49F61BF627F3B000000007564630075A1
:102FE000646330000003009BC49F61BF62833B00A9
:102FF0000000007564630075646331000003009B8A
:10300000C49F61BF62873B00000000756463007568
:10301000646332000003009BC49F61BF628B3B006E
:103020000000007564630075646333000003009B57
:10303000C49F61BF628F3B0000000075646400752F
:10304000646430000003009BC49F61BF62933B0037
:103050000000007564640075646431000003009B27
:10306000C49F61BF62973B000000007564640075F7
:10307000646432000003009BC49F61BF629B3B00FD
:103080000000007564640075646433000003009BF5
:10309000C49F61BF629F3B000000005F7465005FDA
:1030A00074657800000002B8C4C661FF61A05600D4
:1030B0000000005F7465005F74657900000002B86D
:1030C000C4C661FF61A456000000005F7465005F24
:1030D00074657A00000002B8C4C661FF61A856009A
:1030E0000000005F7465005F74656100000002B855
:1030F000C4C661FF61AC56000000005F7465005FEC
:1031000074656200000002B8C4C661FF61B0560079
:103110000000005F7465005F74656300000002B822
:10312000C4C661FF61B456000000005F7472005FA6
:1031300074727800000002B8C4C661FF61C5570010
:103140000000005F7472005F74727900000002B8C2
:10315000C4C661FF61C957000000005F7472005F60
:1031600074727A00000002B8C4C661FF61CD5700D6
:103170000000005F7472005F74726100000002B8AA
:10318000C4C661FF61D157000000005F7472005F28
:1031900074726200000002B8C4C661FF61D55700B6
:1031A0000000005F7472005F74726300000002B878
:1031B000C4C661FF61D957000000005F7473005FEF
:1031C00074733100000002B8C4C661FF613057005B
:1031D0000000005F7073005F70733100000002B880
:1031E000C4C661FF614057000000005F6373005F69
:1031F00063733100000002B8C4C661FF615057001C
:103200000000005F6573005F65733100000002B865
:10321000C4C661FF616057000000005F7873005F03
:1032200078733100000002B8C4C661FF61925A0091
:103230000000005F6665005F66653100000002B84F
:10324000C4C661FF617057000000005F7473005FC7
:1032500074733200000002B8C4C661FF61345700C5
:103260000000005F7073005F70733200000002B8EE
:10327000C4C661FF614457000000005F6373005FD4
:1032800063733200000002B8C4C661FF6154570086
:103290000000005F6573005F65733200000002B8D4
:1032A000C4C661FF616457000000005F7873005F6F
:1032B00078733200000002B8C4C661FF61AA5A00E8
:1032C0000000005F6665005F66653200000002B8BE
:1032D000C4C661FF617457000000005F7473005F33
:1032E00074733300000002B8C4C661FF6138570030
:1032F0000000005F7073005F70733300000002B85D
:10330000C4C661FF614857000000005F6373005F3F
:1033100063733300000002B8C4C661FF61585700F0
:103320000000005F6573005F65733300000002B842
:10333000C4C661FF616857000000005F7873005FDA
:1033400078733300000002B8C4C661FF61C25A003E
:103350000000005F6665005F66653300000002B82C
:10336000C4C661FF617857000000005F7473005F9E
:1033700074733400000002B8C4C661FF613C57009A
:103380000000005F7073005F70733400000002B8CB
:10339000C4C661FF614C57000000005F6373005FAB
:1033A00063733400000002B8C4C661FF615C57005B
:1033B0000000005F6573005F65733400000002B8B1
:1033C000C4C661FF616C57000000005F7873005F46
:1033D00078733400000002B8C4C661FF61DA5A0095
:1033E0000000005F6665005F66653400000002B89B
:1033F000C4C661FF617C5700000000000000005F50
:1034000064616D0000000066C4435E435EA73B003C
:10341000000000000000007365303000000200660C
:10342000C47B6196624959000000000000000073EF
:103430006530310000020066C47B6196624B590022
:1034400000000000000000736530320000020066DA
:10345000C47B6196624D59000000000000000073BB
:103460006530330000020066C47B6196624F5900EC
:1034700000000000000000736530340000020066A8
:10348000C47B619662515900000000000000007387
:103490006530350000020066C47B619662535900B6
:1034A0000000000000000073653036000002006676
:1034B000C47B619662555900000000000000007353
:1034C0006530370000020066C47B61966257590080
:1034D0000000000000000073653038000002006644
:1034E000C47B61966259590000000000000000731F
:1034F0006530390000020066C47B6196625B59004A
:10350000000000000000007365313000000200661A
:10351000C47B6196625D59000000000000000073EA
:103520006531310000020066C47B6196625F59001C
:1035300000000000000000736531320000020066E8
:10354000C47B6196626159000000000000000073B6
:103550006531330000020066C47B619662635900E6
:1035600000000000000000736531340000020066B6
:10357000C47B619662655900000000000000007382
:103580006531350000020066C47B619662675900B0
:103590000000000000000073653136000002006684
:1035A000C47B61966269590000000000000000734E
:1035B0006531370000020066C47B6196626B59007A
:1035C0000000000000000073653138000002006652
:1035D000C47B6196626D590000000000000000731A
:1035E0006531390000020066C47B6196626F590044
:1035F0000000000000000073653230000002006629
:10360000C47B6196627159000000000000000073E5
:103610006532310000020066C47B61966273590016
:1036200000000000000000736532320000020066F6
:10363000C47B6196627559000000000000000073B1
:103640006532330000020066C47B619662775900E0
:1036500000000000000000736532340000020066C4
:10366000C47B61966279590000000000000000737D
:103670006532350000020066C47B6196627B5900AA
:103680000000000000000073653236000002006692
:10369000C47B6196627D5900000000000000007349
:1036A0006532370000020066C47B6196627F590074
:1036B0000000000000000073653238000002006660
:1036C000C47B619662815900000000000000007315
:1036D0006532390000020066C47B6196628359003E
:1036E0000000000000000073797300000000006615
:1036F000C4AB641F63A73B00000000000000007023
:103700003100000000000066C4AB641F63A73B00EB
:103710000000000000000031000000000000006612
:10372000C4AB641F63A73B00000000000000003230
:103730000000000000000066C4AB641F63A73B00EC
:1037400000000000000000330000000000000066E0
:10375000C4AB641F63A73B000000000000000034FE
:103760000000000000000066C4AB641F63A73B00BC
:10377000000000000000007800000000000000666B
:10378000C4AB641F63A73B00000000000000007989
:103790000000000000000066C4AB641F63A73B008C
:1037A000000000000000007A000000000000006639
:1037B000C4AB641F63A73B00000000000000006171
:1037C0000000000000000066C4AB641F63A73B005C
:1037D0000000000000000062000000000000006621
:1037E000C4AB641F63A73B0000000000000000633F
:1037F0000000000000000066C4AB641F63A73B002C
:103800000000000000000067353400000000006682
:10381000C4AB641F63A73B0000000000000000670A
:103820003535000000000066C4AB641F63A73B0091
:103830000000000000000067353600000000006650
:10384000C4AB641F63A73B000000000000000067DA
:103850003537000000000066C4AB641F63A73B005F
:10386000000000000000006735380000000000661E
:10387000C4AB641F63A73B000000000000000067AA
:103880003539000000000066C4AB641F63A73B002D
:1038900000000000000000673932000000000066F0
:1038A000C4AB641F63A73B0000000000000000677A
:1038B0003238000000000066C4AB641F63A73B0001
:1038C00000000000000000673330000000000066C8
:1038D000C4AB641F63A73B00000000000000006D44
:1038E000706F000000000066C4AB641F63A73B005C
:1038F00000000000000000706F7300000000006610
:10390000C4AB641F63A73B00000000000000006F11
:103910006673000000000066C4AB641F63A73B0031
:1039200000000000000000686F6D000000000066ED
:10393000C4AB641F63A73B000000000000000070E0
:103940007262000000000066C4AB641F63A73B0006
:1039500000000000000000707772000000000066A8
:10396000C4AB641F63A73B00000000000000006AB6
:103970006F67000000000066C4AB641F63A73B00D4
:10398000000000000000006A69640000000000669A
:10399000C4AB641F63A73B0000000000000000757B
:1039A0006461000000000066C4AB641F63A73B00B5
:1039B0000000000000000075646200000000006666
:1039C000C4AB641F63A73B0000000000000000754B
:1039D0006463000000000066C4AB641F63A73B0083
:1039E0000000000000000075646400000000006634
:1039F000C4AB641F63A73B00000000000000005F31
:103A00007465000000000066C4AB641F63A73B0040
:103A1000000000000000005F7472000000000066FB
:103A2000C4AB641F63A73B00000000000000005F00
:103A30007473000000000066C4AB641F63A73B0002
:103A4000000000000000005F7073000000000066CE
:103A5000C4AB641F63A73B00000000000000005FD0
:103A60006373000000000066C4AB641F63A73B00E3
:103A7000000000000000005F6573000000000066A9
:103A8000C4AB641F63A73B00000000000000005FA0
:103A90007873000000000066C4AB641F63A73B009E
:103AA000000000000000005F666500000000006686
:103AB000C4AB641F63A73B00000000000000006D62
:103AC0000000000000000066C49C67FF61A73B0087
:103AD000000000000000007100000000000000660F
:103AE000C48267FF61A73B00000000000000006F78
:103AF0000000000000000066C46867FF61A73B008B
:103B0000000000000000002400000000000000662B
:103B1000C4B667FF61A73B00000000486F6D696E87
:103B200067206572726F72202D202563206178698D
:103B3000732073657474696E6773206D6973636F46
:103B40006E666967757265640050726F62696E6750
:103B5000206572726F72202D202563206178697351
:103B60002063616E6E6F74206D6F76652064757270
:103B7000696E672070726F62696E67005B69645D71
:103B8000202054696E7947204944253330730A0058
:103B90005B68765D2020686172647761726520766B
:103BA000657273696F6E2531362E32660A005B6866
:103BB000705D2020686172647761726520706C614D
:103BC00074666F726D2531352E32660A005B66763B
:103BD0005D20206669726D7761726520766572730B
:103BE000696F6E2531362E32660A005B66625D2093
:103BF000206669726D77617265206275696C6425F3
:103C000031382E32660A00456E7465722024626F68
:103C10006F743D3120746F20656E74657220746816
:103C20006520626F6F74206C6F616465722E0A008C
:103C30000A0A0A2323232054696E794720424F4FF2
:103C400054204C4F414445522048656C702023233A
:103C5000230A00456E7465722024646566613D31F7
:103C600020746F20726573657420746865207379A1
:103C70007374656D20746F20746865206661637469
:103C80006F72792064656661756C742076616C75FD
:103C900065732E0A546869732077696C6C206F769F
:103CA0006572777269746520616E79206368616EF0
:103CB00067657320796F752068617665206D616432
:103CC000652E0A000A0A0A2323232054696E7947C5
:103CD00020524553544F52452044454641554C547B
:103CE000532048656C70202323230A00496E766FA9
:103CF0006B652073656C662074657374206279202F
:103D0000656E746572696E672024746573743D4EC8
:103D1000207768657265204E206973206F6E65207C
:103D20006F663A0A202024746573743D3120207335
:103D30006D6F6B6520746573740A2020247465733D
:103D4000743D322020686F6D696E672074657374EE
:103D500020202028796F75206D7573742074726926
:103D60007020686F6D696E6720737769746368652A
:103D700073290A202024746573743D3320207371E5
:103D8000756172652074657374202020286120732A
:103D90006572696573206F662073717561726573F2
:103DA000290A202024746573743D342020617263D5
:103DB000207465737420202020202028736F6D6587
:103DC000206C6172676520636972636C6573290A90
:103DD000202024746573743D3520206477656C6CF5
:103DE000207465737420202020286D6F7665732001
:103DF0007370616365642062792031207365636F3D
:103E00006E64206477656C6C73290A2020247465C5
:103E100073743D36202066656564686F6C64207439
:103E20006573742028656E746572202120616E644C
:103E3000207E20746F20686F6C6420616E64207235
:103E40006573746172742C20726573706563746934
:103E500076656C79290A202024746573743D3720B7
:103E6000204D20636F64657320746573742020286F
:103E70004D20636F64657320696E7465726D696E41
:103E8000676C65642077697468206D6F7665732947
:103E90000A202024746573743D3820204A534F4E05
:103EA00020746573742020202020286D6F74696F42
:103EB0006E20746573742072756E207573696E67F9
:103EC000204A534F4E20636F6D6D616E6473290AF3
:103ED000202024746573743D392020696E766572E4
:103EE00073652074696D6520746573740A202024DD
:103EF000746573743D313020726F74617279206D16
:103F00006F74696F6E20746573740A202024746561
:103F100073743D313120736D616C6C206D6F76650B
:103F20007320746573740A202024746573743D31A2
:103F30003220736C6F77206D6F76657320746573B4
:103F4000740A202024746573743D313320636F6FCD
:103F50007264696E6174652073797374656D206F26
:103F60006666736574207465737420284739322C33
:103F7000204735342D473539290A0A54657374733F
:103F800020617373756D6520612063656E74657261
:103F90006564205859206F726967696E20616E648C
:103FA000206174206C656173742038306D6D2063FE
:103FB0006C656172616E636520696E20616C6C2056
:103FC000646972656374696F6E730A5465737473A0
:103FD00020617373756D65205A2068617320617468
:103FE000206C656173742034306D6D20706F73695F
:103FF000697469766520636C656172616E63650AD8
:104000005465737473207374617274207769746873
:104010002061204730205830205930205A30206D00
:104020006F76650A486F6D696E67206973207468E2
:104030006520657863657074696F6E2E204E6F2001
:10404000696E697469616C20706F736974696F6EF1
:10405000206F7220636C656172616E6365206973A5
:1040600020617373756D65640A000A0A0A232323AD
:104070002054696E79472053454C4620544553548B
:104080002048656C70202323230A00456163682063
:104090002420636F6D6D616E642061626F766520B0
:1040A000616C736F20646973706C617973207468DC
:1040B0006520746F6B656E20666F72206561636842
:1040C0002073657474696E6720696E205B205D20C3
:1040D000627261636B6574730A546F2076696577E9
:1040E0002073657474696E677320656E74657220E1
:1040F0006120746F6B656E3A0A0A2020243C746F4D
:104100006B656E3E0A0A466F72206578616D706C51
:1041100065202479667220746F20646973706C6105
:1041200079207468652059206D6178206665656422
:1041300020726174650A0A546F2075706461746539
:104140002073657474696E677320656E7465722080
:10415000746F6B656E20657175616C732076616C30
:1041600075653A0A0A2020243C746F6B656E3E3DEB
:104170003C76616C75653E0A0A466F72206578610F
:104180006D706C6520247966723D38303020746F14
:1041900020736574207468652059206D61782066ED
:1041A000656564207261746520746F20383030203A
:1041B0006D6D2F6D696E7574650A466F7220636F41
:1041C0006E66696775726174696F6E20646574618B
:1041D000696C73207365653A2068747470733A2F44
:1041E0002F6769746875622E636F6D2F73796E74B3
:1041F0006865746F732F54696E79472F77696B699F
:104200002F54696E79472D436F6E666967757261C9
:1042100074696F6E0A00546865736520636F6D6D15
:10422000616E6473206172652061637469766520D4
:10423000666F7220636F6E66696775726174696F0D
:104240006E3A0A2020247379732053686F772073A5
:10425000797374656D202867656E6572616C2920BD
:1042600073657474696E67730A20202431202020DE
:1042700053686F77206D6F746F722031207365748F
:1042800074696E677320286F722077686174657631
:104290006572206D6F746F7220796F752077616E13
:1042A0007420312C322C332C34290A2020247820FD
:1042B000202053686F7720582061786973207365D8
:1042C0007474696E677320286F72207768617465F3
:1042D000766572206178697320796F752077616ED9
:1042E0007420782C792C7A2C612C622C63290A207A
:1042F00020246D20202053686F7720616C6C206D26
:104300006F746F722073657474696E67730A20200E
:10431000247120202053686F7720616C6C206178B5
:1043200069732073657474696E67730A2020246F43
:1043300020202053686F7720616C6C206F66667355
:1043400065742073657474696E67730A2020242471
:1043500020202053686F7720616C6C207365747423
:10436000696E67730A2020246820202053686F77C5
:1043700020746869732068656C702073637265656A
:104380006E0A0A000A0A0A2323232054696E794719
:1043900020434F4E46494755524154494F4E2048BD
:1043A000656C70202323230A000A466F722064651F
:1043B0007461696C65642054696E794720696E6622
:1043C0006F207365653A2068747470733A2F2F6795
:1043D00069746875622E636F6D2F73796E7468658A
:1043E000746F732F54696E79472F77696B692F0A41
:1043F000466F7220746865206C6174657374206602
:1044000069726D77617265207365653A20687474AE
:1044100070733A2F2F6769746875622E636F6D2F02
:1044200073796E746865746F732F54696E79470A77
:10443000506C65617365206C6F6720616E792069CF
:10444000737375657320617420687474703A2F2FCC
:104450007777772E73796E746865746F732E636FD8
:104460006D2F666F72756D730A486176652066758B
:104470006E0A000A4E6F74653A2054696E794720BF
:1044800067656E657261746573206175746F6D61C7
:1044900074696320737461747573207265706F72D0
:1044A00074732062792064656661756C740A54685F
:1044B00069732063616E2062652064697361626C58
:1044C000656420627920656E746572696E67202468
:1044D00073763D300A536565207468652077696B93
:1044E000692062656C6F7720666F72206D6F7265F0
:1044F0002064657461696C732E0A00546865736585
:1045000020636F6D6D616E647320617265206163FD
:10451000746976652066726F6D2074686520636FBC
:104520006D6D616E64206C696E653A0A205E78205C
:10453000202020202020202020202020526573656C
:10454000742028636F6E74726F6C207829202D2080
:10455000736F6674776172652072657365740A2083
:10456000203F202020202020202020202020204DFF
:10457000616368696E6520706F736974696F6E201E
:10458000616E642067636F6465206D6F64656C2085
:1045900073746174650A20202420202020202020AC
:1045A00020202020202053686F7720616E642073C4
:1045B000657420636F6E66696775726174696F6E8A
:1045C0002073657474696E67730A2020212020208F
:1045D0002020202020202020202046656564686F50
:1045E0006C64202D2073746F70206D6F74696F6E12
:1045F00020776974686F7574206C6F73696E6720BB
:10460000706F736974696F6E0A20207E20202020ED
:104610002020202020202020204379636C65205317
:1046200074617274202D20726573746172742066D7
:10463000726F6D2066656564686F6C640A2020681F
:104640002020202020202020202020202053686FA0
:104650007720746869732068656C70207363726575
:10466000656E0A2020246820202020202020202081
:1046700020202053686F7720636F6E6669677572BC
:104680006174696F6E2068656C7020736372656514
:104690006E0A20202474657374202020202020209E
:1046A00020204C6973742073656C662D7465737477
:1046B000730A202024746573743D4E20202020202E
:1046C000202052756E2073656C662D74657374209E
:1046D0004E0A202024686F6D653D31202020202067
:1046E000202052756E206120686F6D696E672063AF
:1046F00079636C650A202024646566613D31202061
:104700002020202020526573746F726520616C6CCC
:104710002073657474696E677320746F20226661FC
:1047200063746F7279222064656661756C74730AB4
:10473000000A0A0A2323232054696E79472048651A
:104740006C70202323230A005B6A735D20206A7348
:104750006F6E2073657269616C697A652073747914
:104760006C65253964205B303D72656C61786564E9
:104770002C313D7374726963745D0A005B6A765D07
:1047800020206A736F6E20766572626F7369747928
:1047900025313564205B303D73696C656E742C3156
:1047A0003D666F6F7465722C323D6D657373616722
:1047B00065732C333D636F6E666967732C343D6C93
:1047C000696E656E756D2C353D766572626F7365C9
:1047D0005D0A005B656A5D2020656E61626C652024
:1047E0006A736F6E206D6F646525313364205B30B2
:1047F0003D746578742C313D4A534F4E5D0A000C70
:10480000590659FF58FA58F158E658DB58CF58C3A3
:1048100058B5589E588F5882587658625855584007
:10482000582C582958265817580258ED57DE57CE9D
:1048300057BC57A55788576B5752573C572B57199A
:10484000570C57FA56E056DD56DA56D756D456D19D
:1048500056CE56CB56C856C556C256BF56BC56B98C
:1048600056B656B356B056AD56AA56A756A456A13C
:10487000569E569B569856955692568F568C5689EC
:10488000568656835680567D567A5677567456719C
:10489000566E566B566856655662565F565C56594C
:1048A000565656535650564D564A564756445641FC
:1048B000563E561A56FA55E055C655AC5588556BB6
:1048C0005553553D552355FF54E254D054B0549997
:1048D0005480545E54455427540B54F353E153C34E
:1048E00053AE53AA53A653A2539E539A5396539230
:1048F000538E538A53865382537E537A5376537220
:10490000536E5354533A5327530B53F952E252C147
:1049100052B0529052705256523C522552F251C5EA
:1049200051A55183515D5136511A51FB50E150C789
:1049300050A2507950615036500A50D44F9F4F8D3D
:104940004F7B4F6C4F594F404F1E4F0C4FFA4EE864
:104950004ED64EC44EB24EA04E8E4E7C4E6A4E582F
:104960004E464E344E224E1E4E1A4E164E124E0ECD
:104970004E0A4E064E024EFE4DFA4DF64DF24DEEEB
:104980004DEA4DE64DE24DDE4DDA4DD64DD24DBEEF
:104990004DA04D844D594D344D0F4D0B4D074D03DA
:1049A0004DFF4CFB4CF74CF34CEF4CEB4CE74CE31E
:1049B0004CDF4CDB4CD74CC34CA74C8B4C6F4C534F
:1049C0004C374C1B4CFF4BE34BC74BAB4B8F4B73E4
:1049D0004B6F4B6B4B674B634B5F4B5B4B574B4387
:1049E0004B1B4BF44ACE4AA14A7B4A4E4A4A4A469E
:1049F0004A424A2F4A0E4AF9494A6F6767696E6709
:104A0000206379636C65206661696C65640050722F
:104A10006F626520656E64706F696E7420697320C3
:104A20007374617274696E6720706F696E74005080
:104A3000726F6265206379636C65206661696C657D
:104A40006400323439003234380032343700486F71
:104A50006D696E67204572726F72202D20486F6DF0
:104A6000696E67207377697463686573206D697315
:104A7000636F6E6669677572656400486F6D696E15
:104A800067204572726F72202D204E6567617469D0
:104A90007665206C61746368206261636B6F666623
:104AA00000486F6D696E67204572726F72202D200D
:104AB00054726176656C206D696E2026206D617878
:104AC00020617265207468652073616D6500486FB0
:104AD0006D696E67204572726F72202D204C617473
:104AE00063682076656C6F63697479206973207AD6
:104AF00065726F00486F6D696E67204572726F72E4
:104B0000202D205365617263682076656C6F636940
:104B10007479206973207A65726F00486F6D696ED1
:104B200067204572726F72202D20426164206F727F
:104B3000206E6F20617869732073706563696669A0
:104B4000656400486F6D696E67206379636C6520EA
:104B50006661696C65640032333900323338003283
:104B600033370032333600323335003233340032DB
:104B7000333300536F6674206C696D6974206578F7
:104B8000636565646564202D2043206D6178005362
:104B90006F6674206C696D697420657863656564FF
:104BA0006564202D2043206D696E00536F6674206C
:104BB0006C696D6974206578636565646564202D32
:104BC0002042206D617800536F6674206C696D69B6
:104BD00074206578636565646564202D2042206DCE
:104BE000696E00536F6674206C696D697420657816
:104BF000636565646564202D2041206D61780053F4
:104C00006F6674206C696D6974206578636565648E
:104C10006564202D2041206D696E00536F667420FD
:104C20006C696D6974206578636565646564202DC1
:104C3000205A206D617800536F6674206C696D692D
:104C400074206578636565646564202D205A206D45
:104C5000696E00536F6674206C696D6974206578A5
:104C6000636565646564202D2059206D617800536B
:104C70006F6674206C696D6974206578636565641E
:104C80006564202D2059206D696E00536F66742075
:104C90006C696D6974206578636565646564202D51
:104CA0002058206D617800536F6674206C696D69BF
:104CB00074206578636565646564202D2058206DD7
:104CC000696E00536F6674206C696D697420657835
:104CD0006365656465640032313900323138003211
:104CE0003137003231360032313500323134003262
:104CF0003133003231320032313100323130003262
:104D0000303900323038003230370032303600541B
:104D1000726170657A6F696420706C616E6E657225
:104D2000206661696C656420746F20636F6E7665C0
:104D3000726765004C696D69742073776974636884
:104D400020686974202D2053687574646F776E2015
:104D50006F63637572726564004D616368696E6547
:104D600020697320616C61726D6564202D20436F32
:104D70006D6D616E64206E6F742070726F63657309
:104D8000736564004D6F7665206C6573732074687D
:104D9000616E206D696E696D756D2074696D650059
:104DA0004D6F7665206C657373207468616E206D3D
:104DB000696E696D756D206C656E67746800476516
:104DC0006E657269632054696E7947206572726FEF
:104DD0007200313939003139380031393700313911
:104DE0003600313935003139340031393300313949
:104DF0003200313931003139300031383900313841
:104E00003800313837003138360031383500313824
:104E10003400313833003138320031383100313824
:104E200030005420776F726420697320696E766158
:104E30006C6964005420776F7264206973206D6917
:104E40007373696E67005220776F726420697320F4
:104E5000696E76616C6964005220776F72642069B4
:104E600073206D697373696E67005120776F726488
:104E700020697320696E76616C6964005120776FD8
:104E80007264206973206D697373696E67004C20CA
:104E9000776F726420697320696E76616C69640053
:104EA0004C20776F7264206973206D697373696E2B
:104EB00067004820776F726420697320696E76619D
:104EC0006C6964004820776F7264206973206D6993
:104ED0007373696E67004520776F72642069732071
:104EE000696E76616C6964004520776F7264206931
:104EF00073206D697373696E67004420776F726405
:104F000020697320696E76616C6964004420776F54
:104F10007264206973206D697373696E6700502035
:104F2000776F7264206973206E6F742061207661E0
:104F30006C696420746F6F6C206E756D62657200B1
:104F40005020776F7264206973206E6F7420616ED9
:104F500020696E7465676572005020776F726420F7
:104F60006973206E65676174697665005020776F9C
:104F70007264206973207A65726F005020776F72B7
:104F80006420697320696E76616C696400502077D3
:104F90006F7264206973206D697373696E67004175
:104FA00072632073706563696669636174696F6EAB
:104FB000206572726F72202D20656E64706F696E4D
:104FC00074206973207374617274696E6720706FE6
:104FD000696E74004172632073706563696669630A
:104FE0006174696F6E206572726F72202D2072611C
:104FF0006469757320617263206F7574206F662019
:10500000746F6C6572616E636500417263207370CA
:105010006563696669636174696F6E206572726F3A
:1050200072202D206D697373696E67206F666673D9
:105030006574287329004172632073706563696623
:1050400069636174696F6E206572726F72202D20C2
:105050006D697373696E6720617869732865732958
:105060000041726320737065636966696361746986
:105070006F6E206572726F72005370696E646C653A
:10508000206D757374206265207475726E696E6729
:1050900020666F72207468697320636F6D6D616E36
:1050A00064005370696E646C65206D757374206262
:1050B00065206F666620666F72207468697320636E
:1050C0006F6D6D616E64005370696E646C65205322
:1050D00020776F726420697320696E76616C6964F1
:1050E000005370696E646C65205320776F72642082
:1050F0006973206D697373696E67005370696E64BC
:105100006C652073706565642065786365656465AA
:1051100064206D6178696D756D005370696E646CA3
:10512000652073706565642062656C6F77206D69BA
:105130006E696D756D0050726F6772616D6D65643B
:1051400020706F696E742073616D652061732063D8
:10515000757272656E7420706F696E740043757439
:1051600074657220636F6D70656E736174696F6EC4
:105170002063616E6E6F7420626520656E61626C83
:105180006564005265717565737465642076656C3D
:105190006F636974792065786365656473206C69F1
:1051A0006D697473004730206F72204731206D7530
:1051B00073742062652061637469766520666F721E
:1051C0002047353300526F746172792061786573BE
:1051D0002063616E6E6F7420626520757365642054
:1051E00077697468207468697320636F6D6D616E90
:1051F0006400496E76657273652074696D65206D13
:105200006F64652063616E6E6F74206265207573D4
:1052100065642077697468207468697320636F6DB2
:105220006D616E64004665656472617465206E6FC1
:1052300074207370656369666965640053656C65A5
:105240006374656420706C616E6520697320696E9B
:1052500076616C69640053656C6563746564207085
:105260006C616E65206973206D697373696E670088
:10527000417869732074617267657420706F736917
:1052800074696F6E20697320696E76616C69640061
:10529000417869732074617267657420706F7369F7
:1052A00074696F6E206973206D697373696E67002E
:1052B000417869732069732064697361626C656405
:1052C000004178697320697320696E76616C696446
:1052D00020666F72207468697320636F6D6D616EF4
:1052E0006400417869732063616E6E6F742062653B
:1052F0002070726573656E74004178697320776FF2
:105300007264206D697373696E670047636F6465CB
:10531000206D6F64616C2067726F75702076696FA5
:105320006C6174696F6E004D20636F646520756EEB
:10533000737570706F727465640047636F64652085
:10534000636F6D6D616E6420756E737570706F72D2
:105350007465640047656E657269632047636F64B6
:105360006520696E707574206572726F72003132DB
:1053700039003132380031323700313236003132C3
:1053800035003132340031323300313232003132C3
:1053900031003132300031313900313138003131B2
:1053A00037003131360031313500313134004A5364
:1053B0004F4E20737472696E6720746F6F206C6F2C
:1053C0006E67004A534F4E20696E70757420686195
:1053D0007320746F6F206D616E79207061697273D4
:1053E000004A534F4E2073796E7461782065727253
:1053F0006F7200496E7075742076616C75652072ED
:10540000616E6765206572726F7200496E707574A7
:105410002065786365656473206D6178696D756D6D
:105420002076616C756500496E707574206C6573CB
:1054300073207468616E206D696E696D756D20767C
:10544000616C756500496E7075742065786365657B
:105450006473206D6178206C656E67746800436FBB
:105460006D6D616E64206E6F74206163636570742E
:10547000656420617420746869732074696D6500C7
:10548000506172616D657465722063616E6E6F74D8
:10549000206265207265616400506172616D65749F
:1054A000657220697320726561642D6F6E6C79007E
:1054B000556E737570706F72746564206E756D6271
:1054C0006572206F72204A534F4E207479706500C8
:1054D000426164206E756D62657220666F726D61E7
:1054E0007400496E76616C6964206F72206D616C26
:1054F000666F726D656420636F6D6D616E640055DB
:105500006E7265636F676E697A656420636F6D6D37
:10551000616E64206F7220636F6E666967206E61D2
:105520006D650047656E65726963206173736572AE
:1055300074696F6E206661696C757265004D656D8A
:105540006F7279206661756C74206465746563742C
:10555000656400537461636B206F766572666C6F6F
:105560007720646574656374656400436F6E74725C
:105570006F6C6C657220617373657274696F6E20F5
:105580006661696C7572650043616E6F6E69636117
:105590006C206D616368696E6520617373657274F8
:1055A000696F6E206661696C75726500506C616E22
:1055B0006E657220617373657274696F6E206661C7
:1055C000696C7572650053746570706572206173E3
:1055D00073657274696F6E206661696C75726500BF
:1055E000456E636F64657220617373657274696F71
:1055F0006E206661696C75726500494F2073756233
:105600002D73797374656D20617373657274696F3E
:105610006E206661696C75726500436F6E666967BE
:10562000207375622D73797374656D206173736572
:105630007274696F6E206661696C757265003839C5
:105640000038380038370038360038350038340034
:1056500038330038320038310038300037390037FD
:1056600038003737003736003735003734003733E6
:105670000037320037310037300036390036380015
:1056800036370036360036350036340036330036CD
:1056900032003631003630003539003538003537C4
:1056A00000353600353500353400353300353200ED
:1056B00035310035300034390034380034370034A7
:1056C00036003435003434003433003432003431A1
:1056D00000343000333900333800333700333600BC
:1056E00042616420737461747573207265706F72A7
:1056F000742073657474696E6700506572736973A2
:1057000074656E6365206572726F7200466C6F61BE
:1057100074206973204E414E00466C6F617420699D
:105720007320696E66696E697465004D6F766520D9
:1057300074696D65206973204E414E004D6F76652A
:105740002074696D6520697320696E66696E69747D
:10575000650047656E65726963206578636570747E
:10576000696F6E207265706F7274004661696C6556
:105770006420746F2067657420706C616E6E657252
:10578000206275666665720053797374656D206179
:105790006C61726D202D207368757474696E67205A
:1057A000646F776E00496E697469616C697A6174BF
:1057B000696F6E206661696C75726500526561641F
:1057C0002D6F6E6C79206164647265737300496E2D
:1057D00076616C6964204164647265737300446926
:1057E00076696465206279207A65726F00466C6F15
:1057F0006174696E6720706F696E74206572726F74
:105800007200496E7465726E616C2072616E6765BC
:10581000206572726F7200496E7465726E616C20E1
:105820006572726F720031390031380046756E63EF
:1058300074696F6E206973207374756262656400A9
:10584000456E746572696E6720626F6F74206C6F4D
:105850006164657200496E697469616C697A696E28
:1058600067004275666665722066756C6C202D2037
:10587000666174616C004275666665722066756C5F
:105880006C0042756666657220656D707479004EB5
:105890006F207375636820646576696365004D6188
:1058A000782066696C652073697A65206578636520
:1058B000656465640046696C65206E6F74206F7066
:1058C000656E00456E64206F662066696C650045F4
:1058D0006E64206F66206C696E650048617264209A
:1058E0007265736574005465726D696E6174656488
:1058F00000436F6D706C657465004E6F6F7000458E
:10590000616761696E004572726F72004F4B005B98
:105910007031706F665D2070776D2070686173659F
:10592000206F66662020202531352E3366205B30BF
:105930002E2E315D0A005B70317770685D207077C4
:105940006D20636377207068617365206869253115
:10595000352E3366205B302E2E315D0A005B7031B0
:1059600077706C5D2070776D20636377207068615D
:105970007365206C6F2531352E3366205B302E2EFB
:10598000315D0A005B70317773685D2070776D2040
:105990006363772073706565642068692531352EEF
:1059A00030662052504D0A005B703177736C5D2079
:1059B00070776D20636377207370656564206C6F0A
:1059C0002531352E30662052504D0A005B70316310
:1059D00070685D2070776D206377207068617365F3
:1059E000206869202531352E3366205B302E2E311C
:1059F0005D0A005B703163706C5D2070776D2063B1
:105A000077207068617365206C6F202531352E33E7
:105A100066205B302E2E315D0A005B703163736847
:105A20005D2070776D2063772073706565642068F2
:105A300069202531352E30662052504D0A005B70AA
:105A40003163736C5D2070776D20637720737065B0
:105A50006564206C6F202531352E30662052504D04
:105A60000A005B70316672715D2070776D2066721E
:105A7000657175656E63792020202531352E30667D
:105A800020487A0A0053595354454D205245414409
:105A900059004C6F6164696E6720636F6E66696759
:105AA000732066726F6D20454550524F4D00496E10
:105AB000697469616C697A696E6720636F6E666983
:105AC000677320746F2053686170656F6B6F32204D
:105AD0003530306D6D2070726F66696C65007B22A9
:105AE0006572223A7B226662223A25302E32662C7B
:105AF000227374223A25642C226D7367223A222580
:105B000073227D7D0A007B65723A7B66623A25309E
:105B10002E32662C73743A25642C6D73673A2225F5
:105B200073227D7D0A005B71765D2020717565753D
:105B300065207265706F727420766572626F73692A
:105B40007479253764205B303D6F66662C313D7378
:105B5000696E676C652C323D747269706C655D0AA4
:105B600000716F3A25640A0071693A25640A007170
:105B7000723A25640A005B73765D20207374617449
:105B80007573207265706F727420766572626F73C0
:105B9000697479253664205B303D6F66662C313D33
:105BA00066696C74657265642C323D766572626FED
:105BB00073655D0A005B73695D20207374617475A1
:105BC0007320696E74657276616C2531342E30668F
:105BD000206D730A004D6F746F7220256320706F03
:105BE00077657220656E61626C65642073746174A0
:105BF000653A25322E30660A005B257325735D20D9
:105C00006D257320706F776572206D616E616765B9
:105C10006D656E7425313064205B303D646973615D
:105C2000626C65642C313D616C77617973206F6EB5
:105C30002C323D696E206379636C652C333D776847
:105C4000656E206D6F76696E675D0A005B25732552
:105C5000735D206D257320706F6C61726974792596
:105C6000313864205B303D6E6F726D616C2C313D5C
:105C7000726576657273655D0A005B257325735DD9
:105C8000206D2573206D6963726F73746570732561
:105C9000313664205B312C322C342C385D0A005BA9
:105CA000257325735D206D25732074726176656C94
:105CB00020706572207265766F6C7574696F6E25E1
:105CC00031302E346625730A005B257325735D2001
:105CD0006D2573207374657020616E676C65253265
:105CE000302E336625730A005B257325735D206DA6
:105CF0002573206D617020746F2061786973253180
:105D00003564205B303D582C313D592C323D5A2EA4
:105D10002E2E5D0A005B6D745D20206D6F746F72B6
:105D20002069646C652074696D656F757425313404
:105D30002E3266205365630A00485D445D3F5D2056
:105D400064656700206D6D0020696E005B73745D93
:105D50002020737769746368207479706525313801
:105D600064205B303D4E4F2C313D4E435D0A005464
:105D700065737420232564206E6F7420666F756EC2
:105D8000640A004E362047393220583735205930C2
:105D9000205A300A4E3720463530302E300A4E38E1
:105DA00020473159302E3239315A2D322E3139387F
:105DB0000A4E39205837342E37363759302E303581
:105DC000385A2D322E3335350A4E3130205837347B
:105DD0002E373039592D302E3030305A2D322E3367
:105DE00037310A4E3131205837342E3532395A2D59
:105DF000322E3236340A4E3132205837342E363372
:105E00003459302E3130355A2D322E3331390A4E35
:105E10003133205837342E38343359302E3331341F
:105E20005A2D322E3138330A4E3134205837352E20
:105E300030303059302E3437315A2D322E313236FF
:105E40000A4E31352059302E3635305A2D322E310A
:105E500030300A4E3136205837342E3738335930E7
:105E60002E3433345A2D322E3133310A4E3137200D
:105E70005837342E35363659302E3231375A2D3286
:105E80002E3234340A4E3138205837342E333530E0
:105E9000592D302E3030305A2D322E3138320A4EB4
:105EA0003139205837342E3137305A2D322E313493
:105EB000340A4E3230205837342E34323959302E8D
:105EC0003235395A2D322E3136350A4E323120587C
:105ED00037342E35333359302E3336335A2D322E54
:105EE0003139310A4E3232205837342E363839594A
:105EF000302E3531395A2D322E3131340A4E32336B
:105F0000205837342E38343459302E3637345A2D01
:105F1000322E3039360A4E3234205837352E303052
:105F20003059302E3833305A2D322E3131340A4E1A
:105F300032352059312E3031305A2D322E31343411
:105F40000A4E3236205837342E37383759302E37EC
:105F500039375A2D322E3039380A4E3237205837D9
:105F6000342E36323859302E3633385A2D322E31BF
:105F700030380A4E3238205837342E3436395930BA
:105F80002E3437385A2D322E3135370A4E323920D9
:105F90005837342E33303959302E3331395A2D3267
:105FA0002E3131300A4E3330205837342E303434CD
:105FB00059302E3035335A2D322E3130380A4E3387
:105FC00031205837332E39393059302E3030305A4D
:105FD0002D322E3037370A4E3332205837332E3891
:105FE00031315A2D312E3934370A4E333320583758
:105FF000332E39373359302E3136325A2D322E3036
:1060000037390A4E3334205837342E32343359302E
:106010002E3433325A2D322E3038340A4E33352056
:106020005837342E34353959302E3634395A2D32CA
:106030002E3135370A4E3336205837342E36373620
:1060400059302E3836355A2D322E3130390A4E33EA
:1060500037205837342E38333859312E3032375AAA
:106060002D322E3131310A4E3338205837352E300B
:10607000303059312E3138395A2D322E3136300ADE
:106080004E33392059312E3336395A2D322E31398B
:10609000340A4E3430205837342E38343259312EA9
:1060A0003231315A2D322E3133340A4E34312058A8
:1060B00037342E36383459312E3035335A2D322E6E
:1060C0003132300A4E3432205837342E343231597E
:1060D000302E3739305A2D322E3137360A4E34337E
:1060E000205837342E33313659302E3638345A2D25
:1060F000322E3133370A4E3434205837342E31356E
:106100003859302E3532365A2D322E3037370A4E26
:106110003435205837332E39343759302E33313611
:106120005A2D322E3036370A4E3436205837332E19
:1061300038393459302E3236335A2D322E303436E7
:106140000A4E3437205837332E37333759302E31F3
:1061500030355A2D312E3931380A4E3438205837DF
:10616000332E36333159302E3030305A2D312E38CF
:1061700037320A4E3439205837332E3435325A2DBF
:10618000312E3831350A4E3530205837332E3636D9
:106190003559302E3231345A2D312E3931340A4EA0
:1061A0003531205837332E38323559302E33373485
:1061B0005A2D322E3032380A4E3532205837332E8F
:1061C00038373959302E3432375A2D322E3037364F
:1061D0000A4E3533205837342E30393259302E3666
:1061E00034315A2D322E3039340A4E353420583756
:1061F000342E33303659302E3835345A2D322E3134
:1062000039320A4E3535205837342E353139593127
:106210002E3036385A2D322E3134310A4E35362052
:106220005837342E37333359312E3238315A2D32D4
:106230002E3134330A4E3537205837342E38343027
:1062400059312E3338385A2D322E3137340A4E35E3
:1062500038205837342E38393359312E3434325AA5
:106260002D322E3136390A4E3539205837352E30F9
:10627000303059312E3534385A2D322E3132310AE0
:106280004E36302059312E3732385A2D322E303793
:10629000360A4E3631205837342E38343359312EA1
:1062A0003537315A2D322E3133300A4E363220589E
:1062B00037342E37333859312E3436365A2D322E64
:1062C0003139350A4E3633205837342E3437365963
:1062D000312E3230345A2D322E3134370A4E363484
:1062E000205837342E32313559302E3934335A2D27
:1062F000322E3230320A4E3635205837332E39306E
:106300003059302E3632385A2D322E3130310A4E35
:106310003636205837332E38343859302E35373604
:106320005A2D322E3039360A4E3637205837332E12
:1063300035383659302E3331345A2D312E393133E8
:106340000A4E3638205837332E33373759302E31EE
:1063500030355A2D312E3830380A4E3639205837DC
:10636000332E32373259302E3030305A2D312E37CD
:1063700038370A4E3730205837332E3138325A2DBD
:10638000312E3738370A4E3731205837332E3039CF
:10639000325A2D312E3735300A4E373220583733A6
:1063A0002E34313059302E3331385A2D312E383683
:1063B000380A4E3733205837332E37383159302E7C
:1063C0003638395A2D322E3038360A4E3734205866
:1063D00037342E30393959312E3030375A2D322E4C
:1063E0003232340A4E3735205837342E3230355950
:1063F000312E3131335A2D322E3231310A4E373669
:10640000205837342E33363459312E3237325A2D04
:10641000322E3137360A4E3737205837342E36323F
:106420003959312E3533375A2D322E3139310A4E02
:106430003738205837342E36383259312E353930E6
:106440005A2D322E3137370A4E3739205837342EED
:1064500038393459312E3830325A2D322E303636C2
:106460000A4E3830205837352E30303059312E39D9
:1064700030385A2D322E3034360A4E3831205932C7
:106480002E3038375A2D322E3035310A4E383220E0
:106490005837342E38333959312E3932375A2D3254
:1064A0002E3036320A4E3833205837342E363739AC
:1064B00059312E3736365A2D322E3133360A4E3870
:1064C00034205837342E36323559312E3731335A3D
:1064D0002D322E3137300A4E3835205837342E358C
:1064E000373259312E3635395A2D322E3138300A5D
:1064F0004E3836205837342E33353859312E34340F
:10650000355A2D322E3135370A4E38372058373428
:106510002E31393759312E3238345A2D322E313905
:10652000350A4E3838205837342E30393059312E0C
:106530003137375A2D322E3234350A4E38392058F9
:1065400037332E39383359312E3037305A2D322ED9
:106550003232350A4E3930205837332E38323359DB
:10656000302E3931305A2D322E3133380A4E3931EE
:10657000205837332E33393459302E3438325A2D8F
:10658000312E3931370A4E3932205837332E3138CF
:106590003059302E3236385A2D312E3832350A4E97
:1065A0003933205837322E39363659302E3035347B
:1065B0005A2D312E3731310A4E3934205837322E88
:1065C000393133592D302E3030305A2D312E363965
:1065D000330A4E3935205837322E3733335A2D315E
:1065E0002E3634360A4E3936205837322E3939375E
:1065F00059302E3236345A2D312E3735330A4E3932
:1066000037205837332E32363059302E3532375AFC
:106610002D312E3930320A4E3938205837332E3644
:10662000323959302E3839365A2D322E3037370A12
:106630004E3939205837332E38343059312E3130D5
:10664000375A2D322E3232340A4E313030205837FC
:10665000332E38393359312E3136305A2D322E32CD
:1066600034350A4E3130312058373559305A300AD6
:10667000004E312054314D360A4E32204731370A10
:106680004E33204732310A4E382046313830300AF6
:106690004E392047310A4E313030204739322058A8
:1066A0002D32352E313737592D33342E30373220B5
:1066B0005A2D312E303030202854454D502C205248
:1066C000454D4F5645204C41544552290A4E3334CE
:1066D0003320582D32352E353935592D33342E335C
:1066E00034390A4E33343420582D32352E37303178
:1066F000592D33342E3433360A4E33343520582D49
:1067000032352E373931592D33342E3532300A4E49
:1067100033343620582D32352E383634592D333413
:106720002E3630310A4E33343720582D32352E393B
:106730003230592D33342E3637390A4E333438201F
:10674000582D32352E393630592D33342E373534D5
:106750000A4E33343920582D32352E393832592DDE
:1067600033342E3832360A4E33353020582D3235F8
:106770002E393837592D33342E3839350A4E3335C2
:106780003120582D32352E393736592D33342E39A4
:1067900036310A4E33353220582D32352E393438C1
:1067A000592D33352E3032330A4E33353320582DA0
:1067B00032352E393033592D33352E3038320A4E9A
:1067C00033353420582D32352E383431592D333568
:1067D0002E3133380A4E33353520582D32352E3789
:1067E0003633592D33352E3139300A4E3335362074
:1067F000582D32352E363639592D33352E32333920
:106800000A4E33353720582D32352E353539592D2E
:1068100033352E3238340A4E33353820582D323540
:106820002E343333592D33352E3332350A4E33352A
:106830003920582D32352E323931592D33352E33FA
:1068400036330A4E33363020582D32352E3133341C
:10685000592D33352E3339370A4E33363120582DE2
:1068600032342E393633592D33352E3432380A4EE0
:1068700033363220582D32342E373737592D3335B1
:106880002E3435350A4E33363320582D32342E35DA
:106890003737592D33352E3437370A4E33363420B7
:1068A000582D32342E333637592D33352E34393670
:1068B0000A4E33363520582D32342E313434592D8A
:1068C00033352E3531310A4E33363620582D32339A
:1068D0002E393039592D33352E3532320A4E333672
:1068E0003720582D32332E363631592D33352E354B
:1068F00032390A4E33363820582D32332E34303365
:10690000592D33352E3533320A4E33363920582D32
:1069100032332E313333592D33352E3533320A4E3F
:1069200033373020582D32322E383533592D333508
:106930002E3532370A2F4E32353138204730583015
:106940002E333237592D33332E3532315A2D312EE5
:106950003030300A4E32353139204D3330004E312F
:10696000204732300A4E3520473430204731370A2D
:106970004E3130205431204D30360A284E313520EA
:10698000473930204730205830205930205A30299C
:106990000A4E3230205335303030204D3033200A0B
:1069A0004E32352058302E3036342059302E333286
:1069B00036205A300A4E34302047303120463136A6
:1069C0002E300A4E35302058302E30363420593093
:1069D0002E3332360A4E35352058302E30363020A0
:1069E00059302E3239330A4E36302058302E303757
:1069F000372059302E3236370A4E36352058302E51
:106A00003131312059302E3235370A4E3730205847
:106A1000302E3134392059302E3235320A4E373546
:106A20002058302E3138382059302E3235350A4E24
:106A300038302058302E3232372059302E32363806
:106A40000A4E38352058302E3235372059302E3204
:106A500037310A4E39302058302E333335205930F3
:106A60002E3236350A4E39352058302E3431322008
:106A700059302E3237310A4E3130302058302E34D2
:106A800037342059302E3238370A4E3130352058BD
:106A9000302E3439312059302E3238390A4E3131C6
:106AA000302058302E3531372059302E3237330AC6
:106AB0004E3131352058302E3534342059302E3275
:106AC00036330A4E3132302058302E353830205986
:106AD000302E3236310A4E3132352058302E35398B
:106AE000352059302E3236330A4E3133302058306B
:106AF0002E3632312059302E3237340A4E3133356A
:106B00002058302E3635392059302E3330360A4E43
:106B10003134302058302E3637332059302E33332D
:106B2000350A4E3134352058302E36373920593019
:106B30002E3336310A4E3135302058302E36373824
:106B40002059302E3338390A4E3135352058302E01
:106B50003637302059302E3432300A4E313630201C
:106B600058302E3637302059302E3434360A4E31D4
:106B700036352058302E3638302059302E343734C0
:106B80000A4E3137302058302E3730342059302ECD
:106B90003439370A4E3137352058302E37333220CA
:106BA00059302E3531350A4E3138302058302E3795
:106BB00039342059302E3533350A4E313835205886
:106BC000302E3837322059302E3536370A4E31398B
:106BD000302058302E3935302059302E3630340A96
:106BE0004E3139352058312E3033312059302E3640
:106BF00034370A4E3230302058312E313439205952
:106C0000302E3732320A4E3230352058312E333062
:106C1000382059302E3835340A4E32313020583130
:106C20002E3433302059302E3938340A4E32313533
:106C30002058312E3434372059302E3938360A4E08
:106C40003232302058312E3632382059302E3832F8
:106C5000320A4E3232352058312E373332205930F5
:106C60002E3731340A4E3233302058322E303039FC
:106C70002059302E3338310A4E3233352058322ED7
:106C80003131362059302E3236360A4E32343020E9
:106C900058322E3232382059302E3135370A4E32A2
:106CA00034352058322E3238302059302E3132339C
:106CB0000A4E3235302058322E3333322059302E9E
:106CC0003039340A4E3235352058322E34323320A2
:106CD00059302E3037300A4E3236302058322E346A
:106CE00038392059302E3036350A4E323635205854
:106CF000322E3535372059302E3036360A4E32375F
:106D0000302058322E3632372059302E3038340A5F
:106D10004E3237352058322E3639332059302E3105
:106D200030390A4E3238302058322E37333020591D
:106D3000302E3133330A4E3238352058322E383027
:106D4000352059302E3139300A4E32393020583200
:106D50002E3832392059302E3231360A4E323935FA
:106D60002058322E3838302059302E3239310A4EE0
:106D70003330302058322E3838342059302E3330CA
:106D8000300A4E3330352058322E383938205930B9
:106D90002E3333320A4E3331302058322E393035CB
:106DA0002059302E3336370A4E3331352058322EA3
:106DB0003931302059302E3430370A4E33323020BA
:106DC00058322E3930382059302E3434360A4E336A
:106DD00032352058322E3930312059302E34393561
:106DE0000A4E3333302058322E3839372059302E5E
:106DF0003439350A4E3333352058322E3839302065
:106E000059302E3532340A4E3334302058322E3831
:106E100034322059302E3630340A4E33343520582F
:106E2000322E3831342059302E3636350A4E33352D
:106E3000302058322E3739342059302E3735300A29
:106E40004E3335352058322E3739312059302E38CF
:106E500033380A4E3336302058322E3831392059E3
:106E6000302E3937360A4E3336352058322E3833E5
:106E7000372059312E3034340A4E333730205832CF
:106E80002E3836322059312E3131320A4E333735D1
:106E90002058322E3837372059312E3134350A4EAA
:106EA0003338302058322E3931322059312E323198
:106EB000370A4E3338352058322E39313720593180
:106EC0002E3232360A4E3339302058322E3935318F
:106ED0002059312E3238310A4E3339352058322E6E
:106EE0003937302059312E3239350A4E343030207E
:106EF00058322E3939362059312E3239350A4E342E
:106F000030352058332E3031332059312E32373539
:106F10000A4E3431302058332E3032342059312E3D
:106F20003235340A4E3431352058332E3037302044
:106F300059312E3135310A4E3432302058332E300B
:106F400037372059312E3133340A4E3432352058F8
:106F5000332E3132352059312E3033390A4E343305
:106F6000302058332E3133382059312E3031390A00
:106F70004E3433352058332E3230352059302E39A7
:106F800030380A4E3434302058332E3238322059BB
:106F9000302E3739370A4E3434352058332E3336B5
:106FA000312059302E3639310A4E3435302058339D
:106FB0002E3432362059302E3539320A4E3435359A
:106FC0002058332E3435362059302E3534330A4E7E
:106FD0003436302058332E3437392059302E343956
:106FE000330A4E3436352058332E34393420593054
:106FF0002E3437320A4E3437302058332E35303560
:107000002059302E3434360A4E3437352058332E3A
:107010003531382059302E3431370A4E343830204B
:1070200058332E3533302059302E3339310A4E340F
:1070300038352058332E3536342059302E33303001
:107040000A4E3439302058332E3537372059302EF8
:107050003235330A4E3439352058332E3536382000
:1070600059302E3231320A4E3530302058332E35D9
:1070700034342059302E3137360A4E3530352058C9
:10708000332E3534312059302E3134360A4E3531D5
:10709000302058332E3535332059302E3131390ACE
:1070A0004E3531352058332E3537362059302E3174
:1070B00030360A4E3532302058332E353937205984
:1070C000302E3130320A4E3532352058332E36319B
:1070D000382059302E3130390A4E3533302058336C
:1070E0002E3633392059302E3132390A4E35333568
:1070F0002058332E3635302059302E3135390A4E4E
:107100003534302058332E3636332059302E31372F
:10711000380A4E3534352058332E3637382059301A
:107120002E3139320A4E3535302058332E36393922
:107130002059302E3139370A4E3535352058332E07
:107140003732332059302E3139360A4E3536302019
:1071500058332E3736342059302E3137390A4E35D0
:1071600036352058332E3830352059302E313635CB
:107170000A4E3537302058332E3838342059302EC7
:107180003135390A4E3537352058332E39343920C8
:1071900059302E3136350A4E3538302058332E3995
:1071A00036362059302E3137350A4E35383520588D
:1071B000332E3937382059302E3139340A4E35398B
:1071C000302058332E3937382059302E3232330A96
:1071D0004E3539352058332E3936302059302E323D
:1071E00034350A4E3630302058332E383334205957
:1071F000302E3331310A4E3630352058332E373663
:10720000322059302E3334350A4E3631302058333F
:107210002E3732362059302E3338390A4E36313532
:107220002058332E3730332059302E3435380A4E1B
:107230003632302058332E3638322059302E3533FE
:10724000300A4E3632352058332E363739205930F1
:107250002E3533340A4E3633302058332E363236FC
:107260002059302E3638310A4E3633352058332ED9
:107270003536382059302E3832380A4E36343020E0
:1072800058332E3434342059312E3038300A4E36AB
:1072900034352058332E3430352059312E3136379D
:1072A0000A4E3635302058332E3430342059312EA2
:1072B0003136370A4E3635352058332E333837209D
:1072C00059312E3230380A4E3636302058332E336C
:1072D00038342059312E3230380A4E36363520585F
:1072E000332E3336352059312E3236350A4E363765
:1072F000302058332E3335352059312E3238350A67
:107300004E3637352058332E3334382059312E330A
:1073100030380A4E3638302058332E333333205924
:10732000312E3335300A4E3638352058332E33322D
:10733000312059312E3339310A4E36393020583305
:107340002E3331312059312E3432380A4E36393508
:107350002058332E3333392059312E3432330A4EEC
:107360003730302058332E3434302059312E3430D9
:10737000360A4E3730352058332E353130205931CA
:107380002E3430380A4E3731302058332E353835C8
:107390002059312E3432310A4E3731352058332EB0
:1073A0003631312059312E3433390A4E37323020BC
:1073B00058332E3631312059312E3434310A4E377C
:1073C00032352058332E3631352059312E34343170
:1073D0000A4E3733302058332E3633362059312E6B
:1073E0003438380A4E3733352058332E363334206C
:1073F00059312E3531370A4E3734302058332E3636
:1074000032322059312E3534330A4E373435205834
:10741000332E3630352059312E3536330A4E373536
:10742000302058332E3537362059312E3537350A2E
:107430004E3735352058332E3534342059312E35DA
:1074400038310A4E3736302058332E3437392059E8
:10745000312E3539320A4E3736352058332E3435F1
:10746000312059312E3539380A4E373730205833CC
:107470002E3338372059312E3632360A4E373735CB
:107480002058332E3339302059312E3633360A4EB8
:107490003738302058332E3533322059312E36309C
:1074A000320A4E3738352058332E36303120593194
:1074B0002E3539370A4E3739302058332E36363884
:1074C0002059312E3539380A4E3739352058332E68
:1074D0003738322059312E3631320A4E383030208A
:1074E00058332E3739342059312E3631380A4E3838
:1074F00030352058332E3836382059312E36333631
:107500000A4E3831302058332E3931382059312E37
:107510003635350A4E3831352058332E393435203A
:1075200059312E3636370A4E3832302058332E39FC
:1075300036342059312E3638350A4E3832352058F7
:10754000332E3936372059312E3638350A4E3833F6
:10755000302058332E3937342059312E3639390AF4
:107560004E3833352058332E3938342059312E37A0
:1075700032350A4E3834302058332E3938342059B9
:10758000312E3735380A4E3834352058332E3937B6
:10759000302059312E3739300A4E383530205833A3
:1075A0002E3934352059312E3831370A4E38353599
:1075B0002058332E3931382059312E3832360A4E80
:1075C0003836302058332E3839312059312E383260
:1075D000370A4E3836352058332E38343220593158
:1075E0002E3830390A4E3837302058332E37393854
:1075F0002059312E3738340A4E3837352058332E3B
:107600003734362059312E3737320A4E3838302049
:1076100058332E3639382059312E3736340A4E3801
:1076200038352058332E3633352059312E373636FB
:107630000A4E3839302058332E3535332059312E03
:107640003738350A4E3839352058332E34373820FC
:1076500059312E3832300A4E3930302058332E34DA
:1076600030392059312E3836340A4E3930352058C9
:10767000332E3334352059312E3931380A4E3931D1
:10768000302058332E3236342059322E3032330ADD
:107690004E3931352058332E3234382059322E307D
:1076A00035310A4E3932302058332E323430205999
:1076B000322E3038310A4E3932352058332E33319C
:1076C000362059322E3038360A4E3933302058336E
:1076D0002E3339302059322E3130340A4E39333579
:1076E0002058332E3431342059322E3132310A4E63
:1076F0003934302058332E3433312059322E31353D
:10770000330A4E3934352058332E3433332059322E
:107710002E3138300A4E3935302058332E34323736
:107720002059322E3230350A4E3935352058332E15
:107730003431332059322E3232340A4E3936302029
:1077400058332E3339322059322E3234320A4E39E0
:1077500036352058332E3333352059322E323434D7
:107760000A4E3937302058332E3237382059322ECE
:107770003233360A4E3937352058332E32353620DB
:1077800059322E3234320A4E3938302058332E32A4
:1077900033392059322E3235310A4E393835205896
:1077A000332E3231312059322E3238300A4E3939A7
:1077B000302058332E3137342059322E3335360AA3
:1077C0004E3939352058332E3135392059322E3340
:1077D00039370A4E313030302058332E3135302091
:1077E00059322E3433380A4E313030352058332E4A
:1077F0003134302059322E3438310A4E3130313064
:107800002058332E3133322059322E3531300A4E42
:10781000313031352058332E3131382059322E3520
:1078200034330A4E313032302058332E303939203B
:1078300059322E3537360A4E313032352058332EF4
:107840003035312059322E3633310A4E3130333013
:107850002058332E3030332059322E3636360A4EE9
:10786000313033352058322E3935372059322E36C3
:1078700038350A4E313034302058322E39303720E6
:1078800059322E3639390A4E313034352058322E9D
:107890003836302059322E3731310A4E31303530BA
:1078A0002058322E3831392059322E3732370A4E8D
:1078B000313035352058322E3736382059322E3770
:1078C00034350A4E313036302058322E373136209A
:1078D00059322E3735370A4E313036352058322E50
:1078E0003637352059322E3735370A4E313037305A
:1078F0002058322E3537392059322E3733310A4E3F
:10790000313037352058322E3537302059322E3726
:1079100032330A4E313038302058322E3535392046
:1079200059322E3732300A4E313038352058322E07
:107930003533302059322E3730310A4E313039301C
:107940002058322E3530312059322E3639330A4EF6
:10795000313039352058322E3437312059322E36D5
:1079600038330A4E313130302058322E34343320FF
:1079700059322E3636380A4E313130352058322EB3
:107980003339362059322E3633340A4E31313130C4
:107990002058322E3335342059322E3539310A4EA3
:1079A000313131352058322E3335322059322E358F
:1079B00039310A4E313132302058322E33323520AF
:1079C00059322E3534330A4E313132352058322E69
:1079D0003331352059322E3532310A4E3131333080
:1079E0002058322E3330372059322E3439380A4E4F
:1079F000313133352058322E3239362059322E3437
:107A000036340A4E313134302058322E3239332058
:107A100059322E3432370A4E313134352058322E15
:107A20003239352059322E3336360A4E313135301F
:107A30002058322E3332312059322E3330330A4E11
:107A4000313135352058322E3335382059322E32E7
:107A500034370A4E313136302058322E3431392005
:107A600059322E3230330A4E313136352058322ECB
:107A70003431392059322E3137390A4E31313730CD
:107A80002058322E3430352059322E3135380A4EB6
:107A9000313137352058322E3336322059322E319B
:107AA00032330A4E313138302058322E33353420BB
:107AB00059322E3130340A4E313138352058322E79
:107AC0003335342059322E3039310A4E3131393084
:107AD0002058322E3338302059322E3036350A4E67
:107AE000313139352058322E3431302059322E3050
:107AF00035310A4E313230302058322E3431302078
:107B000059322E3034370A4E313230352058322E29
:107B10003430352059322E3032380A4E313231303D
:107B20002058322E3430382059322E3031300A4E1F
:107B3000313231352058322E3431362059312E39F8
:107B400039350A4E313232302058322E3433332018
:107B500059312E3938320A4E313232352058322ED0
:107B60003433382059312E3936330A4E31323330DE
:107B70002058322E3434372059312E3934380A4EB9
:107B8000313233352058322E3436312059312E39A6
:107B900033380A4E313234302058322E34383020C7
:107BA00059312E3933310A4E313234352058322E84
:107BB0003437382059312E3839390A4E3132353080
:107BC0002058322E3438372059312E3837350A4E66
:107BD000313235352058322E3530342059312E3857
:107BE00035340A4E313236302058322E3532372075
:107BF00059312E3834380A4E313236352058322E2B
:107C00003534392059312E3834390A4E3132373033
:107C10002058322E3537372059312E3836310A4E1A
:107C2000313237352058322E3630342059312E3803
:107C300036360A4E313238302058322E3633312023
:107C400059312E3835340A4E313238352058322EDB
:107C50003634302059312E3832370A4E31323930ED
:107C60002058322E3634302059312E3739320A4ED0
:107C7000313239352058322E3632392059312E37AB
:107C800035390A4E313330302058322E36313220D9
:107C900059312E3732370A4E313330352058322E93
:107CA0003537362059312E3639340A4E313331309A
:107CB0002058322E3533362059312E3636320A4E80
:107CC000313331352058322E3437302059312E3669
:107CD00031360A4E313332302058322E333435208B
:107CE00059312E3535310A4E313332352058322E46
:107CF0003330372059312E3532310A4E313333305B
:107D00002058322E3236302059312E3438320A4E35
:107D1000313333352058322E3234332059312E341A
:107D200037370A4E313334302058322E3232382031
:107D300059312E3436390A4E313334352058322EEB
:107D40003232322059312E3434380A4E3133353004
:107D50002058322E3232382059312E3432350A4EE4
:107D6000313335352058322E3235342059312E34C6
:107D700030350A4E313336302058322E32363820E4
:107D800059312E3337330A4E313336352058322E9F
:107D90003237392059312E3334320A4E31333730AD
:107DA0002058322E3330382059312E3238370A4E8F
:107DB000313337352058322E3334302059312E327A
:107DC00035340A4E313338302058322E3430372093
:107DD00059312E3230310A4E313338352058322E57
:107DE0003434312059312E3135360A4E3133393061
:107DF0002058322E3435342059312E3133310A4E49
:107E0000313339352058322E3436302059312E3125
:107E100030360A4E313430302058322E3436342049
:107E200059312E3130320A4E313430352058322E0D
:107E30003437312059312E3033360A4E3134313017
:107E40002058322E3436362059302E3937310A4EEA
:107E5000313431352058322E3435312059302E38D6
:107E600039370A4E313432302058322E34313520F1
:107E700059302E3739310A4E313432352058322EAE
:107E80003430332059302E3736370A4E31343330C0
:107E90002058322E3338382059302E3736350A4E96
:107EA000313433352058322E3330362059302E3885
:107EB00034310A4E313434302058322E32323220AE
:107EC00059302E3931310A4E313434352058322E62
:107ED0003131342059302E3939350A4E313435306C
:107EE0002058322E3030322059312E3037360A4E5B
:107EF000313435352058312E3930352059312E3135
:107F000033390A4E313436302058312E373534204B
:107F100059312E3232330A4E313436352058312E13
:107F20003633372059312E3237380A4E3134373014
:107F30002058312E3538322059312E3330310A4E07
:107F4000313437352058312E3535382059312E33DC
:107F500031350A4E313438302058312E3436302005
:107F600059312E3335320A4E313438352058312EBE
:107F70003339392059312E3336300A4E31343930C5
:107F80002058312E3333382059312E3335340A4EB0
:107F9000313439352058312E3238372059312E338B
:107FA00032390A4E313530302058312E32343820B3
:107FB00059312E3239340A4E313530352058312E70
:107FC0003231372059312E3235340A4E3135313085
:107FD0002058312E3231342059312E3235320A4E6A
:107FE000313531352058312E3137322059312E314B
:107FF00039350A4E313532302058312E3132382061
:1080000059312E3133390A4E313532352058312E1F
:108010003131302059312E3131370A4E313533303C
:108020002058302E3935382059302E3934310A4E07
:10803000313533352058302E3839312059302E38EB
:1080400037330A4E313534302058302E383235200F
:1080500059302E3830380A4E313534352058302ECC
:108060003735352059302E3734370A4E31353530D3
:108070002058302E3631392059302E3633330A4EBF
:10808000313535352058302E3437372059302E359C
:1080900032360A4E313536302058302E34373720BC
:1080A00059302E3532340A4E313536352058302E7F
:1080B0003431312059302E3437360A4E313537308D
:1080C0002058302E3333312059302E3435340A4E77
:1080D000313537352058302E3237382059302E344C
:1080E00032370A4E313538302058302E3233312075
:1080F00059302E3339370A4E313538352058302E25
:108100003138332059302E3337390A4E3135393032
:108110002058302E3133352059302E3336350A4E23
:10812000313539352058302E3037362059302E33FE
:1081300034310A4E31363035204730302046333026
:108140002E300A4E31363130204D3035200A4E3136
:1081500036313520473930205830205930205A30B8
:108160000A4E31363135204D33300A28456E6420B1
:108170006F6620434E432050726F6772616D290015
:10818000284D53472A2A2A2A204D6963726F737437
:1081900065702054657374205B76315D202A2A2A2D
:1081A0002A290A47303020473137204732312047CB
:1081B00034302047343920473830204739300A6777
:1081C00030783079307A300A7B22316D69223A3149
:1081D0007D0A7B22326D69223A317D0A7B22336D22
:1081E00069223A317D0A7B22346D69223A317D0A57
:1081F0006730207831300A7B22316D69223A327D36
:108200000A78300A7B22316D69223A347D0A78314E
:10821000300A7B22316D69223A387D0A78300A674C
:1082200030207931300A7B22326D69223A327D0A60
:1082300079300A7B22326D69223A347D0A793130F5
:108240000A7B22326D69223A387D0A79300A67301A
:10825000207A31300A7B22336D69223A327D0A7AE4
:10826000300A7B22336D69223A347D0A7A31300A32
:108270007B22336D69223A387D0A7A300A673020D2
:108280006131300A7B22346D69223A327D0A6130D5
:108290000A7B22346D69223A347D0A6131300A7BCF
:1082A00022346D69223A387D0A61300A6D32002825
:1082B0004D53472A2A2A2A20436F6F7264696E61E0
:1082C0007465206F666673657473207465737420BB
:1082D0005B76315D202A2A2A2A290A6730306731E5
:1082E000376732316734306734396738306739304F
:1082F0000A6735340A673932783079307A300A665D
:108300003630300A284D53472A2A2A2A20746573AA
:108310007420473932206F6666736574732A2A2A7F
:108320002A290A286D73675374657020313A204DED
:108330006F76652066726F6D20302C3020746F2050
:1083400033302C30206D6D20696E20706F7369742E
:10835000697665205820646972656374696F6E2957
:108360000A286D73675374657020323A2052657322
:108370006574206F726967696E20746F20302E30CB
:10838000207573696E6720473932290A286D736733
:108390005374657020333A204D6F766520746F20DA
:1083A00032302C302E2053686F756C64206D6F76E0
:1083B00065203230206D6D20696E20706F73697496
:1083C000697665205820646972656374696F6E20F0
:1083D000616E6420737461747573207265706F725E
:1083E000742073686F756C64207374617274206696
:1083F000726F6D20302C30290A286D7367537465B5
:108400007020343A204D6F766520746F20302E3006
:1084100020202053686F756C64206D6F7665203264
:1084200030206D6D20696E206E65676174697665B8
:10843000205820646972656374696F6E20616E6490
:1084400020737461747573207265706F7274207319
:10845000686F756C642073746172742066726F6DDE
:108460002032302C30290A67317833300A673932AC
:1084700078300A67317832300A6731783079300ADB
:108480002473720A67393278300A673470302E35B7
:108490000A284D53472A2A2A2A20746573742047D4
:1084A0003535206F6666736574732A2A2A2A290A6D
:1084B000286D73675374657020313A2053657420BA
:1084C000436F6F7264696E6174652073797374654C
:1084D0006D2032205B6735355D20746F206F6666D6
:1084E000736574206F662035302C3530290A286D6D
:1084F00073675374657020323A2053656C656374FA
:108500002047353520636F6F7264696E6174652032
:1085100073797374656D290A286D73675374657078
:1085200020333A204D6F766520746F20302C302E2A
:1085300020486561642073686F756C64206D6F7688
:108540006520646961676F6E616C6C7920696E206B
:108550002B5820616E64202B5920616E6420737447
:1085600061747573207265706F72742073686F75B3
:108570006C642073746172742066726F6D20302C8D
:1085800030290A6731304C327032783530793530E5
:108590000A6735350A6730783079300A67347030C9
:1085A0002E350A284D53472A2A2A2A2074657374C7
:1085B00020473533206162736F6C757465206F7668
:1085C00065727269646573202A2A2A2A290A286D2D
:1085D00073675374657020313A2052756E206120A4
:1085E00073717561726520696E2047353520737926
:1085F0007374656D290A286D736753746570203232
:108600003A2052756E206120737175617265207712
:108610002F473533206F76657272696465290A6762
:1086200030783079300A673078323079300A673004
:108630007832307932300A673078307932300A67F0
:1086400030783079300A673470302E350A67353328
:108650006730783079300A6735336730783230796F
:10866000300A67353367307832307932300A67350F
:1086700033673078307932300A6735336730783095
:1086800079300A6730783079300A673470302E35A7
:108690000A284D53472A2A2A2A20746573742052C7
:1086A000657475726E20746F20686F6D65202A2A5C
:1086B0002A2A290A286D73675374657020313A207D
:1086C00052657475726E20746F20686F6D652075C9
:1086D00073696E6720473238290A286D73675374AF
:1086E000657020323A20526573657420746F20479C
:1086F000353420636F6F72642073797374656D29EC
:108700000A6732380A6735340A6D333000284D5312
:10871000472A2A2A2A20546573742061636375727C
:10872000616379206F6620736C6F77206D6F76655B
:1087300073205B76315D202A2A2A2A290A6735357B
:108740000A6730783079300A673470302E350A671E
:108750003470302E350A67317831306632320A672C
:1087600035340A6730783079300A6D333000284D5F
:1087700053472A2A2A2A2054657374207665727911
:108780002073686F7274206D6F766573205B76312D
:108790005D202A2A2A2A290A6730783079300A6728
:1087A0003470302E350A673178302E3166313030F2
:1087B000300A78300A78302E310A78300A78302E34
:1087C000310A78300A78302E310A78300A78302E23
:1087D000310A78300A78302E310A78300A78302E13
:1087E000310A78300A78302E310A78300A78302E03
:1087F000310A78300A78302E310A78300A78302EF3
:10880000310A78300A78302E310A78300A78302EE2
:10881000310A78300A78302E310A78300A78302ED2
:10882000310A673470302E350A78300A78302E30AD
:10883000310A78300A78302E30310A78300A7830B0
:108840002E30310A78300A78302E30310A78300AEA
:1088500078302E30310A78300A78302E30310A786C
:10886000300A78302E30310A78300A78302E3031A4
:108870000A78300A78302E30310A78300A78302E73
:1088800030310A78300A78302E30310A78300A7860
:10889000302E30310A78300A78302E30310A783074
:1088A0000A78302E30310A6730783079300A6D32EC
:1088B00000284D53472A2A2A2A20526F7461727960
:1088C0002041786973204D6F74696F6E2054657311
:1088D00074205B76315D202A2A2A2A290A673030E3
:1088E000673137673231673430673439673830671A
:1088F00039300A6730783079307A306130623063ED
:10890000300A6735350A6730783079300A66333691
:108910003030300A6730613336300A623336300A1D
:10892000633336300A61300A62300A63300A6731D5
:1089300061313434300A62313434300A63313434D2
:10894000300A61300A62300A63300A6731613134BB
:10895000343062373230633336300A783079307AE7
:10896000306130623063300A6731783630613134DB
:10897000343062373230633336300A783079307AC7
:10898000306130623063300A6731783630793530A3
:10899000613134343062373230633336300A783004
:1089A00079307A306130623063300A67317836303E
:1089B0007935307832356131343430623732306372
:1089C0003336300A783079307A3061306230633053
:1089D0000A6735340A6730783079300A6D333000F1
:1089E000284D53472A2A2A2A20496E7665727365D4
:1089F0002054696D65204D6F74696F6E20546573E6
:108A000074205B76315D202A2A2A2A290A673030B1
:108A100067313767323167343067343967383067E8
:108A200039300A6735350A6730783079300A673966
:108A3000330A66302E30310A67317831300A7931A5
:108A4000300A7A31300A6131300A78300A79300AD6
:108A50007A300A61300A67317831307931307A2DD5
:108A600031306131300A6730783079307A306130B6
:108A70000A66302E310A6732783130792D31307AFA
:108A80002D32306931300A6730783079307A300AE7
:108A90006733783130792D31307A2D323069313089
:108AA0000A6730783079307A300A67327832307934
:108AB000307A2D32306931300A6730783079307A47
:108AC000300A673378323079306931300A6730786C
:108AD0003079307A300A6732783079307A2D333015
:108AE0006931300A6733783079307A306931300A49
:108AF0006730783079307A300A6732783079306987
:108B00003230202843572033363020646567726541
:108B10006573290A67337830793069323020284309
:108B20004357203336302064656772656573290AC0
:108B30006739340A6735340A6730783079300A6D1E
:108B40003330007B226763223A2267303067313747
:108B500067323167343067343967383067393022EB
:108B60007D0A7B226763223A22673535227D0A7BA4
:108B7000226763223A22673078307930227D0A7B7F
:108B8000226763223A2266353030227D0A7B2267D3
:108B900063223A22284D53477371756172657329B8
:108BA000227D0A7B226763223A22673078323022A4
:108BB0007D0A7B226763223A22793230227D0A7B4A
:108BC000226763223A227830227D0A7B2267632261
:108BD0003A227930227D0A7B226763223A2267316A
:108BE000783130227D0A7B226763223A2279313044
:108BF000227D0A7B226763223A227830227D0A7B1B
:108C0000226763223A227930227D0A7B226763221F
:108C10003A22284D5347636972636C657329227D3C
:108C20000A7B226763223A226732783130792D310C
:108C300030693130227D0A7B226763223A22673015
:108C400078307930227D0A7B226763223A226733AB
:108C5000783130792D3130693130227D0A7B2267BD
:108C600063223A22673078307930227D0A7B22678E
:108C700063223A2267327832307930693130227D8E
:108C80000A7B226763223A22673078307930227D6E
:108C90000A7B226763223A2267337832307930695F
:108CA0003130227D0A7B226763223A226730783096
:108CB0007930227D0A7B226763223A22673278303C
:108CC0007930693130227D0A7B226763223A22673C
:108CD0003378307930693130227D0A7B2267632214
:108CE0003A22673534227D0A7B226763223A226763
:108CF0003078307930227D0A7B226763223A226DF8
:108D00003330227D00284D53472A2A2A2A204D63DA
:108D10006F6465732074657374205B76315D202AFF
:108D20002A2A2A290A6735350A6730783079300AC5
:108D30006D330A673470310A6D350A673470310A51
:108D40006D340A673470310A6D350A673470310A40
:108D50006D370A673470310A6D390A673470310A29
:108D60006D380A673470310A6D390A663530300A59
:108D700067307832300A7932300A6D330A78300A37
:108D80006D340A79300A6D350A67317831300A6DF1
:108D9000370A7931300A6D380A78300A6D390A7924
:108DA000300A6732783130792D31306931300A6DCF
:108DB000330A6730783079300A6D340A6733783196
:108DC00030792D31306931300A6D350A67307830AD
:108DD00079300A6D370A673278323079306931304C
:108DE0000A6D380A6730783079300A6D390A67338E
:108DF00078323079306931300A6730783079300A2A
:108E00006732783079306931300A673378307930B9
:108E10006931300A6735340A6730783079300A6D45
:108E2000333000284D53472A2A2A2A204665656494
:108E3000686F6C642054657374205B76315D202A02
:108E40002A2A2A290A284D53472A2A2A2A204D61EC
:108E50006E75616C6C7920656E746572202120617D
:108E60006E64207E20647572696E67206D6F766512
:108E70006D656E7420746F2074657374202A2A2ABD
:108E80002A290A6735350A6730783079300A67341D
:108E900070330A6730306731376732316734306793
:108EA00034396738306739300A663630300A67300F
:108EB000783130307637362E3736350A783079309B
:108EC0000A6735340A6730783079300A6D333000FC
:108ED000284D53472A2A2A2A204477656C6C20544F
:108EE000657374205B76315D202A2A2A2A290A6755
:108EF00030306731376732316739300A6735350AC4
:108F00006730783079300A663530300A673078312A
:108F1000300A673470310A67307832300A6734704B
:108F2000310A67307831300A673470310A67307837
:108F300030300A673470310A79350A6735340A6788
:108F400030783079300A6D330A673470310A67300F
:108F50007831307931300A6D350A673470310A67FB
:108F6000307832307932300A6D340A673470310A21
:108F700067307833307933300A6D380A67347031AE
:108F80000A67307834307934300A6D390A673470C2
:108F9000310A67307835307935300A673078307982
:108FA000300A6D3330004E3120673030673137671B
:108FB00032316734306734396738306739300A4EB8
:108FC0003130206730783079300A4E3230206635C3
:108FD00030300A4E3330206732783130792D3130DD
:108FE000693130202843572032373020646567725A
:108FF000656573290A4E3430206730783079300A3D
:109000004E3530206733783130792D313069313049
:1090100020284343572039302064656772656573A3
:10902000290A4E3630206730783079300A4E383091
:109030002067327832307930693130202843572028
:109040003138302064656772656573290A4E3730A0
:10905000206730783079300A4E38302067337832E4
:10906000307930693130202843435720313830205F
:1090700064656772656573290A4E393020673078F8
:109080003079300A4E39392046313230300A4E318B
:1090900030302067327830793069323020284357B9
:1090A000203336302064656772656573290A4E3156
:1090B0003130206732783079306932302028435798
:1090C0002033363020616761696E290A4E313230B3
:1090D000206637303020284368616E6765206665FA
:1090E00065642072617465207768696C6520696EBB
:1090F000204732206D6F74696F6E206D6F64652933
:109100000A4E31333020673278307930693230207E
:1091100028435720333630203372642074696D65DC
:10912000290A4E3134302067327830793069323054
:109130002028435720333630203474682074696DFA
:1091400065290A4E31353020663530300A4E3136C9
:1091500030206733783079307A34306932302028E3
:10916000434357203336302064656772656573204A
:1091700077697468206C696E6561722074726176BB
:10918000656C290A4E313730206733783079307A70
:10919000306932302028434357203336302061670E
:1091A00061696E290A4E3138302066373030202808
:1091B0006D73672A2A2A2A4368616E67652066658F
:1091C00065642072617465207768696C6520696EDA
:1091D000204733206D6F74696F6E206D6F64652A50
:1091E0002A2A2A290A4E31393020673378307930DB
:1091F000693230202843435720333630203372649D
:109200002074696D65290A4E32303020673378301A
:1092100079306932302028434357203336302034A8
:1092200074682074696D65290A4E32313020286DCA
:1092300073672A2A2A2A473138204576616C2074C0
:109240006573742A2A2A2A290A4E3232302047317D
:10925000205833302E373037205A35302E373237BA
:1092600020463530300A4E323330204731382047DF
:109270003032205836372E373338205A32332E3694
:1092800031372052323520463235300A4E323430B2
:10929000206738300A4E32353020673078307930E8
:1092A0007A300A4E323630206D333000284D534725
:1092B0002A2A2A2A2053717561726573204D6F74B2
:1092C000696F6E2054657374205B76315D202A2AA5
:1092D0002A2A290A673030673137673231673430DC
:1092E0006734396738306739300A67307830793019
:1092F0000A6730783230202874726176657273653F
:1093000020612032306D6D20737175617265206946
:109310006E205820616E642059290A7932300A780B
:10932000300A79300A67317831306635303020289C
:109330006472617720612031306D6D2073717561C9
:10934000726520696E205820616E64205920617416
:109350002046353030290A7931300A78300A7930A0
:109360000A67307A323020287472617665727365CC
:1093700020612032306D6D207371756172652069D6
:109380006E205820616E64205A290A7832300A7A99
:10939000300A78300A67317832307932307A3230B8
:1093A0006635303020286665656420612032306D76
:1093B0006D20646961676F6E616C20696E20582C46
:1093C000205920616E64205A290A783079307A3029
:1093D0000A7834307934307A3430202874726176E7
:1093E0006572736520612034306D6D206375626530
:1093F00020696E20582C205920616E64205A290A59
:1094000078343079307A300A78307934307A3430C0
:109410000A7834307934307A300A783079307A34D6
:10942000300A78307934307A300A78343079307ACA
:1094300034300A783079307A300A6738300A673049
:10944000783079300A673078310A673078300A6DC1
:10945000333000284D53472A2A2A2A20486F6D6945
:109460006E672054657374205B76315D202A2A2A4A
:109470002A290A6732382E32783079307A300A6DEC
:10948000333000284D53472A2A2A2A20536D6F6B08
:10949000652054657374205B76315D202A2A2A2A60
:1094A000290A4730302047313720473231204734AE
:1094B000302047343920473830204739300A6D335F
:1094C000673470310A6D35673470310A6D34673432
:1094D00070310A6D33673470310A6D35673470311D
:1094E0000A6D37673470310A6D39673470310A6D2F
:1094F00038673470310A6D390A6730783079307ADC
:10950000300A673030207832300A78300A793230C9
:109510000A79300A7A32300A7A300A6132300A61C6
:10952000300A4730302078323020793230207A3299
:1095300030206132300A47303020783020793020B6
:109540007A302061300A473031206633302078325B
:10955000207932207A322061320A78302079302026
:109560007A302061300A673078310A673078300A03
:109570006D32002C000A00257300256C7500253122
:109580002E3066002573002C000A0025733A2573DF
:109590000025733A256C750025733A25312E306607
:1095A0000025733A2573005B74765D20207465781E
:1095B0007420766572626F73697479253135642021
:1095C0005B303D73696C656E742C313D76657262FB
:1095D0006F73655D0A0025660A00256C750A002513
:1095E000640A0025730A0074696E7967205B25732D
:1095F0005D206572723A2025733A2025732000742D
:10960000696E7967205B25735D206F6B3E20004596
:109610006E64206F6620636F6D6D616E6420666995
:109620006C650A00DECB4ECA4BCC6CCCCBCC93CA5B
:10963000A3CF4ECA37D0A3D0D1CE93CA00004006E4
:1096400040061040B800B8A3CF4ECA37D0A3D0D13F
:10965000CE93CA0000400620060840B800B819D2D0
:109660004ECA3AD1B5D164D303D1A008400605064D
:1096700009010819D24ECA3AD1B5D1DDCC93CAB08E
:109680000840060540B030800000000000F0E0D047
:10969000C0100100CF673322211F1B1301016E612F
:1096A0006E00696E66004E414E494E495459494E0E
:1096B00046CDCCCC3D0AD7233C17B7D13877CC2B3D
:1096C000329595E6241FB14F0A000020410000C8E2
:1096D0004200401C4620BCBE4CCA1B0E5AAEC59D63
:1096E0007400407A10F35A00A0724E18090010A5B9
:1096F000D4E80000E87648170000E40B54020000AC
:10970000CA9A3B000000E1F5050000809698000031
:109710000040420F000000A086010000001027005A
:10972000000000E803000000006400000000000AE0
:1097300000000000000100000000002C76D888DC4A
:10974000674F0823DFC1DFAE59E1B1B796E5E3E427
:1097500053C63AE651997696E8E6C28426EB898CA0
:109760009B62ED407C6FFCEFBC9C9F40F2BAA56F02
:10977000A5F490055A2AF75C936B6CF9676DC11BD1
:10978000FCE0E40D47FEF520E6B500D0ED902E0399
:1097900000943577050080841E080000204E0A00E2
:1097A0000000C80C333333330F986E12831141EF2E
:1097B0008D2114893BE65516CFFEE6DB18D1844B8C
:1097C000381BF77C1D901DA4BBE424203284725EFC
:1097D000228100C9F124ECA1E53D270011241FBE20
:1097E000CFEFCDBFDFE5DEBF00E00CBF13E2A0E0AE
:1097F000B0E2E6ECFDEC01E00BBF02C007900D9279
:10980000A239B107D9F72BE5A2E9B3E201C01D9255
:10981000AD37B207E1F70E9433840C94E1E60C9473
:109820000000FC0160817181828193810E94B2D825
:109830006093ED330895FC01608171818281938191
:109840000E94B2D86093EC330895AF92BF92CF924A
:10985000DF92EF92FF920F931F93CF93DF937B01E1
:109860008C0180E7C82E83E3D82EE601AA24A394B6
:10987000BC2EBC18F70161917191819191917F018A
:109880002CEA35EC47E257E30E9441DA18164CF413
:10989000F80140815181628173818B2D0E94A185E5
:1098A000A8820C5F1F4F2196F3E3C637DF0701F74D
:1098B000DF91CF911F910F91FF90EF90DF90CF90AC
:1098C000BF90AF900C94AC85FC0160817181828166
:1098D00093810E94B2D86093EE33613019F481E035
:1098E0000E94A87B81E00C94C97BCF93DF93CDB716
:1098F000DEB76897CDBFDEBFFC01608171818281D8
:1099000093810E94B2D86093EF3381E0613019F403
:109910000E94A87B0CC00E94C97BCE01019628E161
:10992000FC0111922A95E9F7BC010E94644C6896EB
:10993000CDBFDEBFDF91CF9108950F931F93CF93DB
:10994000DF93CDB7DEB72D97CDBFDEBF27E0E2EDC9
:10995000F0E28E010F5F1F4FD80101900D922A9502
:10996000E1F7BC01660F771F680F791F660F771F3D
:10997000660F771F660F771F61507A4E45E050E003
:10998000CE0108960E9451E4688570E0C8010E94EB
:109990007FE4009739F46B8570E0C8010E947FE492
:1099A000009711F0801B01C08FEF2D96CDBFDEBF59
:1099B000DF91CF911F910F910895EF92FF920F9336
:1099C0001F93CF93DF938C01F62EE72EEC012D969B
:1099D000FC0161857285838594850E94B2D81F92AF
:1099E0006F93DF93CF930F5E1F4F1F930F93DF9300
:1099F000CF93EF92FF92E9E7FBE581818F9380811E
:109A00008F930E9418E5EDB7FEB73C96EDBFFEBF01
:109A1000DF91CF911F910F91FF90EF9008950F93D9
:109A20001F93CF93DF93EC01162F072F8C819D811D
:109A30000E949D4C83305CF58F3FA1F528C09E01AC
:109A4000235F3F4F9F938F938C858F938B858F934D
:109A50008A858F9389858F933F932F936196DF93A8
:109A6000CF933F932F930F931F9380917A5B8F93A4
:109A70008091795B8F930E9418E58DB79EB74096D1
:109A80008DBF9EBFDF91CF911F910F910895E7E7A2
:109A9000F4E1659174914FE450E081E79EE30E9408
:109AA00051E4CDCFE091E633F0E0EE0FFF1FED582B
:109AB000FB4E659174914FE450E081E79EE30E9474
:109AC00051E4BDCF0F931F93CF93DF93EC01162F7B
:109AD000072F8C819D810E949D4C83307CF58F3FA8
:109AE000C1F52CC0AE014F5E5F4F9E01235F3F4F1B
:109AF0009F938F938C858F938B858F938A858F937C
:109B000089858F935F934F933F932F935F934F93E9
:109B10003F932F930F931F9380917A5B8F93809144
:109B2000795B8F930E9418E58DB79EB742968DBFE3
:109B30009EBFDF91CF911F910F910895E7E7F4E168
:109B4000659174914FE450E081E79EE30E9451E4F7
:109B5000C9CFE091E633F0E0EE0FFF1FED58FB4E6A
:109B6000659174914FE450E081E79EE30E9451E4D7
:109B7000B9CFDF92EF92FF920F931F93CF93DF93B2
:109B8000CDB7DEB72897CDBFDEBF8B01E42ED52E33
:109B900037E0E9EDF0E2DE01119601900D923A9581
:109BA000E1F728870E949D4CF82E288582E08F15CA
:109BB00018F0E22FF0E002C0E2E0F0E0EE0FFF1F4D
:109BC000ED58FB4E659174914FE450E081E79EE3C0
:109BD0000E9451E49F938F93F80183818F93828138
:109BE0008F9381818F9380818F93E1E0F0E0EC0F80
:109BF000FD1FEF0DF11D80811F928F93DF92EF9279
:109C000080917A5B8F938091795B8F930E9418E5A6
:109C1000CDBFDEBF2896CDBFDEBFDF91CF911F91B4
:109C20000F91FF90EF90DF9008954F925F926F92A7
:109C30007F92AF92BF92CF92DF92EF92FF920F93FB
:109C40001F93CF93DF93C0E7D3E305E312E35C01F7
:109C50008991813009F042C0F801C480D580E68046
:109C6000F7804080518062807380A3019201C70118
:109C7000B6010E9495D69F772CEA35EC47E257E370
:109C80000E943ED887FD2AC020E034E244E759EC28
:109C9000C701B6010E9441DA18165CF4F501208173
:109CA000318142815381C701B6010E9441DA181601
:109CB00004F120E034E244E759ECC301B2010E9410
:109CC00041DA18165CF4F50120813181428153811B
:109CD000C301B2010E943ED887FD0BC00B5C1F4F31
:109CE000F4E0AF0EB11C83E3C637D80709F0B0CF5C
:109CF00002C08CED01C080E0DF91CF911F910F91E8
:109D0000FF90EF90DF90CF90BF90AF907F906F90DB
:109D10005F904F90089580916C33811105C08091C0
:109D20006B3380936A3329C0823031F487E08093AB
:109D30006A3380916B3321C0833031F489E08093A2
:109D40006A3380916B3319C0843031F48AE0809398
:109D50006A3380916B3311C080916D33813031F45F
:109D600085E080936A3380916B3307C0823019F4A9
:109D700086E080936A3380916B33863019F080914E
:109D80006A3308958BE080936A33089580916B3332
:109D9000089580936D33813059F018F0823041F08E
:109DA00008958BE993E38093993390939A330895C0
:109DB00080EC97E58093993390939A330895FC0152
:109DC00084810895845B9F4FFC0180810895855BA9
:109DD0009F4FFC0180810895825B9F4FFC01808131
:109DE0000895815B9F4FFC0180810895875B9F4FA1
:109DF000FC01808108950C94A29ACD96FC016081AB
:109E00007181828193810895FC01648308958B5A46
:109E10009F4FFC01608308958F5B9F4FFC0140833F
:109E2000518362837383089560939B3370939C3353
:109E300080939D3390939E3387EE91E20C94F76567
:109E4000BF92CF92DF92EF92FF920F931F93CF9327
:109E5000DF93D090E8337C010DE014E38091E73389
:109E600090E0EC01CC0FDD1FC80FD91FCC0FDD1F18
:109E7000CC0FDD1FCC0FDD1FCC57DE4C81E0D81698
:109E8000A9F0B881A981CA80BB804091603441307B
:109E900091F4F80120813181428153816B2F7A2F17
:109EA0008C2D9B2D0E9496D69B0109C020E030E0AE
:109EB00080E090E004C02B2F3A2F8C2D9B2DA90120
:109EC000BC01F701458F568F678F70A3F4E0EF0E4A
:109ED000F11C0C5F1F4F249684E30532180771F6BE
:109EE000DF91CF911F910F91FF90EF90DF90CF9076
:109EF000BF900895835B9F4FFC0160838BE993E3E0
:109F00000C94204F4F925F926F927F928F929F920C
:109F1000AF92BF92CF92DF92EF92FF920F931F9377
:109F2000CF93DF93CDB7DEB76897CDBFDEBF8C018F
:109F30006091603470E080E090E00E94E0D82B01F6
:109F40003C01F80160817181828193810E94B2D8C5
:109F500070E05B01AA0CBB1CA60EB71EAA0CBB1CB2
:109F6000AA0CBB1CAA0CBB1CC5018C579E4C5C01E7
:109F70000DE014E3FE0131964F01F501C190D1903F
:109F8000E190F1905F01F80161917191819191915E
:109F90008F01A30192010E94E3DA9B01AC01C7018A
:109FA000B6010E9496D6F4016193719381939193C7
:109FB0004F01F4E305321F0701F7CE0101960E941D
:109FC000859A8BE993E30E94204F6896CDBFDEBF50
:109FD000DF91CF911F910F91FF90EF90DF90CF9085
:109FE000BF90AF909F908F907F906F905F904F90B9
:109FF00008958B59934369F4E62FF0E0EE0FFF1FAD
:10A00000EE0FFF1FEB50FC4C6081718182819381C8
:10A010000895862F0C947A9ACF92DF92EF92FF9256
:10A020000F931F93CF93DF93EC0183E3CB39D807D2
:10A0300009F04AC070E0FB01EE0FFF1FEE0FFF1F9B
:10A04000EB50FC4CC080D180E280F3808091E833FB
:10A05000813059F18091E73390E0FC01EE0FFF1F52
:10A06000E80FF91FEE0FFF1FE60FF71FEE0FFF1FA0
:10A07000EE0FFF1FEC57FE4C00811181B281A381CE
:10A08000209160342130B1F4FB01EE0FFF1FEE0F81
:10A09000FF1FE35FFB4C2081318142815381B80176
:10A0A0008B2F9A2F0E9496D608C060E070E080E067
:10A0B00090E003C0B8018B2F9A2F9B01AC01C70120
:10A0C000B6010E9495D603C0862F0E948E9AC55B6A
:10A0D000DF4F2881211106C023E333E34BEC51E429
:10A0E0000E9445D8DF91CF911F910F91FF90EF9083
:10A0F000DF90CF90089588E1E0EAF3E3A5EFB3E3C2
:10A1000001900D928A95E1F78091E43381110CC0A2
:10A1100080919F33813041F41092D8331092D9331B
:10A120001092DA331092DB3308954F925F926F9260
:10A130007F928F929F92AF92BF92CF92DF92EF92D7
:10A14000FF920F931F93CF93DF93CDB7DEB769973D
:10A15000CDBFDEBF80916C33811155C080919133AA
:10A16000813009F050C00E94EDC981114CC010929D
:10A1700091339CE9692E91E3792E26E3822E912C6E
:10A180008E010E5E1F4F30EEA32E30E2B32E33C091
:10A19000F70181917F011F928F935F924F92BF923F
:10A1A000AF921F930F930E94E3E5B80180E593E21D
:10A1B0000E945D638D839E83F60181919191A191AF
:10A1C000B1916F018A879B87AC87BD87CE010196CD
:10A1D0000E947460CDBFDEBF98EDE91690E2F906EB
:10A1E000B9F6E8E16E0E711CFFEF8F1A9F0A8CE33F
:10A1F0008816910441F0240183EDE82E80E2F82EC8
:10A20000630188E7C8CF80E06996CDBFDEBFDF91EC
:10A21000CF911F910F91FF90EF90DF90CF90BF9063
:10A22000AF909F908F907F906F905F904F90089528
:10A230002F923F924F925F926F927F928F929F9256
:10A24000AF92BF92CF92DF92EF92FF920F931F9344
:10A25000CF93DF93CDB7DEB72997CDBFDEBF4C01DB
:10A260005B014090EA335090E8332090E7336090F0
:10A2700060347090E6336B0180EA93E388879987B6
:10A280005CE2E52E52E3F52E98E1299E100111249F
:10A290008401D6016D917D918D919D916D012CEA86
:10A2A00035EC47E257E30E943ED887FD80C0F701B6
:10A2B00080818150823008F07AC041104CC0F1E0BA
:10A2C0005F1609F1E885F985E20DF31DEC51F240C6
:10A2D0008081898391819D83B281A381E1E06E12A7
:10A2E00017C0E885F985E359FF4F2081318142810C
:10A2F0005381BC018B2F9A2F0E9496D669837D8350
:10A300008E839F8307C019821D821E821F8202C016
:10A31000BE83AF8371100CC023E333E34BEC51E4F5
:10A32000D8016D917D918D919C910E94E3DA05C0D9
:10A33000F801608171818281938129813D814E8103
:10A340005F810E9496D6A885B9856D937D938D9384
:10A350009C9313972CC0A885B9858D919D910D90E4
:10A36000BC91A02D89839A83AB83BC8371100EC0EE
:10A3700023E333E34BEC51E4F80160817181828186
:10A3800093810E94E3DA9B01AC0105C0D8012D91B5
:10A390003D914D915C9169817A818B819C810E9474
:10A3A00096D6E885F9856083718382839383888557
:10A3B000998504968887998795E3E90EF11C0C5FCF
:10A3C0001F4FA885B985AC5AB34309F062CF60909E
:10A3D000E6337090EA33F091E833F983C090E733C5
:10A3E000209160342D838CE0A80EB11CABECB2E35D
:10A3F000A887B9874CEAE42E43E3F42EB8E1CB9E5C
:10A40000600111248401F501619171918191919113
:10A410005F012CEA35EC47E257E30E943ED887FD06
:10A420008CC0A885B9858C91882309F486C0815099
:10A43000823030F4F80124843584468457843BC04C
:10A44000611016C023E333E34BEC51E4D8011C96B2
:10A450006D917D918D919C911F970E94E3DA20E090
:10A4600030E044EB53E40E94E3DA1B012C010DC001
:10A4700020E030E044EB53E4F8016485758586857F
:10A4800097850E94E3DA1B012C012BED3FE049EC9C
:10A4900050E4A885B98591966D917D918D919C919F
:10A4A00094970E94E3DA9B01AC01C201B1010E94C2
:10A4B00045D81B012C01711031C0B981B130E1F0D8
:10A4C000F701EC0DFD1DEC51F240A081B1819280AD
:10A4D0008380ED81E130A1F4F701E359FF4F208142
:10A4E000318142815381BD01892D982D0E9496D6DC
:10A4F000DB01982E892E04C0A0E0B0E0912C812CC5
:10A50000A2019101BD01892D982D0E9496D6D701F7
:10A510006D937D938D939C9313970FC0A20191012E
:10A52000F70160817181828193810E9496D6D70163
:10A530006D937D938D939C931397E885F985F5969C
:10A54000E887F987F4E0EF0EF11C0C5F1F4F888558
:10A5500099858A56934309F056CF2996CDBFDEBF21
:10A56000DF91CF911F910F91FF90EF90DF90CF90EF
:10A57000BF90AF909F908F907F906F905F904F9023
:10A580003F902F90089580916831909169318F3E6E
:10A59000924111F08FE5089580911F3590912035FB
:10A5A0008F3E9241B9F78091F1339091F2338F3E13
:10A5B000924181F780916734909168348F3E924147
:10A5C00049F780911858909119588F3E924111F790
:10A5D0008091D5589091D6588F3E9241D9F680E01F
:10A5E000089580916C33811104C083E080936B33B4
:10A5F00003C085E080936B3380E00895CF93C82F2C
:10A600000E9450B680E00E94F1B18C2F0E9473AB83
:10A6100086E080936B338C2FCF9108958093E53340
:10A6200080E008958093E63380E008958093EA33D4
:10A6300080E00895AF92BF92CF92DF92EF92FF92A7
:10A640000F931F93CF93DF939FEF980F963008F0EF
:10A6500041C0A090E6337A018B0198E1899F6001A7
:10A660001124F601E859FE4C6F01C0E0D0E0BB2494
:10A67000B394F70161917191819191917F012CEADD
:10A6800035EC47E257E30E9441DA1816E4F4A110D2
:10A690000CC023E333E34BEC51E4F801608171819A
:10A6A000828193810E94E3DA05C0F80160817181A3
:10A6B00082819381F601EC0FFD1F648F758F868F69
:10A6C000978FB092913324960C5F1F4FC831D105FC
:10A6D00081F602C08EE601C080E0DF91CF911F912C
:10A6E0000F91FF90EF90DF90CF90BF90AF900895C3
:10A6F000CF93DF93CDB7DEB76897CDBFDEBF809332
:10A70000E733682F70E080E090E00E94DED8698334
:10A710007A838B839C831D821E821F8218861986F2
:10A720001A861B861C861D861E861F86188A198A15
:10A730001A8A1B8A1C8A1D8A1E8A1F8A188EAE01DD
:10A740004F5F5F4FBA0182E89FE40E94E38680E09A
:10A750006896CDBFDEBFDF91CF910895CF93DF9391
:10A76000EBE9F3E386E5DF011D928A95E9F78BE5D6
:10A77000A9E6B4E3ED01982F19929A95E9F7A4ECB4
:10A78000B4E3ED0119928A95E9F78FEE92E1809397
:10A7900068319093693180931F3590932035809371
:10A7A000F1339093F23380936734909368348093BD
:10A7B0001858909319588093D5589093D658E09391
:10A7C0009933F0939A33809181318093E63380916D
:10A7D0007F310E947853809180318093E53380915E
:10A7E00082318093E933809183318093EA3381E031
:10A7F0008093E4338093613494E090939F3310927C
:10A800009233109293331092943380936B338093EE
:10A810006A330E948FB0DF91CF910C942588CF923C
:10A82000DF92EF92FF92CF93C82F6A017B01E82F4E
:10A83000F0E0DF01AA0FBB1FAA0FBB1FAB50BC4C3F
:10A84000CD92DD92ED92FC921397EE0FFF1FEE0F6B
:10A85000FF1FE056FC4CC082D182E282F382B70136
:10A86000A6010E949685B701A6018C2F0E94A185A2
:10A87000CF91FF90EF90DF90CF900C94AC859F929A
:10A88000AF92BF92CF92DF92EF92FF920F931F93FE
:10A89000CF93DF93CDB7DEB76897CDBFDEBF962EDF
:10A8A000A72EC62ED72E7C0100E010E0B12CF601B9
:10A8B00061917191819191916F012CEA35EC47E2A0
:10A8C00057E30E9441DA1816A4F58091E63381110E
:10A8D0000EC023E333E34BEC51E4F7016081718157
:10A8E000828193810E94E3DAAB01BC0105C0F701CC
:10A8F0004081518162817381E1E0F0E0EC0FFD1F46
:10A90000E00FF11F4083518362837383C80188592C
:10A910009E4CFC01E357FD4F408351836283738358
:10A92000E555F10940835183628373838B2D0E9427
:10A930009685B3940C5F1F4FF4E0EF0EF11C0831C5
:10A94000110509F0B4CF492D5A2DBE016F5F7F4F1D
:10A9500085E29CE40E94E38680E06896CDBFDEBF7E
:10A96000DF91CF911F910F91FF90EF90DF90CF90EB
:10A97000BF90AF909F9008954F925F926F927F9299
:10A980008F929F92AF92BF92CF92DF92EF92FF92FF
:10A990000F931F93CF93DF93CDB7DEB76897CDBFEB
:10A9A000DEBF21E0209360348090E7339090E6335F
:10A9B0005B016C0105EF13E3882D90E07C01EE0C48
:10A9C000FF1CE80EF91EEE0CFF1CEE0CFF1CEE0C3B
:10A9D000FF1CC7018C579E4C7C01F5016191719160
:10A9E000819191915F012CEA35EC47E257E30E9497
:10A9F00041DA181664F5F7012081318142815381D3
:10AA0000F80160817181828193810E9495D62B012A
:10AA10003C0191100EC023E333E34BEC51E4F6010B
:10AA200060817181828193810E94E3DA9B01AC0194
:10AA300005C0F6012081318142815381C301B201F9
:10AA40000E9495D6F801608F718F828F938FF4E00A
:10AA5000CF0ED11C0C5F1F4F84E0E80EF11C94E375
:10AA60000D30190709F0B9CF682D70E080E090E053
:10AA70000E94DED869837A838B839C831D821E8229
:10AA80001F82188619861A861B861C861D861E86BE
:10AA90001F86188A198A1A8A1B8A1C8A1D8A1E8A8E
:10AAA0001F8A188EAE014F5F5F4FBA0182E89FE4A4
:10AAB0000E94E38680E06896CDBFDEBFDF91CF9134
:10AAC0001F910F91FF90EF90DF90CF90BF90AF90CC
:10AAD0009F908F907F906F905F904F900895CF934D
:10AAE000DF93CDB7DEB76897CDBFDEBF109260347D
:10AAF00010920D3410920E3410920F3410921034C4
:10AB000010921134109212341092133410921434A3
:10AB10001092153410921634109217341092183483
:10AB20001092193410921A3410921B3410921C3463
:10AB300010921D3410921E3410921F341092203443
:10AB40001092213410922234109223341092243423
:10AB50006091E73370E080E090E00E94DED8698386
:10AB60007A838B839C831D821E821F82188619869E
:10AB70001A861B861C861D861E861F86188A198AC1
:10AB80001A8A1B8A1C8A1D8A1E8A1F8A188EAE0189
:10AB90004F5F5F4FBA0182E89FE40E94E38680E046
:10ABA0006896CDBFDEBFDF91CF910895CF93DF933D
:10ABB000CDB7DEB76897CDBFDEBF1092603460912D
:10ABC000E73370E080E090E00E94DED869837A830A
:10ABD0008B839C831D821E821F82188619861A868B
:10ABE0001B861C861D861E861F86188A198A1A8A4D
:10ABF0001B8A1C8A1D8A1E8A1F8A188EAE014F5F0F
:10AC00005F4FBA0182E89FE40E94E38680E0689685
:10AC1000CDBFDEBFDF91CF910895CF93DF93CDB746
:10AC2000DEB76897CDBFDEBF81E08093603460916E
:10AC3000E73370E080E090E00E94DED869837A8399
:10AC40008B839C831D821E821F82188619861A861A
:10AC50001B861C861D861E861F86188A198A1A8ADC
:10AC60001B8A1C8A1D8A1E8A1F8A188EAE014F5F9E
:10AC70005F4FBA0182E89FE40E94E38680E0689615
:10AC8000CDBFDEBFDF91CF910895CF9310929F3358
:10AC90000E94185180917231813069F480EA93E307
:10ACA0000E94154EC82F882331F00E9473AB82E0BA
:10ACB00080936B3317C08BE993E30E94204F85E0AC
:10ACC00080936B3380916C33811105C081E0809358
:10ACD0006C330E94E7AE8BE993E30E94AF9A0E9427
:10ACE0007B50C0E08C2FCF91089588E1E5EFF3E32E
:10ACF000A5E2B4E301900D928A95E1F780E0089512
:10AD00000F931F93CF93DF93CDB7DEB76A97CDBF75
:10AD1000DEBF8C0181E08093E8338BE993E3698F98
:10AD20007A8F0E94204F698D7A8DC8010E94455606
:10AD30000E941D868823E1F388E1E0E0F0E2DE0175
:10AD4000119601900D928A95E1F7BE016F5F7F4FDA
:10AD500085E294E30E9445566A96CDBFDEBFDF913F
:10AD6000CF911F910F91089588E1E5EFF3E3ADE3F3
:10AD7000B4E301900D928A95E1F780E008950F9376
:10AD80001F93CF93DF93CDB7DEB76A97CDBFDEBFFA
:10AD90008C0181E08093E8338BE993E3698F7A8FAC
:10ADA0000E94204F698D7A8DC8010E9445560E94ED
:10ADB0001D868823E1F388E1E0E0F0E2DE011196F0
:10ADC00001900D928A95E1F7BE016F5F7F4F8DE391
:10ADD00094E30E9445566A96CDBFDEBFDF91CF91C6
:10ADE0001F910F910895FB01DC018091E4338111E3
:10ADF00011C09B01AD0160E070E080E89FE30E941C
:10AE000045D86093D8337093D9338093DA339093D5
:10AE1000DB3318C08091E633811109C023E333E3AB
:10AE20004BEC51E4CD010E94E3DAFB0101C0CD01FE
:10AE3000AF01BC014093D8335093D9336093DA33D8
:10AE40007093DB3380E008958093E43380E00895CD
:10AE50008093E93380E008956093E0337093E133A9
:10AE60008093E2339093E3330E943B8780E0089520
:10AE70000F931F93CF93DF93EC018B018091E43309
:10AE8000882399F08091D8339091D933A091DA3307
:10AE9000B091DB33BC01CD019F772CEA35EC47E262
:10AEA00057E30E943ED887FD30C081E080939F33F6
:10AEB000B801CE010E94185180917231813069F43D
:10AEC00080EA93E30E94154EC82F882331F00E9438
:10AED00073AB82E080936B3319C08BE993E30E94DC
:10AEE000204F85E080936B3380916C33811105C0D6
:10AEF00081E080936C330E94E7AE8BE993E30E947C
:10AF0000AF9AC82F0E947B5001C0CEE88C2FDF91F2
:10AF1000CF911F910F910895CF93DF93CDB7DEB7F7
:10AF20006897CDBFDEBF682F70E080E090E00E94A0
:10AF3000DED869837A838B839C831D821E821F8265
:10AF4000188619861A861B861C861D861E861F86F5
:10AF5000188A198A1A8A1B8A1C8A1D8A1E8A1F8AC5
:10AF6000188EAE014F5F5F4FBA0181E19CE40E94F1
:10AF7000E38680E06896CDBFDEBFDF91CF91089574
:10AF8000CF93DF93CDB7DEB76897CDBFDEBF6091BB
:10AF9000ED3370E080E090E00E94DED869837A8330
:10AFA0008B839C831D821E821F82188619861A86B7
:10AFB0001B861C861D861E861F86188A198A1A8A79
:10AFC0001B8A1C8A1D8A1E8A1F8A188EAE014F5F3B
:10AFD0005F4FBA018BE19CE40E94E38680E06896B3
:10AFE000CDBFDEBFDF91CF910895CF93DF93CDB773
:10AFF000DEB76897CDBFDEBF682F70E080E090E0DD
:10B000000E94DED869837A838B839C831D821E8293
:10B010001F82188619861A861B861C861D861E8628
:10B020001F86188A198A1A8A1B8A1C8A1D8A1E8AF8
:10B030001F8A188EAE014F5F5F4FBA0184E69CE411
:10B040000E94E38680E06896CDBFDEBFDF91CF919E
:10B050000895CF93DF93CDB7DEB76897CDBFDEBF3E
:10B06000682F70E080E090E00E94DED869837A83E8
:10B070008B839C831D821E821F82188619861A86E6
:10B080001B861C861D861E861F86188A198A1A8AA8
:10B090001B8A1C8A1D8A1E8A1F8A188EAE014F5F6A
:10B0A0005F4FBA0185E79CE40E94E38680E06896E2
:10B0B000CDBFDEBFDF91CF910895CF93FC016081BA
:10B0C0007181828193810E94B2D860936B33109218
:10B0D0006D338BE993E38093993390939A33809106
:10B0E0006C33813011F410926C3310926E331092E5
:10B0F00094330E94689AC0916B33C430C9F40E94A3
:10B100006F5580917F310E94785380918031809378
:10B11000E533809183318093EA3380E00E94F1B17E
:10B1200080E00E94295881E08093E433C0939F33EC
:10B1300081E0CF910C94ABAD80935D3480935E340D
:10B140008093663480E008952CEA35EC47E257E3BB
:10B1500060910B3570910C3580910D3590910E35C5
:10B160000E9441DA1816B4F48091B0349091B13451
:10B17000A091B234B091B334BC01CD019F772CEAD9
:10B1800035EC47E257E30E943ED887FF03C0109298
:10B190005D3403C081E080935D3480E00895809346
:10B1A0005D348091B0349091B134A091B234B091BB
:10B1B000B3348093553490935634A0935734B0935E
:10B1C000583480E008952CEA35EC47E257E360916B
:10B1D0000B3570910C3580910D3590910E350E9494
:10B1E00041DA1816B4F48091B0349091B134A09142
:10B1F000B234B091B334BC01CD019F772CEA35EC69
:10B2000047E257E30E943ED887FF03C010925E34A6
:10B2100003C081E080935E3480E0089580935E34C3
:10B220008091B0349091B134A091B234B091B334E4
:10B230008093593490935A34A0935B34B0935C3428
:10B2400080E008952CEA35EC47E257E360910B3536
:10B2500070910C3580910D3590910E350E9441DA38
:10B260001816B4F48091B0349091B134A091B234F6
:10B27000B091B334BC01CD019F772CEA35EC47E2A5
:10B2800057E30E943ED887FF03C01092663403C084
:10B2900081E08093663480E00895809366348091E5
:10B2A000B0349091B134A091B234B091B334809362
:10B2B000623490936334A0936434B093653480E037
:10B2C0000895BC0187EE90E20C941A6681E08093A9
:10B2D0009233089581E080939333089581E08093C1
:10B2E000943308951F93CF93DF93CDB7DEB768975C
:10B2F000CDBFDEBF0E94A29A8130C9F10E94DCD48A
:10B300000E94A08680E00E94FCAE0E9405B010E082
:10B31000812F0E947A9AAB01BC01812F0E940F54A9
:10B320001F5F1630A9F780E090E0A0E4B0E48983C5
:10B330009A83AB83BC831D821E821F821886198666
:10B340001A861B861C861D861E861F86188A198AE9
:10B350001A8A1B8A1C8A1D8A1E8A1F8A188EBE01A1
:10B360006F5F7F4FCB010E945D5880E001C08AE68D
:10B370006896CDBFDEBFDF91CF911F910895809178
:10B3800092338130A9F420916D33213079F480918A
:10B390006E3381110BC082E080936D3380EC97E5B2
:10B3A0008093993390939A3320936E331092923313
:10B3B00080919333813091F480916D33882331F003
:10B3C000823061F490916E33943051F40E94A29ACD
:10B3D000811104C0109293330E94725990916E3380
:10B3E000809194338130C1F420919333211114C0A2
:10B3F0009150933088F01092943395E090936E338F
:10B4000090936B3390916C33911104C080936C33A3
:10B410000E94E7AE0E9414A380E0089585E0809327
:10B420006B3380916C33811105C081E080936C3364
:10B430000C94E7AE0895CF93DF93CDB7DEB768974E
:10B44000CDBFDEBF80916C33882311F180E090E0A6
:10B45000A0E4B0E489839A83AB83BC831D821E82FF
:10B460001F82188619861A861B861C861D861E86D4
:10B470001F86188A198A1A8A1B8A1C8A1D8A1E8AA4
:10B480001F8A188EBE016F5F7F4FCB010E945D58EF
:10B490006896CDBFDEBFDF91CF910895CF93DF9344
:10B4A000CDB7DEB76897CDBFDEBF80E090E0A0E407
:10B4B000B0E489839A83AB83BC831D821E821F8282
:10B4C000188619861A861B861C861D861E861F8670
:10B4D000188A198A1A8A1B8A1C8A1D8A1E8A1F8A40
:10B4E000188EAE014F5F5F4FBA018DE598E50E945F
:10B4F000E3866896CDBFDEBFDF91CF910895CF93ED
:10B50000DF93CDB7DEB76897CDBFDEBF80E090E0B8
:10B51000A0E8B0E489839A83AB83BC831D821E823A
:10B520001F82188619861A861B861C861D861E8613
:10B530001F86188A198A1A8A1B8A1C8A1D8A1E8AE3
:10B540001F8A188EAE014F5F5F4FBA018DE598E5F7
:10B550000E94E3866896CDBFDEBFDF91CF9108954C
:10B56000CF93DF93CDB7DEB72797CDBFDEBF97E090
:10B57000E9EDF0E2DE01119601900D929A95E1F766
:10B58000873050F4E1E0F0E0EC0FFD1FE80FF11D13
:10B5900087FDFA95808101C080E22796CDBFDEBF8E
:10B5A000DF91CF910895EF92FF920F931F93CF9366
:10B5B000DF931F92CDB7DEB77C018B01642F70E063
:10B5C00080E090E049830E94DED8F70161877287AE
:10B5D0008387948782E087834981E42FF0E0EE0F30
:10B5E000FF1FE00FF11F659174914FE450E081E778
:10B5F0009EE30E9451E4BC01C7010F90DF91CF91FF
:10B600001F910F91FF90EF900C94BC65CF93DF9347
:10B61000EC010E948B4E482F61EB73E1CE01DF916C
:10B62000CF910C94D35A40916B3362E773E10C9441
:10B63000D35A40916C3369E473E10C94D35A40912E
:10B640006D3365E373E10C94D35A40916E3367E038
:10B6500073E10C94D35A40916F336AEE72E10C940B
:10B66000D35AE0919933F0919A33E55BFF4F4081D3
:10B6700064E174E10C94D35AE0919933F0919A33D8
:10B68000E45BFF4F408160E272E10C94D35AE09199
:10B690009933F0919A33448166E871E10C94D35A5E
:10B6A000E0919933F0919A33E65BFF4F408163E577
:10B6B00071E10C94D35AE0919933F0919A33E25BA3
:10B6C000FF4F408169E071E10C94D35AE0919933C6
:10B6D000F0919A33E15BFF4F408168EC70E10C948C
:10B6E000D35AE0919933F0919A33E75BFF4F408151
:10B6F00069E570E10C94D35ACF93DF93EC01E091AC
:10B700009933F0919A33EF5AFF4F608170E080E0F7
:10B7100090E00E94DED869877A878B879C8782E0D9
:10B720008F8380E0DF91CF910895CF93DF93EC0179
:10B7300060919B3370919C3380919D3390919E33A7
:10B740000E94DED869877A878B879C8782E08F8307
:10B7500080E0DF91CF910895CF93DF93EC01E091EA
:10B760009933F0919A3360817181828193810E9433
:10B77000DED869877A878B879C8782E08F8380E019
:10B78000DF91CF910895CF93DF93EC0180916D33DA
:10B79000811105C019861A861B861C8614C00E945A
:10B7A000719A69877A878B879C8720910B58211122
:10B7B0000AC025E832E441E25DE30E94E3DA6987EA
:10B7C0007A878B879C878C819D81FC01EE0FFF1F00
:10B7D000E80FF91FEE0FFF1FEE0FFF1FEE0FFF1F09
:10B7E000EA5FF94E85919491888784E08F8380E0A9
:10B7F000DF91CF910895CF93DF93EC01209199339E
:10B8000030919A33F901FD96608171818281938133
:10B8100069877A878B879C873E96208121110AC091
:10B8200025E832E441E25DE30E94E3DA69877A8742
:10B830008B879C878C819D81FC01EE0FFF1FE80F99
:10B84000F91FEE0FFF1FEE0FFF1FEE0FFF1FEA5F46
:10B85000F94E85919491888784E08F8380E0DF9111
:10B86000CF910895CF93DF93EC018C819D810E944D
:10B870009D4C682F8091993390919A330E940C507F
:10B8800069877A878B879C878C819D81FC01EE0F6D
:10B89000FF1FE80FF91FEE0FFF1FEE0FFF1FEE0F48
:10B8A000FF1FEA5FF94E85919491888784E08F832A
:10B8B00080E0DF91CF910895CF93DF93EC018C81ED
:10B8C0009D810E949D4C2091993330919A332B5940
:10B8D000334369F4E82FF0E0EE0FFF1FEE0FFF1F78
:10B8E000EB50FC4C608171818281938102C00E9487
:10B8F0007A9A69877A878B879C878C819D81FC01E6
:10B90000EE0FFF1FE80FF91FEE0FFF1FEE0FFF1FD7
:10B91000EE0FFF1FEA5FF94E85919491888784E0CE
:10B920008F8380E0DF91CF910895CF93DF93EC0177
:10B930008C819D810E949D4CE0919933F0919A33C6
:10B9400094E0899FE00DF11D1124458D568D678D82
:10B9500070A149875A876B877C878C819D81FC0108
:10B96000EE0FFF1FE80FF91FEE0FFF1FEE0FFF1F77
:10B97000EE0FFF1FEA5FF94E85919491888784E06E
:10B980008F8380E0DF91CF910895CF93DF93EC0117
:10B990000E94576169857A858B859C850E94B2D803
:10B9A000462F60E474E1CE01DF91CF910C94D35A1D
:10B9B000CF93DF93EC018C819D810E949D4C83305D
:10B9C00054F48F3FA9F407C0CE010E94016280E0C9
:10B9D0001CC08DE61AC020E030E040E450E46985E8
:10B9E0007A858B859C850E9441DA181694F3ECCFFA
:10B9F00020E030E040E050E469857A858B859C85C5
:10BA00000E9441DA18162CF3DFCFDF91CF91089511
:10BA100095E3899FF0011124E35CFD4C6081718105
:10BA2000828193810895CF92DF92EF92FF92CF931C
:10BA3000DF936A017B0125E3829FC00111248859AD
:10BA40009E4CFC01EB52FF4F408351836283738312
:10BA5000EC01C352DF4F20E034E244E759E4C70170
:10BA6000B6010E94E3DA9B01AC0160E070E080E87F
:10BA70009FE30E9445D8688379838A839B83DF9103
:10BA8000CF91FF90EF90DF90CF900895CF92DF920B
:10BA9000EF92FF92CF93DF93EC01C984DA84EB84B9
:10BAA000FC8420E034E244E759E4C701B6010E9477
:10BAB00041DA181664F420E034E244E759E4C7019F
:10BAC000B6010E9445D869877A878B879C87CE010B
:10BAD0000E94D666C984DA84EB84FC848C819D81C3
:10BAE0000E949D4C25E3829FC001112488599E4CE1
:10BAF000FC01EB52FF4FC082D182E282F382EC0163
:10BB0000C352DF4F20E034E244E759E4C701B601F5
:10BB10000E94E3DA9B01AC0160E070E080E89FE303
:10BB20000E9445D8688379838A839B8380E0DF9174
:10BB3000CF91FF90EF90DF90CF900895CF92DF925A
:10BB4000EF92FF92CF93DF93EC01C984DA84EB8408
:10BB5000FC8420E034E244E759E4C701B6010E94C6
:10BB600041DA181664F420E034E244E759E4C701EE
:10BB7000B6010E9445D869877A878B879C87CE015A
:10BB80000E94D66680E0DF91CF91FF90EF90DF902A
:10BB9000CF90089581E08093933380E008952CEA5C
:10BBA00035EC47E257E3FC01618572858385948516
:10BBB0000E9441DA181614F40E94D46E80E00895B1
:10BBC000609195337091963380919733909198332B
:10BBD00008950E94E66280E00E94577180E0089517
:10BBE0000E94E66281E00E94577180E008950E9401
:10BBF000E66282E00E94577180E008950E94E6624A
:10BC000083E00E94577180E00895CF93DF93EC01A9
:10BC1000E0919933F0919A33E55BFF4FE081F0E0DA
:10BC2000EE0FFF1FED58FB4E659174914FE450E00D
:10BC300081E79EE30E9451E4AC0162E470E1CE0131
:10BC4000DF91CF910C9441C5CF93DF93EC01E0914C
:10BC50009933F0919A33E55BFF4FE081F0E0EE0F0E
:10BC6000FF1FED58FB4E659174914FE450E081E762
:10BC70009EE30E9451E4AC016AE270E1CE01DF91E3
:10BC8000CF910C9441C5CF93DF93EC018BEE90E202
:10BC90000E94B6E5CE010E94055ECE010E94245EA0
:10BCA00066E170E1CE010E9408C56DEF7FE0CE0134
:10BCB0000E94D3C464EE7FE0CE010E94D3C46BEC3B
:10BCC0007FE0CE010E94D3C462EB7FE0CE010E94F0
:10BCD000D3C469E97FE0CE010E94D3C460E87FE06D
:10BCE000CE010E94D3C467E67FE0CE010E94D3C498
:10BCF0006EE47FE0CE010E94D3C465E37FE0CE0115
:10BD00000E94D3C46CE17FE0CE010E94D3C463E003
:10BD10007FE0CE010E94D3C46AEE7EE0CE010E9495
:10BD2000D3C461ED7EE0CE010E94D3C468EB7EE017
:10BD3000CE010E9408C580E0DF91CF91089566E1B1
:10BD400070E10C9408C56DEF7FE00C94D3C464EEF1
:10BD50007FE00C94D3C46BEC7FE00C94D3C462EB13
:10BD60007FE00C94D3C469E97FE00C94D3C460E80D
:10BD70007FE00C94D3C467E67FE00C94D3C46EE4F8
:10BD80007FE00C94D3C465E37FE00C94D3C46CE1F2
:10BD90007FE00C94D3C463E07FE00C94D3C46AEEDC
:10BDA0007EE00C94D3C461ED7EE00C94D3C468EBC8
:10BDB0007EE00C9408C56CE37EE00C9408C56BE053
:10BDC0007EE00C9408C566ED7DE00C9408C56BE937
:10BDD0007DE00C9408C567E67DE00C9408C5CF9320
:10BDE000DF93EC01E0919933F0919A33E55BFF4FDB
:10BDF000E081F0E0EE0FFF1FED58FB4E659174916E
:10BE00004FE450E081E79EE30E9451E4AC0163E41B
:10BE10007DE0CE01DF91CF910C9441C5CF93DF93AC
:10BE2000EC01E0919933F0919A33E55BFF4FE081AB
:10BE3000F0E0EE0FFF1FED58FB4E659174914FE45B
:10BE400050E081E79EE30E9451E4AC0162E27DE0B4
:10BE5000CE01DF91CF910C9441C565E07DE00C945B
:10BE6000E9C4CF93DF93EC01E0919933F0919A33D9
:10BE7000E55BFF4FE081F0E0EE0FFF1FED58FB4E5A
:10BE8000659174914FE450E081E79EE30E9451E494
:10BE9000AC0166EE7CE0CE01DF91CF910C9441C500
:10BEA0000F931F93CF93DF938C01FC016185728503
:10BEB000838594850E94B2D8E62FF0E0EE0FFF1F35
:10BEC000E05CFB4E659174914FE450E081E79EE3A6
:10BED0000E9451E4E8012D969F938F93F8016185AC
:10BEE0007285838594850E94B2D81F926F93DF93E9
:10BEF000CF930F5E1F4F1F930F93DF93CF938AEC67
:10BF00009CE09F938F93E9E7FBE581818F9380818C
:10BF10008F930E9418E5EDB7FEB73E96EDBFFEBFCA
:10BF2000DF91CF911F910F91089562EA7CE00C940C
:10BF30000F4D6AE77CE00C940F4D68E57CE00C94B3
:10BF40000F4D66E37CE00C940F4D64E07CE00C94B4
:10BF50000F4D63ED7BE00C940F4D6AE97BE00C9490
:10BF60000F4D6AE77BE00C940F4D68E37BE00C9487
:10BF7000DD4C66EF7AE00C94DD4C6FEC7AE00C94CB
:10BF80000F4D69EA7AE00C940F4D68E87AE00C9462
:10BF90000F4D68E67AE00C940F4D6BE47AE00C9458
:10BFA000624D6CE27AE00C94624DBC01675F7F4F9A
:10BFB0002091E63342EA5EE0FC01848195810C9495
:10BFC000B94DBC01675F7F4F21E048E85EE0FC01AE
:10BFD000848195810C94B94DBC01675F7F4F21E04E
:10BFE0004FE65EE0FC01848195810C94B94D0F937E
:10BFF0001F93CF93DF93EC010C811D810E94A168F8
:10C0000008171907C0F48C819D81FC01EE0FFF1FFA
:10C01000E80FF91FEE0FFF1FEE0FFF1FEE0FFF1FC0
:10C02000E55FF94E25913491CE01F901DF91CF9171
:10C030001F910F91199485E1DF91CF911F910F917D
:10C0400008950F931F93CF93DF93EC010C811D8113
:10C050000E94A16808171907C0F48C819D81FC011A
:10C06000EE0FFF1FE80FF91FEE0FFF1FEE0FFF1F70
:10C07000EE0FFF1FE75FF94E25913491CE01F901D4
:10C08000DF91CF911F910F91199485E1DF91CF91AD
:10C090001F910F9108950F931F93CF93DF93EC019E
:10C0A0000C811D810E94A16808171907C0F48C81BA
:10C0B0009D81FC01EE0FFF1FE80FF91FEE0FFF1F20
:10C0C000EE0FFF1FEE0FFF1FE95FF94E2591349130
:10C0D000CE01F901DF91CF911F910F911994DF915A
:10C0E000CF911F910F910895CF93DF93EC018C8135
:10C0F0009D810E94B4688823C9F08C819D81FC01D8
:10C10000EE0FFF1FE80FF91FEE0FFF1FEE0FFF1FCF
:10C11000EE0FFF1FEB5FF94EE491E1FF05C0CE018A
:10C12000DF91CF910C94BC8480E001C085E1DF9168
:10C13000CF9108950F931F93CF93DF93EC0181E08C
:10C140000E9412531C821D8280E090E08E010F5EDF
:10C150001F4F47C08C819D819C01220F331FF90125
:10C16000E80FF91FEE0FFF1FEE0FFF1FEE0FFF1F6F
:10C17000EB5FF94EE491E0FF2EC0280F391F220F2C
:10C18000331F220F331F220F331F215F394EF90156
:10C19000459155916591749149875A876B877C8742
:10C1A000BC01660F771F680F791F660F771F660F38
:10C1B000771F660F771F61507A4E45E050E0C80147
:10C1C0000E9451E4CE010E94F75FCE010E9474608C
:10C1D0002C813D8101C09C012F5F3F4F2C833D830B
:10C1E000C9010E94A4688111B5CF0E9429ACDF91DA
:10C1F000CF911F910F910C94E1ABCF93DF93EC01A2
:10C200002CEA35EC47E257E369857A858B859C8576
:10C210000E943ED887FF05C0CE01DF91CF910C94DC
:10C22000B67DCE010E949A6082E08F8340E050E0AC
:10C2300060E87FE349875A876B877C8780E0DF91DE
:10C24000CF9108958091613B9091623B8F3E9241E6
:10C2500011F08AE508958091A33B9091A43B8F3E15
:10C260009241B9F780913736909138368F3E92419E
:10C2700081F78091593990915A398F3E924149F70F
:10C2800080915B3990915C398F3E924111F780919A
:10C290005F3B9091603B8F3E9241D9F68091C03ECA
:10C2A0008111D7CF0895FC01178289E60895CF93B5
:10C2B000DF93EC018C819D81FC01EE0FFF1FE80FE5
:10C2C000F91FEE0FFF1FEE0FFF1FEE0FFF1FE35FC3
:10C2D000F94EA591B4916C9170E080E090E00E94DD
:10C2E000DED869877A878B879C8782E08F8380E09E
:10C2F000DF91CF910895CF93DF93EC018C819D81E5
:10C30000FC01EE0FFF1FE80FF91FEE0FFF1FEE0FEE
:10C31000FF1FEE0FFF1FE35FF94EA591B4916D91E2
:10C320007D918D919C910E94DED869877A878B8759
:10C330009C8782E08F8380E0DF91CF910895CF9337
:10C34000DF93DC0114968D919C911597FC01EE0F03
:10C35000FF1FE80FF91FEE0FFF1FEE0FFF1FEE0F7D
:10C36000FF1FE35FF94EC591D491488159816A81DD
:10C370007B8119964D935D936D937C931C9783E01D
:10C3800017968C9380E0DF91CF910895CF93DF9340
:10C39000DC0114968D919C911597FC01EE0FFF1F07
:10C3A000E80FF91FEE0FFF1FEE0FFF1FEE0FFF1F2D
:10C3B000E35FF94EC591D491488159816A817B81AF
:10C3C00019964D935D936D937C931C97FC01EE0F32
:10C3D000FF1FE80FF91FEE0FFF1FEE0FFF1FEE0FFD
:10C3E000FF1FEA5FF94E8591949118968C931897E8
:10C3F00084E017968C9380E0DF91CF91089588E6D2
:10C4000008950F931F93CF93DF93EC018C819D814F
:10C41000FC01EE0FFF1FE80FF91FEE0FFF1FEE0FDD
:10C42000FF1FEE0FFF1FE35FF94E05911491698521
:10C430007A858B859C850E94B2D8F801608382E062
:10C440008F8380E0DF91CF911F910F910895CF935B
:10C45000DF93EC0169857A858B859C850E94B2D833
:10C460006230B0F48C819D81FC01EE0FFF1FE80F5C
:10C47000F91FEE0FFF1FEE0FFF1FEE0FFF1FE35F11
:10C48000F94EA591B4916C9382E08F8380E001C056
:10C490008EE6DF91CF910895CF93DF93EC0169850C
:10C4A0007A858B859C850E94B2D86330B0F48C81EC
:10C4B0009D81FC01EE0FFF1FE80FF91FEE0FFF1F1C
:10C4C000EE0FFF1FEE0FFF1FE35FF94EA591B49132
:10C4D0006C9382E08F8380E001C08EE6DF91CF9184
:10C4E0000895CF93DF93EC0169857A858B859C85D0
:10C4F0000E94B2D86430B0F48C819D81FC01EE0FB3
:10C50000FF1FE80FF91FEE0FFF1FEE0FFF1FEE0FCB
:10C51000FF1FE35FF94EA591B4916C9382E08F8386
:10C5200080E001C08EE6DF91CF9108950F931F93B5
:10C53000CF93DF93EC018C819D81FC01EE0FFF1FF7
:10C54000E80FF91FEE0FFF1FEE0FFF1FEE0FFF1F8B
:10C55000E35FF94E0591149169857A858B859C85F9
:10C560000E94B2D8F801608371838283938382E052
:10C570008F8380E0DF91CF911F910F910895CF932A
:10C58000DF93DC0114968D919C911597FC01EE0FC1
:10C59000FF1FE80FF91FEE0FFF1FEE0FFF1FEE0F3B
:10C5A000FF1FE35FF94EC591D49119964D915D91AE
:10C5B0006D917C911C97488359836A837B8383E0C8
:10C5C00017968C9380E0DF91CF910895CF93DF93FE
:10C5D000DC0114968D919C911597FC01EE0FFF1FC5
:10C5E000E80FF91FEE0FFF1FEE0FFF1FEE0FFF1FEB
:10C5F000E35FF94EC591D49119964D915D916D917E
:10C600007C911C97488359836A837B83FC01EE0FDE
:10C61000FF1FE80FF91FEE0FFF1FEE0FFF1FEE0FBA
:10C62000FF1FEA5FF94E8591949118968C931897A5
:10C6300084E017968C9380E0DF91CF9108951F934B
:10C64000CF93DF93EC018091C33B8823D1F01DE1B0
:10C650000A80DB81C02D209711F480E013C08F8108
:10C660008F3FD9F3811104C0CE010E94216006C022
:10C67000CE010E94F75FCE010E947460115041F715
:10C68000ECCF85E6DF91CF911F910895CF93DF9393
:10C69000EC01BC0189EF90E20E948AE4892B41F011
:10C6A000BE018CEF90E20E948AE421E0892B09F41C
:10C6B00020E0822FDF91CF9108950F931F93CF93A6
:10C6C000DF93CDB7DEB72997CDBFDEBF8B0144E046
:10C6D00050E0BC01CE0101960E94AAE446E050E081
:10C6E000B801CE0101960E949AE40E94A1680097C9
:10C6F00009F43FC07981AA81BB811C810D812FEF94
:10C7000035E140E050E0F9016491671327C03196AC
:10C71000E491E11103C0A11121C029C0EA131EC098
:10C72000F9013296E491E11103C0B11117C01FC0A5
:10C73000EB1314C0F9013396E491E11103C0111118
:10C740000DC015C0E1130AC0F9013496E491E1115E
:10C7500003C0011103C00BC0E01749F04F5F5F4FEA
:10C76000285E3F4F4817590709F0CDCF02C0CA01D4
:10C7700002C08FEF9FEF2996CDBFDEBFDF91CF9133
:10C780001F910F910895CF93DF93FC0121892223FC
:10C7900071F1EC016196BE0180E091E20E948AE4B1
:10C7A000892B39F1BE0189EF90E20E948AE4892B3E
:10C7B00011F1BE0183E091E20E948AE4892BD9F055
:10C7C000BE0187EE90E20E948AE4892BB1F0BE019F
:10C7D00086E091E20E948AE4892B79F0BE0187EE1F
:10C7E00091E20E948AE4892B51F485E009C080E03F
:10C7F00007C082E005C083E003C084E001C081E09F
:10C80000DF91CF910895FC018FEF87831482158209
:10C8100011861286138614861086118A1586178A49
:10C82000108EA081B181109711F416820DC0179659
:10C830008C911797873029F416968C918F5F868399
:10C8400003C016968C918683CF010895EF92FF92D4
:10C850000F931F93CF93DF93EC010C811D810E94F6
:10C86000A1680817190708F06FC00C811D81CE015F
:10C870000E9403640C831D837E0181E1E80EF11C9C
:10C88000B801660F771F600F711F660F771F660F65
:10C89000771F660F771F61507A4EC7010E9432E4FE
:10C8A0008E01035F1F4F2C813D81B901660F771FF9
:10C8B000620F731F660F771F660F771F660F771F54
:10C8C00065507A4EC8010E9432E48D85882311F1AB
:10C8D0008C819D81FC01EE0FFF1FE80FF91FEE0F09
:10C8E000FF1FEE0FFF1FEE0FFF1FEB5FF94EE491EE
:10C8F000E2FF02C01D8610C0F80101900020E9F798
:10C90000BF01601B710B605F7F4F6C0F7D1FC70104
:10C910000E9493E48C819D81FC01EE0FFF1FE80FC4
:10C92000F91FEE0FFF1FEE0FFF1FEE0FFF1FE75F58
:10C93000F94E25913491CE01F901DF91CF911F91EC
:10C940000F91FF90EF901994DF91CF911F910F916C
:10C95000FF90EF9008958F929F92AF92BF92CF92E7
:10C96000DF92EF92FF920F931F93CF93DF9300D04C
:10C970001F92CDB7DEB76C015C0181E1A80EB11C3E
:10C9800087E0F6018783ABEFEA2EA5E1FA2E00E0FF
:10C9900010E01DC0B701CE0101960E9432E4BE0135
:10C9A0006F5F7F4FC5010E948AE4892B59F44601CD
:10C9B000F9E18F0E911CF601058F168FC4010E94BC
:10C9C000266464010F5F1F4FF8E1EF0EF11CC801F0
:10C9D0000E94A4688111DECF2496CDBFDEBFDF9117
:10C9E000CF911F910F91FF90EF90DF90CF90BF906C
:10C9F000AF909F908F900895CF93DF9310925D3901
:10CA000010925E39A0E2B6E3E9E3F6E391E08FEF3E
:10CA1000A083B18379965B96ED93FC935C975D96CA
:10CA20001D921C925E97EF0163979883229618825D
:10CA3000219788832A961882599629E3E935F207C7
:10CA400039F71092423910924339109239361092C8
:10CA50003A3610923F3687E08093403682E790E086
:10CA600080934A3690934B3682E596E3DF91CF91DF
:10CA700008950F931F93CF93DF930E94FC64EC0102
:10CA80008FEE92E18093613B9093623B8093A33B56
:10CA90009093A43B809337369093383680935939DE
:10CAA00090935A3980935B3990935C3980935F3BC4
:10CAB0009093603B81E00E9412531C821D82CE0144
:10CAC0000E9493842091AB3B3091AC3B4091AD3BB5
:10CAD0005091AE3B69857A858B859C850E943ED8B6
:10CAE000882339F0CE01DF91CF911F910F910C94E3
:10CAF0009A600E94E6AB1C821D8280E090E08E016D
:10CB00000F5E1F4F2FC06C817D819B01220F331F51
:10CB1000F901E60FF71FEE0FFF1FEE0FFF1FEE0FDD
:10CB2000FF1FEB5FF94EE491E0FF17C0620F731F28
:10CB3000660F771F660F771F660F771F61507A4E5B
:10CB400045E050E0C8010E9451E4CE010E94938468
:10CB5000CE010E94F75F6C817D816F5F7F4F6C8398
:10CB60007D83CB010E94A4688111CDCFDF91CF914D
:10CB70001F910F910C9429ACEF92FF920F931F938A
:10CB8000CF93DF938C0120915D3930915E39EB01B9
:10CB900009900020E9F72197C61BD70BAE01420F81
:10CBA000531F41305240D8F4F901E15AF64C7F014D
:10CBB000AE014F5F5F4FCF010E946BE440915D3942
:10CBC00050915E394F5F5F4F4C0F5D1F40935D3951
:10CBD00050935E39F801E78AF08E80E001C08DE065
:10CBE000DF91CF911F910F91FF90EF900895CF9318
:10CBF000DF932EE1C2E5D6E33F813F3F59F00A8043
:10CC0000DB81C02D209719F480E090E010C0215006
:10CC100099F7FACFBC0180E593E20E945D638C83B3
:10CC20009D83019689F3CE010E942664CE01DF9197
:10CC3000CF910895EF92FF920F931F93CF93DF93BD
:10CC40008B012EE1C2E5D6E33F813F3F59F00A80D8
:10CC5000DB81C02D209719F480E090E01DC02150A9
:10CC600099F7FACF7E0121E1E20EF11C45E050E098
:10CC7000BC01C7010E94AAE4B801CE010E94BC65B4
:10CC80008111EACFB70180E593E20E945D638C8356
:10CC90009D8385E08F83CE01DF91CF911F910F910E
:10CCA000FF90EF9008952091C33B213021F4209113
:10CCB0006D3E213029F4BC0187EE90E20C941A6697
:10CCC00080E090E008959091C33B913019F4642F77
:10CCD0000C940F830C9453C4CF93DF93EC01809199
:10CCE000BD29811103C00E94D4D402C00E94D0CBC0
:10CCF000682F70E080E090E00E94DED869877A8734
:10CD00008B879C8782E08F8380E0DF91CF910895AD
:10CD10000F931F93CF93DF93CDB7DEB7C058D109E0
:10CD2000CDBFDEBFFC0161857285838594850E943D
:10CD3000B2D88FEF860F863030F08AE391E20E94FE
:10CD400053668EE62AC06093B82981E08093B929A2
:10CD5000E62FF0E0EE0FFF1FEA53FA4E6591749153
:10CD60004FE450E081E79EE30E9451E49F938F934C
:10CD700086E894E19F938F938E010F5F1F4F1F935F
:10CD80000F930E940CE6C8010E9453660F900F900B
:10CD90000F900F900F900F9080E0C058DF4FCDBFE5
:10CDA000DEBFDF91CF911F910F9108950F931F93D5
:10CDB000CF93DF93EC018BE993E30E94E74E882346
:10CDC00029F009851A858B859C8511C023E333E3FF
:10CDD0004BEC51E469857A858B859C850E94E3DA6A
:10CDE0008B01AB01BC0149875A876B877C872C81FB
:10CDF0003D81F901EE0FFF1FE20FF31FEE0FFF1F42
:10CE0000EE0FFF1FEE0FFF1FE35FF94EA591B491E8
:10CE1000A801BC014D935D936D937C931397F90129
:10CE2000EE0FFF1FE20FF31FEE0FFF1FEE0FFF1FAE
:10CE3000EE0FFF1FEA5FF94E85919491888784E099
:10CE40008F8380E0DF91CF911F910F91089567E963
:10CE500075E10C94E9C463E775E10C94E9C467E3F8
:10CE600075E10C94E9C46CEF74E10C94E9C46FEAC9
:10CE700074E10C94E9C41F93CF93DF93EC0110E0AD
:10CE80008881882301F10E94FC6445E050E0BE01E6
:10CE900083E696E30E94AAE463E676E380E593E204
:10CEA0000E945D63809356369093573682E596E3F1
:10CEB0000E94266442E063E080E00E9463661F5F98
:10CEC00026961D31E9F684E0DF91CF911F910895F8
:10CED000CF93DF93CDB7DEB7EC97CDBFDEBF8CE34A
:10CEE000E8E1F0E2DE01119601900D928A95E1F7FA
:10CEF000CE0101960E943B67EC96CDBFDEBFDF916D
:10CF0000CF910895CF93DF93CDB7DEB7AA97CDBF6A
:10CF1000DEBF8AE2E4E5F0E2DE01119601900D92B7
:10CF20008A95E1F7CE0101960E943B67AA96CDBF94
:10CF3000DEBFDF91CF910895CF93DF93CDB7DEB7FA
:10CF40006E97CDBFDEBF8EE1EEE7F0E2DE01119617
:10CF500001900D928A95E1F7CE0101960E943B6700
:10CF60006E96CDBFDEBFDF91CF910895CF93DF9353
:10CF7000EC0143E759E763E770E0498B5A8B6B8B11
:10CF80007C8B0E94AB6442E063E080E00E946366B9
:10CF9000CE010E949C67CE010E94826720E731E3A8
:10CFA00040E0298B3A8B4B8BCE010E94AB6442E070
:10CFB00063E080E00E946366CE01DF91CF910C9424
:10CFC0006867CF92DF92EF92FF92CF93DF93EC01ED
:10CFD000C984DA84EB84FC8420E030E040E85FE33D
:10CFE000C701B6010E9441DA18161CF1C701B6014B
:10CFF0000E94B2D86093BA2989859A85AB85BC8591
:10D00000BC01CD019F772CEA35EC47E257E30E9443
:10D0100041DA18163CF460E470E080E00E947CCABB
:10D0200080E008C060E870E080E00E947CCA80E098
:10D0300001C08EE6DF91CF91FF90EF90DF90CF900F
:10D040000895CF92DF92EF92FF92CF93DF93EC019E
:10D05000C984DA84EB84FC8420E030E040E050E4D2
:10D06000C701B6010E9441DA18161CF1C701B601CA
:10D070000E94B2D86093BC2989859A85AB85BC850E
:10D08000BC01CD019F772CEA35EC47E257E30E94C3
:10D0900041DA18163CF464E070E080E00E947CCA3B
:10D0A00080E008C068E070E080E00E947CCA80E018
:10D0B00001C08EE6DF91CF91FF90EF90DF90CF908F
:10D0C0000895CF92DF92EF92FF92CF93DF93EC011E
:10D0D000C984DA84EB84FC8420E030E040E85FE33C
:10D0E000C701B6010E9441DA18161CF1C701B6014A
:10D0F0000E94B2D86093BB2989859A85AB85BC858F
:10D10000BC01CD019F772CEA35EC47E257E30E9442
:10D1100041DA18163CF460E170E080E00E947CCABD
:10D1200080E008C060E270E080E00E947CCA80E09D
:10D1300001C08EE6DF91CF91FF90EF90DF90CF900E
:10D1400008958CE891E0089521E08334914008F03F
:10D1500020E0822F08959C012F55314081E0293233
:10D16000310508F080E0089521E08036914008F014
:10D1700020E0822F0895CF92DF92EF92FF92CF931B
:10D18000DF93EC01C984DA84EB84FC84A701960167
:10D19000C701B6010E9404DC81113CC0E894F7F895
:10D1A0002FEF3FEF4FE75FE7C701B6010E9404DCB6
:10D1B00081110AC02FEF3FEF4FE75FE7C701B601CC
:10D1C0000E943ED8181634F18C819D81FC01EE0F2F
:10D1D000FF1FE80FF91FEE0FFF1FEE0FFF1FEE0FEF
:10D1E000FF1FEB5FF94EE491E3FF14C08BE993E37B
:10D1F0000E94E74E81110EC025E832E441E25DE372
:10D2000069857A858B859C850E94E3DA69877A87B0
:10D210008B879C87DF91CF91FF90EF90DF90CF902D
:10D2200008958091B929882349F01092B929609115
:10D23000B82980E00E9484CA80E0089583E00895C0
:10D24000CF93DF93E091E13BF091E23B04C0E093A8
:10D25000E13BF093E23BEF018191982F9D7F90326B
:10D26000B1F38930A1F34FE450E0BE0187EE9DE3B6
:10D270000E94AAE46881611105C08091C33B8111BD
:10D280005DC028C0613221F4DF91CF910C946659C2
:10D29000653221F4DF91CF910C946A596E3721F4F5
:10D2A000DF91CF910C946E596B3741F481E08093FC
:10D2B000C33BCE01DF91CF910C940C7E70E08AE6E7
:10D2C00091E20E947FE4892B59F01092C33BCE017A
:10D2D0000E94ABC067EE7DE3DF91CF910C94EBC170
:10D2E0008091C33B811109C0CE010E94217467EE79
:10D2F0007DE3DF91CF910C94EBC147EF50E0BE018D
:10D3000087EE9BE30E94AAE487EE9BE39F938F93B3
:10D310008FE691E29F938F93DF93CF930E94E3E593
:10D320000F900F900F900F900F900F908091E13B16
:10D330009091E23BDF91CF910C940C7EDF91CF91E5
:10D340000895FF920F931F93CF93DF931F921F9225
:10D35000CDB7DEB7F82EE5EAFBE324E932E0DF01E2
:10D36000C9011D920197E9F72FEE32E12083318345
:10D370002093373E3093383E0AE919E12CED33E42F
:10D380000093AB3B1093AC3B2093AD3B3093AE3B53
:10D390000CEE11E528E73FE30093AF3B1093B03B61
:10D3A0002093B13B3093B23B00E010E020EA30E440
:10D3B0000093B33B1093B43B2093B53B3093B63B03
:10D3C00000E010E020E83FE30093B73B1093B83B48
:10D3D0002093B93B3093BA3B83E08093C43B8F2DBD
:10D3E0004A8369830E9494CA6981862F0E949FCADA
:10D3F0004A81842F0E94AACAF092B729F092B529D7
:10D400000F900F90DF91CF911F910F91FF90089592
:10D41000CF93DF931F921F92CDB7DEB780E6F82E31
:10D4200001E010E00E94747C8230E1F30E947B7C7A
:10D430008230C1F30E94C64E863009F0C6C00E94F9
:10D4400075C88090CA3B9090CB3BA090CC3BB090ED
:10D45000CD3B86169706A806B90620F70E9475C828
:10D460006C597F4F8F4F9F4F6093CA3B7093CB3B5C
:10D470008093CC3B9093CD3B0E94EA7BD3CF0E941C
:10D480007EBF882329F08CEC0E94FE52823051F23C
:10D490000E94BF59823031F20E946EA1823011F297
:10D4A0000E9422618093C13E81112EC08091A53BD4
:10D4B0009091A63B8F3E924109F08DC08091373EFE
:10D4C0009091383E8F3E924109F085C08AC00E94FB
:10D4D00068858093C13E811117C00E940BB680936E
:10D4E000C13E811111C00E94EC738093C13E811135
:10D4F0000BC00E9496C98093C13E811105C00E9455
:10D50000DFB6823031F48ECF0E94FE528230B9F7FE
:10D5100089CF0E94DDAD823009F484CF0E9449AFEB
:10D52000823009F47FCF0E9410B0823009F47ACFA4
:10D5300009831A8363EE7BE3CE0101960E94B9CA88
:10D540008093E13B9093E23B892B11F00E9420698C
:10D550000E94CD8F823009F465CF0E94236F823004
:10D5600009F460CF0E94E271823009F45BCF0E941F
:10D57000C773823009F456CF0E949550823009F467
:10D580004FCF0E941D868430B0F54ACF8091C43BB6
:10D59000843038F484E08093C43B0E946A590E942E
:10D5A000EBAB83E090E089839A8363EE7BE3CE016B
:10D5B00001960E94B9CA8093E13B9093E23B892B8C
:10D5C00009F42ECF0E9420692BCF0E94C64E8230D4
:10D5D00009F45ECF54CFF092C13E80E60E94FE5225
:10D5E00095CF1092C13E0E94C3528093C13E8823C2
:10D5F00009F46DCF89CF8091CD289091CE280E94DB
:10D6000048D3682F70E080E090E00E94E0D823E3E8
:10D6100033E34BE451E40E9441DA87FF01CF0E94DB
:10D620001169823009F0B2CFFBCE8091B729809387
:10D63000B52908958093B52908958093B629089552
:10D64000CF93C82F80919B23882379F040E050E04E
:10D65000BA018C2F0E940F54EC2FFF27E7FDF095A5
:10D66000E059FC4C81E080830AC06C2F80EC97E588
:10D670000E940C50AB01BC018C2F0E940F544091B2
:10D68000C2235091C3236091C4237091C5238C2F72
:10D690000E94135D89EE9CE680939C2390939D23CA
:10D6A00082E0CF910895CF92DF92EF92FF920F9395
:10D6B0001F93CF93DF93CDB7DEB7E097CDBFDEBF2B
:10D6C00098E17E01A9E1EA0EF11CF701A92F119260
:10D6D000AA95E9F7FE0131966F0111929A95E9F743
:10D6E000F60194E08902E00DF11D1124408F518F65
:10D6F000628F738F80E090E0A0E8BFE38083918326
:10D70000A283B3830093D8331093D9332093DA33B1
:10D710003093DB330E94A0860E946E59B601C70188
:10D720000E9438578093C13E811101C082E0E0968B
:10D73000CDBFDEBFDF91CF911F910F91FF90EF9092
:10D74000DF90CF9008950F931F93E0919523FF27CB
:10D75000E7FDF095EB5BFE4C9381913099F40091DD
:10D76000A6231091A7232091A8233091A9234091AB
:10D77000AE235091AF236091B0237091B1230E94EA
:10D78000536B1DC0E0919623FF27E7FDF095EB5BFF
:10D79000FE4C9381913099F40091A6231091A72318
:10D7A0002091A8233091A9234091AE235091AF231B
:10D7B0006091B0237091B12370580E94536B89EE31
:10D7C0009BE680939C2390939D2382E01F910F9171
:10D7D00008950F931F93CF93C82F85E3C802F001DC
:10D7E0001124EF5BFD4C40815181628173818C2F4C
:10D7F0000E94135D0091A6231091A7232091A823D6
:10D800003091A9234091A2235091A3236091A42396
:10D810007091A5238C2F0E94536B88E79CE6809320
:10D820009C2390939D2382E0CF911F910F910895A7
:10D830000F931F930091A6231091A7232091A82353
:10D840003091A9234091B2235091B3236091B42326
:10D850007091B5230E94536B80E29BE680939C23DA
:10D8600090939D2382E01F910F9108950E94A086BE
:10D870008091BB230E9478538091BA230E94125357
:10D880008091BC230E9416538091BD230E9424578F
:10D890008091BE239091BF23A091C023B091C1235A
:10D8A0008093D8339093D933A093DA33B093DB339A
:10D8B00064E08BE993E30E94044F0E941B5A10928C
:10D8C0006C3380E00895CF93C82F4091C2235091CC
:10D8D000C3236091C4237091C5230E94135D8C2FD4
:10D8E0000E94366C80E00E94ABAD80EFCF9108952E
:10D8F0000F931F93E0919523FF27E7FDF095EB5BD6
:10D90000FE4C9381913039F083E69CE680939C2312
:10D9100090939D2318C00091AA231091AB232091CE
:10D92000AC233091AD234091AE235091AF23609151
:10D93000B0237091B1230E94536B88E19CE68093E1
:10D940009C2390939D2382E01F910F910895FF9255
:10D950000F931F93CF93DF93CDB7DEB7C058D10994
:10D96000CDBFDEBFF82E0E94FC648EEFF81205C01A
:10D970008CE791E20E94536619C08F2D0E94B05A25
:10D980001F928F932BE13BE33F932F938E010F5F09
:10D990001F4F1F930F930E940CE6C8010E9453660D
:10D9A0000F900F900F900F900F900F9042E062E059
:10D9B00080EF0E9463668F2D0E94366C80EFC05806
:10D9C000DF4FCDBFDEBFDF91CF911F910F91FF9051
:10D9D00008954F925F926F927F929F92AF92BF9203
:10D9E000CF92DF92EF92FF920F931F93CF93DF932B
:10D9F0008F3F09F045C02CEA35EC47E257E36091D0
:10DA0000D3347091D4348091D5349091D6340E941F
:10DA100041DA18160CF469C12CEA35EC47E257E3F9
:10DA20006091CB347091CC348091CD349091CE34D0
:10DA30000E9441DA18160CF45DC12CEA35EC47E27D
:10DA400057E36091CF347091D0348091D13490916C
:10DA5000D2340E9441DA18160CF455C12CEA35EC88
:10DA600047E257E36091D7347091D8348091D9342C
:10DA70009091DA340E9441DA18160CF43FC171C15A
:10DA80008230A1F52CEA35EC47E257E36091CB34C4
:10DA90007091CC348091CD349091CE340E9441DA93
:10DAA00018160CF427C12CEA35EC47E257E36091D5
:10DAB000CF347091D0348091D1349091D2340E947F
:10DAC00041DA18160CF41FC12CEA35EC47E257E393
:10DAD0006091D7347091D8348091D9349091DA34F0
:10DAE0000E9441DA18160CF409C131C18823D9F219
:10DAF000813051F32CC17E018DEEE80EF11CF7014F
:10DB000080819181A281B381BC01CD019F772CEAF4
:10DB100035EC47E257E30E943ED887FD46C06E01D0
:10DB2000F1EFCF0ED11CF6014080518062807380EE
:10DB300020E030E0A901C301B2010E943ED887FD78
:10DB400034C0FE01EF52FF4F208131814281538169
:10DB5000349760817181828193810E9495D69B0167
:10DB6000AC015F77C301B2010E9496D62B013C0144
:10DB70009F772CEA35EC47E257E30E943ED887FDB9
:10DB800014C0AB2CAA0C8A2D0E9478BF80939323DB
:10DB9000992493949A0C892D0E9478BF80939423A2
:10DBA00020919323822780FD02C08B2DDBC0B09291
:10DBB0009223F80180819181A281B381BF77809304
:10DBC000A6239093A723A093A823B093A923F7019A
:10DBD00040815181628173817F774093AA23509362
:10DBE000AB236093AC237093AD2320FF2DC0A09294
:10DBF00095239092962377FA709477F870944092D8
:10DC0000A2235092A3236092A4237092A523F6012D
:10DC100080819181A281B3818093AE239093AF23C1
:10DC2000A093B023B093B123CB50DF4F888199816B
:10DC3000AA81BB818093B2239093B323A093B42392
:10DC4000B093B5238A2D2AC090929523A092962353
:10DC50004092A2235092A3236092A4237092A52302
:10DC6000F60180819181A281B381B0588093AE2367
:10DC70009093AF23A093B023B093B123CB50DF4F49
:10DC800088819981AA81BB81B0588093B2239093F7
:10DC9000B323A093B423B093B523892D0E9478BFFA
:10DCA0008D7F813039F089EE9CE680939C239093A0
:10DCB0009D2369C0809196230E9478BF811103C083
:10DCC0008FEF809396238B2D0E94085D6093C22373
:10DCD0007093C3238093C4239093C52383EA9BE668
:10DCE00080939C2390939D234EC082E090E032E08D
:10DCF000B32E0DC080E090E0B12C09C083E090E02D
:10DD000023E0B22E04C081E090E0BB24B394FC0178
:10DD1000E059FC4C108225E3289FE001299FD00D9B
:10DD20001124C859DE4C8E0107511F4FF801808124
:10DD30009181A281B381BC01CD019F772CEA35ECA2
:10DD400047E257E30E943ED887FFD5CE2ECF81E031
:10DD500080936F3386E39CE680939C2390939D236E
:10DD600012C08EEFDF91CF911F910F91FF90EF9036
:10DD7000DF90CF90BF90AF909F907F906F905F901B
:10DD80004F900C94A76C82E0DF91CF911F910F917F
:10DD9000FF90EF90DF90CF90BF90AF909F907F90DB
:10DDA0006F905F904F900895CF93DF93C9E9D3E3CD
:10DDB000888199810E94E74E8093BA238881998156
:10DDC0000E94E24E8093BB23888199810E94F14E8C
:10DDD0008093BC23888199810E94F64E8093BD2355
:10DDE000888199810E94FD4E6093BE237093BF236A
:10DDF0008093C0239093C12381E00E94125381E05D
:10DE00000E94165380E00E94785381E00E942457BC
:10DE100081E080939B238FEF8093922389EE9CE691
:10DE200080939C2390939D2383E080936C33109286
:10DE30006F3380E0DF91CF9108950E94D46E1092ED
:10DE40009B2380E0089580916C33833059F40E94C5
:10DE5000FB4E813049F0E0919C23F0919D2380910D
:10DE60009223199483E0089582E008958EE39FE65B
:10DE70008093D7239093D82382E008952F923F92E6
:10DE80004F925F926F927F928F929F92AF92BF92CA
:10DE9000CF92DF92EF92FF920F931F93CF93DF9376
:10DEA000CDB7DEB7CA54D109CDBFDEBF98E19E0120
:10DEB000275E3F4F29AB3AABD901E92F1D92EA9576
:10DEC000E9F7285131091901D9011D929A95E9F70D
:10DED00024E08202F00111242B96EEAFFFAF2B97C6
:10DEE000E20DF31D80E090E0A0E8BFE38083918322
:10DEF000A283B383C090CF23D090D023E090D123CE
:10DF0000F090D2234090CB235090CC236090CD232F
:10DF10007090CE238090C7239090C823A090C923EF
:10DF2000B090CA23A5019401C301B2010E943ED85A
:10DF300018165CF080E090E0A0E8BFE329968CAF73
:10DF40009DAFAEAFBFAF29970AC080E090E0A0E8D8
:10DF5000BFEB29968CAF9DAFAEAFBFAF2997A301A2
:10DF60009201C501B4010E9495D60E94ADD89B01D3
:10DF700077FF04C022273327261B370BB9018827D8
:10DF800077FD8095982F0E94E0D825966CAF7DAFE5
:10DF90008EAF9FAF2597C092D833D092D933E092FD
:10DFA000DA33F092DB330E94A0860E946E5920E0A3
:10DFB00030E040E050E425966CAD7DAD8EAD9FAD78
:10DFC00025970E9441DA18166CF08091D323909126
:10DFD000D423A091D523B091D6238BAF9CAFADAF06
:10DFE000BEAFDBC02AE037ED43E25CE325966CADC3
:10DFF0007DAD8EAD9FAD25970E9441DA18162CF7A6
:10E0000009E110E08AE0882E87ED982E83E2A82EA1
:10E010008CE3B82E412C512C32012B96AEADBFAD06
:10E020002B97A20DB31D58962196AEAFBFAF219787
:10E030004BAA5CAA6DAA7EAA8FAA98AEA9AEBAAE68
:10E0400029962CAD3DAD4EAD5FAD29976FA978AD4A
:10E0500089AD9AAD0E94E3DA9B01AC016091CB23BC
:10E060007091CC238091CD239091CE230E9496D69F
:10E070002196EEADFFAD21976083718382839383F8
:10E08000C092D833D092D933E092DA33F092DB33B6
:10E09000B101CE0149960E9438578093C13E81114B
:10E0A000AAC020E030E040E85FE36BA97CA98DA91D
:10E0B0009EA90E9496D66BAB7CAB8DAB9EAB20E04D
:10E0C00030E048EC51E40E9445D89B01AC0160E08F
:10E0D00070E080E291E40E9446DB2B013C018091DC
:10E0E000D3239091D423A091D523B091D6238BAF85
:10E0F0009CAFADAFBEAFC090CF23D090D023E09007
:10E10000D123F090D223A7019601BC01CD010E943A
:10E1100095D64B015C0120E030E040E251E4C301C0
:10E12000B2010E9445D89B01AC01C501B4010E9417
:10E13000E3DA9B01AC01C701B6010E9496D66B01E0
:10E140007C012BA93CA94DA95EA9CA01B9010E9475
:10E1500096D620E030E048EC51E40E9445D89B017F
:10E16000AC016FA978AD89AD9AAD0E9496D66FAB20
:10E1700078AF89AF9AAF9B01AC0125966CAD7DADB0
:10E180008EAD9FAD25970E9441DA181634F40150E8
:10E1900011090115110509F053CF8BAD9CADADAD43
:10E1A000BEAD8093D8339093D933A093DA33B09334
:10E1B000DB332B96EEADFFAD2B97E20DF31D809177
:10E1C000C7239091C823A091C923B091CA23808FFF
:10E1D000918FA28FB38FB101CE0149960E9438571B
:10E1E0008093C13E811107C082E191E78093D723DC
:10E1F0009093D82382E0C65BDF4FCDBFDEBFDF91B7
:10E20000CF911F910F91FF90EF90DF90CF90BF9033
:10E21000AF909F908F907F906F905F904F903F90C6
:10E220002F900895CF93DF931F92CDB7DEB78983E8
:10E230000E94A0864091E1235091E2236091E32364
:10E240007091E42389810E94135D8091DE230E94F6
:10E2500078538091DD230E9412538091DF230E9426
:10E2600016538091E0230E9424578091D9239091E6
:10E27000DA23A091DB23B091DC238093D8339093F1
:10E28000D933A093DA33B093DB3364E08BE993E3C3
:10E290000E94044F0E941B5A10926C3388EA91E24C
:10E2A0000E94B6E580E00F90DF91CF9108950F9323
:10E2B0001F93CF93C82F09E913E3F801808191815F
:10E2C0000E94E74E8093DD23F801808191810E94B6
:10E2D000E24E8093DE23F801808191810E94F14E0D
:10E2E0008093DF23F801808191810E94F64E809314
:10E2F000E023F801808191810E94FD4E6093D92333
:10E300007093DA238093DB239093DC238C2F0E947D
:10E31000085D6093E1237093E2238093E32390935D
:10E32000E42381E00E94125380E00E94165380E0B3
:10E330000E94785381E00E94245740E050E060E260
:10E3400071E44093CF235093D0236093D1237093F3
:10E35000D22385E3C89FF0011124EF5CFD4C40817E
:10E360005181628173814093D3235093D42360936E
:10E37000D5237093D6236C2F80EC97E50E94F94F3C
:10E380006093CB237093CC238093CD239093CE23A3
:10E390000E94E05D6093C7237093C8238093C923D4
:10E3A0009093CA23C093C62386E39FE68093D72326
:10E3B0009093D82384E080936C3380E0CF911F91B9
:10E3C0000F91089580916C33843059F40E94FB4E74
:10E3D000813049F0E091D723F091D8238091C62372
:10E3E000199483E0089582E00895E091E723F0E036
:10E3F000EB5BFE4C8381882341F080E192E78093C0
:10E40000E5239093E62382E0089564E374E28CE1CF
:10E4100094E20E9438578093C13E882371F3089597
:10E420001F93CF93DF93E091E723F0E0EB5BFE4C8B
:10E4300081E09381913009F080E080937633C7E7E3
:10E44000D3E310E0812F0E948E9AAB01BC01812F93
:10E450000E940F54612F8091993390919A330E94BA
:10E46000F94F69937993899399931F5F163051F708
:10E4700082EB91E20E940C7E8CE792E78093E52389
:10E480009093E62382E0DF91CF911F9108951F932F
:10E49000CF93DF930E94A0868091E823809345313B
:10E4A000E091E723F0E08091E923EB5BFE4C83876A
:10E4B0000E9495BFCCEED3E210E049915991699149
:10E4C0007991812F0E94135D1F5F1630B1F7809103
:10E4D000EB230E9478538091EA230E94165364E054
:10E4E0008BE993E30E94044F0E941B5A10926C33F5
:10E4F000DF91CF911F9108950E94477280E00895A7
:10E500000F931F93CF93DF93CDB7DEB7C058D109D8
:10E51000CDBFDEBF182F0E94FC641E3F29F48FEB95
:10E5200091E20E94536619C0812F0E94B05A1F9237
:10E530008F9389E49BE39F938F938E010F5F1F4F0F
:10E540001F930F930E940CE6C8010E9453660F9020
:10E550000F900F900F900F900F9042E062E08AEFC3
:10E560000E9463660E9447728AEFC058DF4FCDBF9A
:10E57000DEBFDF91CF911F910F910895FF920F930E
:10E580001F93CF93DF931092763382E080936C33A6
:10E590000CEE13E2C1E4D2E3F12C8F2D0E94085D52
:10E5A000F80161937193819391938F01488159810F
:10E5B0006A817B818F2D0E94135D6F2D809199332D
:10E5C00090919A330E94F94FF801648B758B868B7A
:10E5D000978BF394E596F6E0FF12DFCF6CE174E2DF
:10E5E00084E094E20E9478C52AE43CE042E85EE3DD
:10E5F0000E943ED887FF03C08EEF0E948072C0E168
:10E60000D4E213E069917991899199912C893D899E
:10E610004E895F890E9495D69F772CEA35EC47E2B8
:10E6200057E30E9441DA18161CF4812F0E94807271
:10E630001F5F163039F784E08093E72380915431CF
:10E640008093E92381E08093543180914531809318
:10E65000E823109245310E9495BF809199339091A3
:10E660009A330E94E24E8093EB23809199339091EC
:10E670009A330E94F14E8093EA2380E00E94165361
:10E6800080E00E94785380E00E94F1B185EF91E72D
:10E690008093E5239093E62382E0DF91CF911F9151
:10E6A0000F91FF9008950F931F93CF93DF938C01E9
:10E6B000EB018091E433882399F08091D8339091D5
:10E6C000D933A091DA33B091DB33BC01CD019F7710
:10E6D0002CEA35EC47E257E30E943ED887FD4FC055
:10E6E00088819981AA81BB81BC01CD019F772CEAE9
:10E6F00035EC47E257E30E9441DA1816F4F48C81B6
:10E700009D81AE81BF81BC01CD019F772CEA35ECA4
:10E7100047E257E30E9441DA18167CF48885998510
:10E72000AA85BB85BC01CD019F772CEA35EC47E279
:10E7300057E30E9441DA181624F188E1F801ACE1B0
:10E74000B4E201900D928A95E1F788E1FE01A4E31D
:10E75000B4E201900D928A95E1F788E1E7E7F3E3EF
:10E76000DF011D928A95E9F782E0809376338EEB84
:10E7700092E78093E5239093E62380E003C08EE840
:10E7800001C086E8DF91CF911F910F91089580918C
:10E790006C33823021F080917633823049F40E94CC
:10E7A000FB4E813039F0E091E523F091E623199496
:10E7B00083E0089582E00895E9E3FEE380E2DF016B
:10E7C0001D928A95E9F78FEE92E18093573E9093E0
:10E7D000583E8083918308958091573E9091583E92
:10E7E0008F3E924111F08CE508958091393E9091D1
:10E7F0003A3E8F3E9241B9F780E00895CF93DF9380
:10E80000C82FCB01BA010E9492DB27E0C29FE00132
:10E810001124C75CD14C0E94ADD86D837E838F8359
:10E820009887DF91CF91089597E0899FF001112497
:10E83000E75CF14C65817681878190850E94E0D804
:10E8400008952F923F924F925F926F927F928F9294
:10E850009F92AF92BF92CF92DF92EF92FF920F936F
:10E860001F93CF93DF93CDB7DEB72797CDBFDEBF22
:10E870008C011B8280916B33823009F40CC7D80164
:10E88000BC90B11035C780E06E01B3E0CB0ED11C57
:10E890003DC0F6018081811108C0B72CD7011C92C0
:10E8A0006E01B3E0CB0ED11C20C7883239F4B72CEF
:10E8B000F7011082FFEFCF1ADF0A17C78B33B9F3C6
:10E8C000A82EB12CC5010E9406E4892B39F4B501AC
:10E8D00089EE91E20E947FE4892B51F047018FEF8E
:10E8E000881A980AC5010E942AE4D7018C93740102
:10E8F000BFEFCB1ADB0AF70180818111CACFB72C99
:10E90000D8018C916E01B3E0CB0ED11CF8011CC074
:10E910008E32E1F090E0C0970A9790F081818033C9
:10E9200091F4828190E0C0970A9760F4DF0111961C
:10E9300011968C9111978D938111FACF808104C02B
:10E94000818101C080E331968111E2CFF601A08080
:10E95000A11007C036C0D6011196AC90BFEFCB1AFC
:10E96000DB0A76018A2C912CC4010E941AE4892BBF
:10E9700091F7C4010E9422E48D369105A1F4F601BD
:10E98000818190E00E9422E48337910561F4D601F1
:10E9900012968C9190E00E9422E48736910519F43A
:10E9A000F601339602C0FE013396AA2061F08A2D4B
:10E9B000D701893209F41C9211968C918111F9CFFB
:10E9C00002C0FE013396BFE2BB1609F466C6808121
:10E9D000882319F0CF010E94615980E1E9E5FEE347
:10E9E000DF011D928A95E9F78BE5E4ECF4E3DF01A2
:10E9F000982F1D929A95E9F7E9E6F4E3DF011D925D
:10EA00008A95E9F78BE993E30E94DF4E80936A349D
:10EA1000812C912C80E8A82E8FE3B82E5524539496
:10EA200092E0492E24E0322E23C4C701B6010E9491
:10EA3000B2D8862F90E08F35910508F032C6FC01E0
:10EA4000EC50FF4F0C9489E010926A345092C53418
:10EA500080915A3E8F5F80935A3E0AC450926A3426
:10EA60005092C53480915A3E8F5F80935A3E00C4C5
:10EA700040926A345092C53480915A3E8F5F8093A1
:10EA80005A3EF6C383E080936A345092C534809135
:10EA90005A3E8F5F80935A3EEBC38DE0809369347A
:10EAA0005092C434E5C388E0B2C0109299345092B9
:10EAB000F43480915B3E8F5F80935B3ED9C350926C
:10EAC00099345092F43480915B3E8F5F80935B3E2B
:10EAD000CFC3409299345092F43480915B3E8F5F63
:10EAE00080935B3EC5C310929A345092F534809166
:10EAF0005E3E8F5F80935E3EBBC350929A345092CD
:10EB0000F53480915E3E8F5F80935E3EB1C3C70156
:10EB1000B6010E94FDDB6C837D838E839F8320E0A2
:10EB200030E040E251E4C701B6010E94E3DA6B0134
:10EB30007C0120E030E040E251E46C817D818E81F7
:10EB40009F810E94E3DA9B01AC01C701B6010E94DC
:10EB500095D60E94B2D8623001F128F4662341F0C4
:10EB6000613089F09EC56330E9F0643001F199C5E8
:10EB7000B5E0B09369345092C4348091593E8F5FB0
:10EB80008093593E75C3309269346093C434809148
:10EB9000593E8F5F8093593E6BC3509269345092B7
:10EBA000C43466C3409269345092C43461C383E074
:10EBB000809369345092C4345BC3C701B6010E948C
:10EBC000FDDB6C837D838E839F8320E030E040E219
:10EBD00051E4C701B6010E94E3DA6B017C0120E039
:10EBE00030E040E251E46C817D818E819F810E9402
:10EBF000E3DA9B01AC01C701B6010E9495D60E94E1
:10EC0000B2D8662319F0613061F04BC587E080937C
:10EC100069345092C4348091593E8F5F8093593E3D
:10EC200027C3E6E0E09369346093C4348091593E91
:10EC30008F5F8093593E1CC3C701B6010E94FDDB64
:10EC40006C837D838E839F8320E030E040E251E43B
:10EC5000C701B6010E94E3DA6B017C0120E030E0DD
:10EC600040E251E46C817D818E819F810E94E3DAD4
:10EC70009B01AC01C701B6010E9495D60E94B2D893
:10EC8000623009F00EC58EE0809369345092C4342E
:10EC9000EFC250929C345092F734EAC250929B34A7
:10ECA0005092F6348091623E8F5F8093623EE0C264
:10ECB00040929B345092F6348091623E8F5F8093F5
:10ECC000623ED6C283E016C030929B345092F63436
:10ECD0008091623E8F5F8093623ECAC2F5E0F093FE
:10ECE0009B345092F6348091623E8F5F8093623EF7
:10ECF000BFC286E080939B345092F6348091623E8E
:10ED00008F5F8093623EB4C2C701B6010E94FDDBF3
:10ED10006C837D838E839F8320E030E040E251E46A
:10ED2000C701B6010E94E3DA6B017C0120E030E00C
:10ED300040E251E46C817D818E819F810E94E3DA03
:10ED40009B01AC01C701B6010E9495D60E94B2D8C2
:10ED5000662319F0613059F0A4C410929E34509289
:10ED6000F9348091633E8F5F8093633E81C26093EC
:10ED70009E346093F9348091633E8F5F8093633E4D
:10ED800077C240929E345092F9348091633E8F5FF7
:10ED90008093633E6DC230926A345092C534809144
:10EDA0005A3E8F5F80935A3E63C2C701B6010E94EC
:10EDB000FDDB6C837D838E839F8320E030E040E227
:10EDC00051E4C701B6010E94E3DA6B017C0120E047
:10EDD00030E040E251E46C817D818E819F810E9410
:10EDE000E3DA9B01AC01C701B6010E9495D60E94EF
:10EDF000B2D8662319F0613059F053C410929F3491
:10EE00005092FA3480915C3E8F5F80935C3E30C2BA
:10EE10001092A0346093FB3480915C3E8F5F8093AE
:10EE20005C3E26C2C701B6010E94FDDB6C837D8378
:10EE30008E839F8320E030E040E251E4C701B601B9
:10EE40000E94E3DA6B017C0120E030E040E251E413
:10EE50006C817D818E819F810E94E3DA9B01AC01F0
:10EE6000C701B6010E9495D60E94B2D8662319F058
:10EE7000613059F016C450929F345092FA34809108
:10EE80005C3E8F5F80935C3EF3C16093A0346093DF
:10EE9000FB3480915C3E8F5F80935C3EE9C1C7018B
:10EEA000B6010E94FDDB6C837D838E839F8320E00F
:10EEB00030E040E251E4C701B6010E94E3DA6B01A1
:10EEC0007C0120E030E040E251E46C817D818E8164
:10EED0009F810E94E3DA9B01AC01C701B6010E9449
:10EEE00095D60E94B2D8613089F028F06230A1F046
:10EEF0006330C1F0D6C399E0909369345092C43422
:10EF00008091593E8F5F8093593EB2C1AAE0A09391
:10EF100069346093C434ACC1BBE0B093693450929F
:10EF2000C434A6C1ECE0E09369345092C434A0C16B
:10EF3000109294345092EF3480915D3E8F5F8093B5
:10EF40005D3E96C1509294345092EF3480915D3E74
:10EF50008F5F80935D3E8CC1C701B6010E94B2D81D
:10EF6000862F90E08D33910508F099C3FC01ED5A8E
:10EF7000FE4F0C9489E010926B345092C63480910D
:10EF8000643E8F5F8093643E73C150926B345092A5
:10EF9000C6348091643E8F5F8093643E69C1509215
:10EFA000A634509201358091663E8F5F8093663E15
:10EFB0005FC14092A634509201358091663E8F5FCA
:10EFC0008093663E55C11092A634509201358091CF
:10EFD000663E8F5F8093663E4BC15092A334509241
:10EFE000FE3446C15092A4345092FF348091673E63
:10EFF0008F5F8093673E3CC15092A534509200359C
:10F000008091673E8F5F8093673E32C11092A53436
:10F01000509200358091673E8F5F8093673E28C194
:10F02000509297345092F2348091683E8F5F809373
:10F03000683E1EC1109297345092F2348091683E1F
:10F040008F5F8093683E14C1509295345092F03493
:10F050008091683E8F5F8093683E0AC15092AF34C2
:10F0600050920A358091683E8F5F8093683E00C160
:10F07000C701B6010E94FDDB0E94B2D86093A234A2
:10F080005092FD34F5C0C0928834D0928934E09219
:10F090008A34F0928B348092E3349092E434A092DC
:10F0A000E534B092E634E4C0C092B034D092B134CA
:10F0B000E092B234F092B33480920B3590920C35DA
:10F0C000A0920D35B0920E35D3C0C092A734D09225
:10F0D000A834E092A934F092AA348092023590923A
:10F0E0000335A0920435B0920535C2C0C092703489
:10F0F000D0927134E0927234F09273348092CB34B7
:10F100009092CC34A092CD34B092CE34B1C0C092A3
:10F110007434D0927534E0927634F09277348092E1
:10F12000CF349092D034A092D134B092D234A0C0D7
:10F13000C0927834D0927934E0927A34F0927B3471
:10F140008092D3349092D434A092D534B092D634F5
:10F150008FC0C0927C34D0927D34E0927E34F092A5
:10F160007F348092D7349092D834A092D934B09220
:10F17000DA347EC0C0928034D0928134E0928234FE
:10F18000F09283348092DB349092DC34A092DD34B0
:10F19000B092DE346DC0C0928434D0928534E09257
:10F1A0008634F09287348092DF349092E034A092DB
:10F1B000E134B092E2345CC0C092B834D092B93439
:10F1C000E092BA34F092BB348092133590921435A9
:10F1D000A0921535B09216354BC0C092BC34D09277
:10F1E000BD34E092BE34F092BF34809217359092D5
:10F1F0001835A0921935B0921A353AC0C092C03471
:10F20000D092C134E092C234F092C33480921B3564
:10F2100090921C35A0921D35B0921E3529C0C09227
:10F22000B434D092B534E092B634F092B7348092D0
:10F230000F3590921035A0921135B092123518C04A
:10F24000C701B6010E94B2D860936C3470936D34DC
:10F2500080936E3490936F3481E090E0A0E0B0E052
:10F260008093C7349093C834A093C934B093CA3400
:10F27000D8012C90222009F422C2822D90E00E9415
:10F2800011E4892B09F42DC23801BFEF6B1A7B0AF8
:10F29000F8018181803349F48281883531F40E5F31
:10F2A0001F4FC12CD12C7601FEC1BE016F5F7F4F75
:10F2B000C3010E94A9E06B017C0109811A816016DB
:10F2C000710609F0F0C10FC2809194340E94245756
:10F2D000182F01C010E06091E3347091E434809104
:10F2E000E5349091E6340E94B2D8662359F06091DB
:10F2F00088347091893480918A3490918B340E9443
:10F30000F356182F6091E7347091E8348091E93416
:10F310009091EA340E94B2D8662371F060918C34E7
:10F3200070918D3480918E3490918F340E94B2D838
:10F33000862F0E94CF58182F6091EB347091EC34D7
:10F340008091ED349091EE340E94B2D8662371F032
:10F350006091903470919134809192349091933473
:10F360000E94B2D8862F0E940E59182F6091023544
:10F370007091033580910435909105350E94B2D883
:10F38000662359F06091A7347091A8348091A93414
:10F390009091AA340E9425B2182F60910635709181
:10F3A000073580910835909109350E94B2D86623BF
:10F3B00071F06091AB347091AC348091AD34909128
:10F3C000AE340E94B2D8862F0E944D59182F8091DA
:10F3D000FD34882329F08091A2340E948C57182F85
:10F3E0008091FE34882329F08091A3340E94C05775
:10F3F000182F80910135882329F08091A6340E942E
:10F40000F1B1182F8091FF34882329F08091A43422
:10F410000E94F557182F80910035882329F080919C
:10F42000A5340E942958182F8091F034882329F0A0
:10F43000809195340E94A458182F8091F13488232C
:10F4400029F0809196340E94E358182F80910A3554
:10F45000882329F08091AF340E942259182F80917F
:10F46000F234882329F0809197340E949C58182FF9
:10F47000809169348D3029F08091F4348823A9F08B
:10F480000FC06091B0347091B1348091B2349091DA
:10F49000B3340E942C578093C13E882369F32DC159
:10F4A000809199340E940E53182F8091F53488234F
:10F4B00029F080919A340E941253182F8091F634CB
:10F4C000882329F080919B340E947853182F8091D3
:10F4D000F934882329F080919E340E942857182FF0
:10F4E0008091FA34882329F080919F340E9416532A
:10F4F000182F4091693450E04F30510508F0B4C0E6
:10F50000FA01E057FE4F0C9489E00E947556182FBF
:10F51000ABC06BEC74E380E794E30E948056182F35
:10F52000A3C00E94B456182F9FC06BEC74E380E711
:10F5300094E30E94BF56182F97C00E94D46E182FD4
:10F5400093C06BEC74E380E794E30E943F54182F60
:10F550008BC00E941D6F182F87C06BEC74E380E78F
:10F5600094E30E945373182F7FC06091B034709160
:10F57000B1348091B2349091B3340E94B2D8862FC6
:10F580004BEC54E360E774E30E941A53182F6CC0ED
:10F590006BEC74E380E794E30E94BC54182F64C0C2
:10F5A0000E946F55182F60C00E94D655182F5CC05E
:10F5B0000E940D56182F58C060919C348BE993E33C
:10F5C0000E947A4F80916A34843038F48230D8F4C3
:10F5D000882349F0813079F047C0843009F044C075
:10F5E00080939F3341C06BEC74E380E794E30E9407
:10F5F0004556182F39C06BEC74E380E794E30E9402
:10F600003857182F31C0A090C034B090C134C0908A
:10F61000C234D090C334E090BC34F090BD3400913B
:10F62000BE341091BF342091B8343091B934409138
:10F63000BA345091BB348F938091B7348F938091BB
:10F64000B6348F938091B5348F938091B4348F9377
:10F650006BEC74E380E794E30E943088182F0F90DE
:10F660000F900F900F900F9060E08BE993E30E9452
:10F670007A4F8091C634813061F480916B3481116E
:10F6800004C00E944E5A812F38C00E947F5A812F99
:10F6900034C0812F32C08BEC30C083E02EC084E8B0
:10F6A0002CC083E82AC0822D90E0FC01E154F109CE
:10F6B000EA31F105B0F7E156FE4F0C9489E0109263
:10F6C000C13E60916C3470916D3480916E34909134
:10F6D0006F340E94144F8091EF34882309F4FACDDF
:10F6E000F3CD85E60AC086E608C0D8018C910EC924
:10F6F00068018B2D78017B2CD8C82796CDBFDEBF43
:10F70000DF91CF911F910F91FF90EF90DF90CF90FD
:10F71000BF90AF909F908F907F906F905F904F9031
:10F720003F902F900895CF93DF93EC0167EE7DE338
:10F730000E94BC658093C13E811102C095E09F8309
:10F74000DF91CF910895FC018789908D0C942174ED
:10F7500083FF06C0E0913D31F0913E3190E2958308
:10F7600082FF06C0E0913F31F091403190E29583F5
:10F7700081FF06C0E0914131F091423190E29583E2
:10F7800080FF06C0E0914331F091443180E28583EF
:10F79000089583FF06C0E0913D31F0913E3190E243
:10F7A000968382FF06C0E0913F31F091403190E2B4
:10F7B000968381FF06C0E0914131F091423190E2A1
:10F7C000968380FF06C0E0914331F091443180E29E
:10F7D000868308958091C53B811107C084E00E9413
:10F7E000A87B81E08093C53B089584E00E94C97B9B
:10F7F0001092C53B0895CF92DF92EF92FF920F9344
:10F800001F93CF93DF93C12C26E0D22EC0922D31CF
:10F81000D0922E3130EAE32E36E0F32EE0922F31F3
:10F82000F092303100E816E000933131109332311C
:10F83000C0E6D6E0C0933331D0933431C092353135
:10F84000D0923631C0933731D0933831009339316B
:10F8500010933A31E0923B31F0923C312DEC3CEC8C
:10F860004CED50E40E9441DAC0923D31D0923E31DD
:10F87000E0923F31F092403118164CF4C093413180
:10F88000D0934231009343311093443108C0009328
:10F89000413110934231C0934331D0934431DF91D1
:10F8A000CF911F910F91FF90EF90DF90CF9008952F
:10F8B0000E94E8D560E070E080E091E40E94FB7B6C
:10F8C0000C9407D681E08093CE3B089520E093E02E
:10F8D00088ED08B618BE84BF909380002091820006
:10F8E00021FDFCCF08BEFFCF8091CE3B81110E944D
:10F8F000667C83E008958091CF3B882341F0F894A3
:10F9000061E089E790E00E94EAD582E0089583E013
:10F910000895CF93DF93CDB7DEB7AD97CDBFDEBFF0
:10F9200021E2ECEEF1E2DE01119601900D922A95B2
:10F93000E1F722E02093CA01DE019296E8E0F0E0D0
:10F9400024912D933196EE30F105D1F72DE228A7C1
:10F95000E0E1F0E0E491EF7121E030E02C0F3D1F99
:10F960002E0F311DF901208129A7E2E1F0E0E49199
:10F97000EF719E012E0F311DF90121812AA7E4E1CB
:10F98000F0E0E491EF719E012E0F311DF90121810C
:10F990002BA71CA61092CA0125E0FC012783BE01FB
:10F9A0006E5D7F4F0E94BC658093C13EAD96CDBF1A
:10F9B000DEBFDF91CF91089581E08093CF3B80E05F
:10F9C0000895CF93DF93EC0120E030E040E051E474
:10F9D00069857A858B859C850E9441DA18166CF0C2
:10F9E000CE010E94E66269857A858B859C850E949E
:10F9F000FB7B0E9495BF80E001C08DE6DF91CF9137
:10FA000008956BEE7BE30C9428C56DEC7BE30C94BE
:10FA100028C56EEA7BE30C9428C560E97BE30C946F
:10FA200028C56CE77BE30C94D3C4CF93DF9381E3C9
:10FA300097E49F938F93C9E7DBE589818F93888152
:10FA40008F930E9418E58BEF94E49F938F938981A5
:10FA50008F9388818F930E9418E583E794E49F93A6
:10FA60008F9389818F9388818F930E9418E589EA0B
:10FA700093E49F938F9389818F9388818F930E94C2
:10FA800018E50E94EBAB8DB79EB740968DBF9EBF29
:10FA900080E0DF91CF910895CF93DF9384E893E4E2
:10FAA0009F938F93C9E7DBE589818F9388818F933B
:10FAB0000E9418E586E192E49F938F9389818F934A
:10FAC00088818F930E9418E58BE890E49F938F9331
:10FAD00089818F9388818F930E9418E583E794E44E
:10FAE0009F938F9389818F9388818F930E9418E5CC
:10FAF00089EA93E49F938F9389818F9388818F9371
:10FB00000E9418E58DB79EB744968DBF9EBF80E0DA
:10FB1000DF91CF910895CF93DF938AE690E49F938E
:10FB20008F93C9E7DBE589818F9388818F930E944A
:10FB300018E58CEE9CE39F938F9389818F93888146
:10FB40008F930E9418E589EA93E49F938F938981AC
:10FB50008F9388818F930E9418E58DB79EB70C967E
:10FB60008DBF9EBF80E0DF91CF910895CF93DF934B
:10FB700084EC9CE39F938F93C9E7DBE589818F93A6
:10FB800088818F930E9418E583E59CE39F938F9370
:10FB900089818F9388818F930E9418E589EA93E485
:10FBA0009F938F9389818F9388818F930E9418E50B
:10FBB0008DB79EB70C968DBF9EBF80E0DF91CF9131
:10FBC0000895CF93DF9380E39CE39F938F93C9E7DE
:10FBD000DBE589818F9388818F930E9418E587E008
:10FBE0009CE39F938F9389818F9388818F930E9449
:10FBF00018E589EA93E49F938F9389818F93888195
:10FC00008F930E9418E58DB79EB70C968DBF9EBF4F
:10FC100080E0DF91CF9108952F923F924F925F92B3
:10FC20006F927F928F929F92AF92BF92CF92DF920C
:10FC3000EF92FF920F931F93CF93DF93CDB7DEB771
:10FC40006A97CDBFDEBF5C010E94FC642C011F8659
:10FC5000188A198A1A8AF50101900020E9F731976C
:10FC6000EA19FB09E130F24008F002C2D5018C919B
:10FC7000882359F17501BFEFEB1AFB0A850120E0DB
:10FC8000211115C0883229F08132C8F08F37B9F0C0
:10FC900001C021E06801EFEFCE1ADE0A90E02A8F62
:10FCA0000E9422E4D8018C9386012A8D08C021E0AD
:10FCB000893209F420E0F80180830F5F1F4FD701DC
:10FCC0008D917D018111DCCF01C08501F801108289
:10FCD0001092C13EFDE19F2EAAE36A2EA2E27A2E87
:10FCE000812CB6E02B2E03C09A9409F49CC18BE7BB
:10FCF0009CE2A2E2B0E08B879C87AD87BE876B8ACF
:10FD00007C8A8D8A8DE79CE2A2E2B0E08F8398879F
:10FD1000A987BA87EDE0F2E2DE011196822D01900B
:10FD20000D928A95E1F7C2010E9403648501075F85
:10FD30001F4F75019FEFA91AB90AD7016C9170E0A6
:10FD4000CE010B960E947FE4892B21F487010E5D82
:10FD50001F4F04C0A016B10661F793C16501BFEF44
:10FD6000AB1ABB0AF601608170E0CE0143960E9497
:10FD70007FE4892B91F0D6011D928D0192012F5EB7
:10FD80003F4F288F398F46E050E0B701C9010E94EC
:10FD9000AAE43AE0C30ED11C04C0A016B106F1F6E5
:10FDA00070C15801D8013D908D01E32CF12CC701A1
:10FDB0000E9406E4892B59F4B701CE0101960E94F6
:10FDC0007FE4892B21F40C151D0559F75AC18501D3
:10FDD000BEE63B1641F0E2E23E120CC0D5011196A0
:10FDE0008C918232A9F5F201178211861286138650
:10FDF0001486A3C0B0E3EB1AF108EAE0EE16F104B2
:10FE000018F0FDE23F1217C0BE016A5E7F4FC501C8
:10FE10000E94A9E0D20119966D937D938D939C93D6
:10FE20001C978E899F898A159B0509F42DC1E4E0F2
:10FE30001796EC9382C0FBE73F124FC0E7E0D20178
:10FE40001796EC93FFEFAF1ABF0AE2E0FE2E95C0C3
:10FE50002FEFA21AB20AE5E0D2011796EC9362E204
:10FE600070E0C5010E947FE48E8B9F8B009709F4A0
:10FE700008C1DC011C92F50101900020E9F73197DF
:10FE8000EA19FB093397C8F0F80181818033A9F49E
:10FE90008281883791F440E050E060E070E0C50175
:10FEA0000E941AE2D20119966D937D938D939C93D3
:10FEB0001C9783E017968C9308C0B501C2010E947D
:10FEC000BC658093C13E811153C0AE88BF88BFEF2F
:10FED000AB1ABB0AAE8ABF8A30C0E4E73E120EC03E
:10FEE000E1E0D2011796EC9380E090E0A0E8BFE358
:10FEF000F20181879287A387B4871FC0F6E63F127D
:10FF00000CC0E1E0D2011796EC93179719961D9259
:10FF10001D921D921C921C9710C0BBE53B12B1C0F4
:10FF2000F2012782B501C2010E94BC658093C13EE7
:10FF300081111EC077E6F72E7DC0BE01695F7F4F3D
:10FF4000C5010E94C4E45C01009709F49AC0DC0179
:10FF50008C918D3729F411968C91F50131965F01C2
:10FF60008C3209F48BC0FFEFAF1ABF0AF12C05C029
:10FF7000F82E22E0281708F45DC08F858201035F08
:10FF80001F4F882341F043E050E0BE01615F7F4F87
:10FF9000C8010E94AAE4688D798DC8010E945D6342
:10FFA000D20114968D939C9315978F3FBFEF9B07BB
:10FFB000B9F10E94AB68882371F0888D998D0E94F9
:10FFC0004663882341F043E050E0688D798DCE018F
:10FFD0000F960E94AAE4F20142805380411451041A
:10FFE00011F1F11081CE80915936811108C082E55E
:10FFF00096E30E9421608093C13EF82E1BC0809141
:020000021000EC
:100000006B33823099F082E596E30E94F75F80932C
:10001000C13E81110EC082E596E30E9474600AC061
:1000200064E6F62E07C050E7F52E04C04BECF42E24
:1000300001C0F82E42E060E08F2D0E94636681E0EF
:100040000E94ABAD6A96CDBFDEBFDF91CF911F910D
:100050000F91FF90EF90DF90CF90BF90AF909F9067
:100060008F907F906F905F904F903F902F9008956A
:100070008BE68093C13E3BE6F32EDCCF22E0F22EEE
:100080007CCF9FE6F92ED6CF86E6F82ED3CF2F92DF
:100090003F924F925F926F927F928F929F92AF9218
:1000A000BF92CF92DF92EF92FF920F931F93CF9365
:1000B000DF9300D000D0CDB7DEB78C0169837A839F
:1000C0004B835C835A0128E0A21AB108A60EB71E22
:1000D000DC0116967C907B01BFEFEB1AFB0A8BE7E5
:1000E000FB01808380E0912C95E0692E27E1422E70
:1000F00022E2522E33E1232E32E2332E4DE7842EBC
:10010000ED82FE82D80117969C919F3F09F429C188
:10011000882339F02CE2ED81FE8120833196ED8336
:10012000FE8380916B3E811119C0C80141969F9357
:100130008F933F922F923E813F938D818F930E94A8
:10014000E3E5AD81BE81A80FB91FAD83BE830F90DB
:100150000F900F900F900F900F9018C0C80141960C
:100160009F938F935F924F92BE81BF93ED81EF93E8
:100170000E94E3E52D813E81280F391F2D833E83A8
:100180000F900F900F900F900F900F90D80117962F
:100190008C911797843059F51996CD90DD90ED909C
:1001A000FC901C97A7019601C701B6010E9404DCD0
:1001B000811117C0E894F7F82FEF3FEF4FE75FE7A3
:1001C000C701B6010E9404DC811121C12FEF3FEF6E
:1001D0004FE75FE7C701B6010E943ED818160CF042
:1001E00016C1F801118612861386148610C181117A
:1001F00013C0EDE1F2E2AD81BE81862D01900D923A
:100200008A95E1F72D813E812C5F3F4F2D833E8300
:10021000D80117968C9199C0823061F4F8018485D9
:100220008F9383858F9382858F9381858F93A2E2AD
:10023000B2E214C0833029F5D8011C968C911C972A
:100240008F931B968C911B978F931A968C911A976C
:100250008F9319968C918F93A8E2B2E2BF93AF93DC
:10026000FE81FF932D812F930E94E3E5AD81BE8136
:10027000A80FB11DAD83BE83F8018781CDBFDEBF5E
:1002800064C0853059F4D80158968C9158978F9353
:1002900057968C918F93A0E3B2E20CC0863009F59B
:1002A000D80158968C9158978F9357968C918F932D
:1002B000A5E3B2E2BF93AF93FE81FF932D812F930D
:1002C0000E94E3E5AD81BE81A80FB11DAD83BE8361
:1002D000F80187810F900F900F900F900F900F9063
:1002E00034C0813091F52CEA35EC47E257E3D80170
:1002F00019966D917D918D919C911C970E943ED88D
:1003000087FF12C0EAE3F2E2AD81BE8186E0019090
:100310000D928A95E1F7ED81FE813596ED83FE839E
:10032000D80117968C9111C0E0E4F2E2AD81BE8154
:10033000862D01900D928A95E1F7ED81FE8134962C
:10034000ED83FE83D80117968C91873049F42BE713
:10035000ED81FE8120833196ED83FE8380E001C034
:1003600081E0AD81BE81AA15BB0518F08FEF9FEF2C
:1003700065C0F801028113810115110549F0D8010A
:1003800016969C912FEF290D99153CF0992EBACE17
:10039000ED80FE807914B4F020C0ED81FE81D8019B
:1003A000CF010196808216969C9016973FEF320FF0
:1003B00092161CF4232FFC01F3CF8D839E838D01B5
:1003C00081E0A0CEF7012DE7CF01019620839A941A
:1003D000791414F4FC01F8CF7C018DE79AE0A0E0D9
:1003E000F70180839183A283F2E0EF0EF11C8981F3
:1003F0009A812B813C81820F931F8E159F0508F4F3
:10040000B5CFC701A981BA818A1B9B0B17C0C80150
:100410000E94BB68F80141855285638574852085FB
:100420008D819E810E946CC72D813E81280F311DD8
:100430002D833E83D80117968C9187CF2696CDBF0A
:10044000DEBFDF91CF911F910F91FF90EF90DF9072
:10045000CF90BF90AF909F908F907F906F905F9064
:100460004F903F902F90089540E052E067EE7BE37D
:100470000E9447806091795B70917A5B87EE9BE385
:100480000C9467E5EF92FF920F931F93CF93DF9346
:10049000CDB7DEB76297CDBFDEBFF82E9091693E33
:1004A000992309F4B2C08FE6F81212C00E94FC64CE
:1004B00067EE7DE38091E13B9091E23B0E944CC767
:1004C000BC0186E091E20E941A6602E516E34AC08A
:1004D00080916B3302E516E3882309F443C0EE24D0
:1004E000EA94C8010E94C3638823E1F1823029F4B1
:1004F0008091703E811120C01DC0843029F480910C
:100500006D3E811119C016C08530B1F480916F3EE7
:10051000882381F0F80181859285A385B485BC018B
:10052000CD019F772CEA35EC47E257E30E943ED895
:1005300087FF02C0F801E782F801028113810115EB
:10054000110579F60FC0F80102811381011511051B
:1005500049F440E052E067EE7BE389E396E30E94D2
:10056000478053C0F80197819F3F69F78091BD296B
:1005700081111AC08091E43B8F938091E33B8F936C
:100580001F92FF9285E492E29F938F93CE01019692
:100590007C01FF928F930E94E3E51092E33B10925F
:1005A000E43BCDBFDEBF13C00E94D0CB1F928F9320
:1005B0001F92FF928DE492E29F938F93CE0101965A
:1005C0007C01FF928F930E94E3E5CDBFDEBFB701B0
:1005D000C8010E94BC65F801168286E0878386E622
:1005E00090E0818B928B1282138240E052E067EEA2
:1005F0007BE389E396E30E9447806091795B709189
:100600007A5B87EE9BE30E9467E56296CDBFDEBF13
:10061000DF91CF911F910F91FF90EF90089561307E
:1006200019F0623029F0089582E596E30C94348243
:100630000C944282CF92DF92EF92FF92FC01C18430
:10064000D284E384F48420E030E040EA50E4C7013F
:10065000B6010E9441DA18160CF453C0C701B60166
:100660000E94B2D86093693E10926C3E10926D3E2B
:1006700010926E3E10926F3E1092703E20E030E07D
:1006800040E85FE3C701B6010E9441DA87FD03C07D
:1006900081E080936C3E20E030E040E050E4C70110
:1006A000B6010E9441DA87FD03C081E080936D3E70
:1006B00020E030E040E450E4C701B6010E9441DA96
:1006C00087FD03C081E080936E3E20E030E040E88B
:1006D00050E4C701B6010E9441DA87FD03C081E002
:1006E00080936F3E20E030E040EA50E4C701B6015D
:1006F0000E9441DA87FD07C081E08093703E80E070
:1007000003C08EE601C080E0FF90EF90DF90CF90B5
:10071000089563ED77E40C94E9C46CE777E40C94F6
:10072000E9C468E477E40C94E9C4BF92CF92DF9205
:10073000EF92FF920F931F93CF93DF93CDB7DEB766
:100740006897CDBFDEBF6B0128E1FC01DE01119689
:1007500001900D922A95E1F78CE2E82E82E3F82EC3
:100760008E010F5F1F4FB12CF7018081823029F479
:10077000F80110821182128213828091FB598B1131
:1007800014C020910E5A30910F5A4091105A509136
:10079000115AF80160817181828193810E94E3DAAC
:1007A000F601608371838283938380911A5A8B113F
:1007B00014C020912D5A30912E5A40912F5A5091A9
:1007C000305AF80160817181828193810E94E3DA5D
:1007D000F60164837583868397838091395A8B11E0
:1007E00014C020914C5A30914D5A40914E5A50911C
:1007F0004F5AF80160817181828193810E94E3DA0E
:10080000F60160877187828793878091585A8B1190
:1008100014C020916B5A30916C5A40916D5A50918E
:100820006E5AF80160817181828193810E94E3DABE
:10083000F6016487758786879787B394F5E3EF0E93
:10084000F11C0C5F1F4F86E0B8128ECF6896CDBFAB
:10085000DEBFDF91CF911F910F91FF90EF90DF905E
:10086000CF90BF900895F8940E94587C0E948A848B
:100870000E9407D60E944BC90E9450B60E94DC73AA
:100880000E9495BF0E9472A940E060E080E00E9453
:10089000A1690E9439650E9478840E947C860E942A
:1008A000AE530E94FFD58091A20084608093A20085
:1008B0008091A20082608093A2008091A20081605A
:1008C0008093A20078940E94EBAB0E94AAC00E9481
:1008D000086AFDCFE82FF0E0EE0FFF1FE150F84B64
:1008E000659174914FE450E081E79EE30C9451E4EC
:1008F0008091C23B823041F440E060E081E00E94A0
:10090000A16980E00E941D6B0C94CECC682F81E021
:100910000C943ECA1092C23E1092C33E1092C43E46
:100920001092C53E0895CF93DF93EC018C819D8199
:10093000880F991F880F991F2091C43E3091C53EA2
:10094000820F931F8093C63E9093C73E44E050E0D1
:100950006CEC7EE30E94FFD44091CC3E5091CD3EA2
:100960006091CE3E7091CF3E49875A876B877C87D6
:1009700080E0DF91CF9108958F929F92AF92BF92C6
:10098000CF92DF92EF92FF92CF93DF93EC018091B1
:100990006C33882369F089E0DF91CF91FF90EF906D
:1009A000DF90CF90BF90AF909F908F900C9473ABDF
:1009B00089859A85AB85BC858093C83E9093C93E56
:1009C000A093CA3EB093CB3ECE010E949384809305
:1009D000C13E81116EC0C984DA84EB84FC84A70116
:1009E0009601C701B6010E9404DC81112FC04601A7
:1009F0005701E894B7F82FEF3FEF4FE75FE7C501E6
:100A0000B4010E9404DC81110AC02FEF3FEF4FE7D1
:100A10005FE7C501B4010E943ED81816BCF0809073
:100A2000C83E9090C93EA090CA3EB090CB3EA50172
:100A30009401C701B6010E9495D69F772CEA35EC48
:100A400047E257E30E9441DA181674F58091C83ED8
:100A50009091C93EA091CA3EB091CB3E8093CC3ECE
:100A60009093CD3EA093CE3EB093CF3E8C819D819E
:100A7000880F991F880F991F2091C43E3091C53E61
:100A8000820F931F8093C63E9093C73E44E050E090
:100A90006CEC7EE30E9490D58090C83E9090C93E59
:100AA000A090CA3EB090CB3E89869A86AB86BC8623
:100AB00080E0DF91CF91FF90EF90DF90CF90BF90DB
:100AC000AF909F908F9008950E94ABBB80E00895F7
:100AD0008091D03E9091D13E8F3E924111F08EE5B3
:100AE00008958091F63E9091F73E8F3E9241B9F77E
:100AF0008091F83E9091F93E8F3E924181F780912E
:100B00008156909182568F3E924149F7809183564B
:100B1000909184568F3E924111F780911658909192
:100B200017588F3E9241D9F680E0089594E0899F4E
:100B3000F0011124E053F14C4283538364837583A5
:100B4000089594E0899FF0011124ED57F94A45ABCF
:100B500056AB67AB70AF08955F926F927F928F92A2
:100B60009F92AF92BF92CF92DF92EF92FF920F933C
:100B70001F93CF93DF93CDB7DEB76097CDBFDEBFB6
:100B8000BE016F5F7F4F88EB96E50E949583CE0193
:100B900001964C0180E3A82E87E5B82E90E4C92E7B
:100BA00097E5D92E20E5E22E27E5F22E00E717E59E
:100BB00032E9632E3AE5732E512CF40141915191A3
:100BC000619171914F01F50141935193619371933B
:100BD0005F01F60141935193619371936F01F701A6
:100BE00041935193619371937F01852D0E94FE7310
:100BF000F80111921192119211928F01F30110825A
:100C00001182128213825394F8E16F0E711C84E0FA
:100C10005812D3CF6096CDBFDEBFDF91CF911F9129
:100C20000F91FF90EF90DF90CF90BF90AF909F908B
:100C30008F907F906F905F9008958091FA3E089515
:100C40001F93CF93DF938BE897E1E8EFFEE3DF019B
:100C50009C011D9221503040E1F78FEE92E180938C
:100C6000F83E9093F93E8093815690938256C1E06E
:100C7000DFE3C093FB3ED093FC3EC093FD3ED09398
:100C8000FE3EC093FF3ED093003F81E090E065ECD4
:100C900075E520E030E01CEB129FA001139F500D82
:100CA0001124FA01E850F14CD90111961A9F9001D4
:100CB0001B9F300D11242F5F304C238734876187B1
:100CC0007287BA016F5F704C9C010196803291056A
:100CD00019F78CEB829FF001839FF00D1124E850EF
:100CE000F14CC387D4876187728780E28093FA3E94
:100CF000DF91CF911F910895CF93DF93E3E8F6E55D
:100D000085E991E0DF01EC011D922197E9F7A0ED63
:100D1000BEE388E2ED0119928A95E9F78FEE92E140
:100D20008D939C938093F63E9093F73E80839183BE
:100D30008093165890931758DF91CF910C9420868A
:100D40000E9499900E94208680E00C94C94EE09108
:100D5000FB3EF091FC3E848581111BC022813381D2
:100D6000808191814CEBDF011D924A95E9F7228346
:100D700033838083918381E084878091FA3E815020
:100D80008093FA3E828193818093FB3E9093FC3E58
:100D900005C08CE10E9473ABE0E0F0E0CF01089564
:100DA000ADEFBEE3ED91FC911197858781E08787D8
:100DB00082E08487828193818D939C9381E00E945D
:100DC000FCAE0C94F1B8EF92FF920F931F93CF9368
:100DD000DF9300D01F92CDB7DEB78C014B835C83CD
:100DE00069837A830E94A786FC014B815C816981BB
:100DF0007A81009761F48EE02496CDBFDEBFDF914B
:100E0000CF911F910F91FF90EF900C94FE5283E0D1
:100E1000858784E695E884839583068317838B0111
:100E20007A0126E0D8014D915D916D917D918D0102
:100E3000CF0185599F4FDC014D935D936D937C935A
:100E40001397D7014D915D916D917D917D01418BFE
:100E5000528B638B748B215034962111E3CF83E046
:100E60002496CDBFDEBFDF91CF911F910F91FF90F0
:100E7000EF900C94D086CF92DF92EF92FF926B01AD
:100E80007C010E94A786009739F48EE0FF90EF90D6
:100E9000DF90CF900C94FE522EEB37E8FC012483B8
:100EA0003583E556FF4FC082D182E282F38221E092
:100EB000FC01278782E00E94D08680E0FF90EF90BF
:100EC000DF90CF9008958091FF3E9091003FFC010C
:100ED00024853EEF320F323018F424E02487089541
:100EE000243011F080E090E00895E091FF3EF09111
:100EF000003F22813381808191814CEBDF011D9283
:100F00004A95E9F72283338380839183E091FF3E02
:100F1000F091003F0280F381E02DE093FF3EF093DB
:100F2000003F8485823011F483E084878091FA3E0B
:100F30008F5F8093FA3E8FEF0E94FCAE81E040917C
:100F4000FB3E5091FC3E2091FF3E3091003F421706
:100F5000530709F080E00895BC016F5E7F4FDC010C
:100F60001696ED91FC91179785599F4F19950E9400
:100F7000758781110E941B5A80E0089585569F4F06
:100F800020E034E244E759E4FC0160817181828110
:100F900093810E94E3DA0E94B2D80E94DED80E94B8
:100FA000B5BB0E94758781110E941B5A80E008958D
:100FB0008091FF3E9091003FFC0124853EEF320F6F
:100FC000323018F424E024870895243011F080E0B2
:100FD00090E00895CF93DF93C091FF3ED091003F02
:100FE0008C859EEF980F923018F484E08C8705C0B2
:100FF000843019F080E090E010C02097D9F3DE0132
:101000001296ED91FC9113978785882329F0EC17B0
:10101000FD0711F0DF01F4CFCD01DF91CF910895ED
:10102000CF93DF93EC012A813B81888199814CEB3E
:10103000FB01DE0101900D924A95E1F72A833B8383
:1010400088839983DF91CF9108958FEE92E1809309
:101050001858909319588093D5589093D65808955E
:101060002F923F924F925F926F927F928F929F92B8
:10107000AF92BF92CF92DF92EF92FF920F931F93A6
:10108000CF93DF93CDB7DEB76A97CDBFDEBF4C01FC
:101090001B0129013A01E986FA860B871C871A2D64
:1010A0000B2DE8A8B9A8AAA82BA929838091E4331D
:1010B000882399F08091D8339091D933A091DA3375
:1010C000B091DB33BC01CD019F772CEA35EC47E2D0
:1010D00057E30E943ED887FD11C780910F3590914C
:1010E0001035A0911135B0911235BC01CD019F771B
:1010F00031E03D832CEA35EC47E257E30E9441DAC8
:10110000181614F01D8210C02DEC3CEC4CEC5DE385
:101110006091B4347091B5348091B6349091B73405
:101120000E943ED887FDECC6F10180819181A281A9
:10113000B381BC01CD019F77F1E0FD872CEA35EC4E
:1011400047E257E30E9441DA18160CF01D86F101C0
:1011500084819581A681B781BC01CD019F77F1E0A3
:10116000F98B2CEA35EC47E257E30E9441DA181676
:101170000CF0198AF10180859185A285B3852091B3
:1011800013353091143540911535509116352E8B0D
:101190003F8B488F598F20911735309118354091EA
:1011A000193550911A352A8B3B8B4C8B5D8B4091B6
:1011B0001B3550911C3560911D3570911E35F09096
:1011C000E533F11021C01092605881E0809361589E
:1011D00082E0809362583D81332341F04D85411177
:1011E00095C65989511192C68CE9C1C6CB01BA0185
:1011F0009F772CEA35EC47E257E30E9441DA181654
:101200000CF089C68BE9B3C6BC01CD019F77A1E084
:10121000AA8F2CEA35EC47E257E30E9441DA181610
:101220000CF01A8EB1E0FB1216C01092605882E0EA
:1012300080936158F0926258ED81EE2339F0FD857C
:10124000F11164C62A8D222379F260C66A897B89EE
:101250008C899D89CDCF32E0F31217C081E0809355
:101260006058F0926158109262584D81442341F0C9
:10127000598951114BC68A8D882309F4B5CF46C6CA
:101280006E897F89888D998DB3CFB101C4010E9489
:1012900018519D81992309F451C02091A0333091B8
:1012A000A1334091A2335091A3336091F5337091F3
:1012B000F6338091F7339091F8330E9495D69F775B
:1012C0002CEA35EC47E257E30E943ED887FF36C050
:1012D0002091A4333091A5334091A6335091A73388
:1012E0006091F9337091FA338091FB339091FC3324
:1012F0000E9495D69F772CEA35EC47E257E30E948F
:101300003ED887FF1BC02091A8333091A93340916C
:10131000AA335091AB336091FD337091FE338091CD
:10132000FF33909100340E9495D69F772CEA35ECDC
:1013300047E257E30E943ED887FDE4C58CA980931D
:101340009F338BE993E30E94204F86E5EBE9F3E3BB
:10135000AFE7B8E501900D928A95E1F788E1E5EFF6
:10136000F3E3ABE1B8E501900D928A95E1F7809146
:10137000E6338111D5C523E333E34BEC51E46E2D05
:101380007B2D8A2D99810E94E3DA4B015C016093E9
:101390004B5870934C5880934D5890934E5823E37C
:1013A00033E34BEC51E4C301B2010E94E3DA6093F2
:1013B000335870933458809335589093365823E3BC
:1013C00033E34BEC51E469857A858B859C850E94DB
:1013D000E3DA609337587093385880933958909374
:1013E0003A5823E333E34BEC51E4612F702FC601ED
:1013F0000E94E3DA162F072F412F502FBC01409394
:101400003B5850933C5860933D5870933E588091A0
:10141000B0349091B134A091B234B091B334BC01E6
:10142000CD019F770E941BD90E94B2D860935C586F
:1014300070935D5880935E5890935F58A091605868
:10144000A98BB0916158BA8BEB2FF0E0ED83FE834E
:101450007F01EE0CFF1CEE0CFF1CF101EE0DFF1DD9
:1014600080819181A281B381BC01CD019F772CEA5B
:1014700035EC47E257E30E943ED8D82EDD1CDD2430
:10148000DD1C3989232F30E029833A838901000F3D
:10149000111F000F111FF101E00FF11F80819181D9
:1014A000A281B381BC01CD019F772CEA35EC47E2E4
:1014B00057E30E943ED8881F8827881F8D2180937C
:1014C0005B582CEA35EC47E257E3C501B4019F773E
:1014D0000E9441DA18160CF0F9C0F801E056FC4CF5
:1014E000D801AB50BC4C2D913D914D915C916081E8
:1014F0007181828193810E9495D66B017C01ED817F
:10150000FE81EE0FFF1FEE0FFF1FE056FC4CAD817A
:10151000BE81AA0FBB1FAA0FBB1FAB50BC4C2D91A5
:101520003D914D915C9160817181828193810E9496
:1015300095D669877A878B879C87A5019401C50119
:10154000B4010E94E3DA20E030E040E850E40E9479
:10155000E3DA6D877E878F87988BA7019601C70195
:10156000B6010E94E3DA2B013C0129853A854B85BF
:101570005C85CA01B9010E94E3DA9B01AC01C30199
:10158000B2010E9496D69B01AC016D857E858F8548
:1015900098890E9495D62B013C0120E030E0A901FA
:1015A0000E9441DA1816C4F4C301B2010E94BCDBE8
:1015B0002B013C0129853A854B855C85C701B60125
:1015C0000E944EDA9B01AC01C301B20190580E9407
:1015D00045D82B013C0103C0412C512C3201809194
:1015E0009F33833021F477FA709477F8709420E079
:1015F00030E0A901C501B4010E943ED887FF04C0B4
:1016000077FA709477F8709409811A81000F111F8E
:10161000000F111FA801485E574A5A01A301920109
:1016200069857A858B859C850E94E3DA9B01AC01F4
:10163000C701B6010E9495D620E030E040E05FE3AC
:101640000E94E3DAD5015B966D937D938D939C9315
:101650005E97AD80BE80AA0CBB1CAA0CBB1CF5011A
:10166000E85EF74A4F01A3019201C701B6010E944B
:10167000E3DA9B01AC0169857A858B859C850E94A4
:1016800096D620E030E040E05FE30E94E3DAD40148
:101690005B966D937D938D939C935E97E0916258DA
:1016A000F0E0EE0FFF1FEE0FFF1FE85EF74A138E0C
:1016B000148E158E168EB0914B58B987E0914C5808
:1016C000ED8720904D5830904E5825C05701F701B6
:1016D000E85EF74A838D948DA58DB68D9C01AD0192
:1016E0005058F801E85EF74A838D948DA58DB68D2C
:1016F000BC01CD0190580E944EDA9B01AB01BC01A8
:1017000040934B5850934C5860934D5870934E589B
:1017100029873D871C01D801A85EB74A5B96CD900A
:10172000DD90ED90FC905E97E981FA81EE0FFF1F4E
:10173000EE0FFF1FEC57F74A13962D913D914D91F7
:101740005C91169760817181828193810E9495D608
:10175000A70196010E9495D669837A838B839C8327
:10176000D501A85EB74A5B964D905D906D907C90D8
:101770005E97ED81FE81EE0FFF1FEE0FFF1FEC570E
:10178000F74A13962D913D914D915C91169760818A
:101790007181828193810E9495D6A30192010E945A
:1017A00095D66D837E838F8398879B01AC01698179
:1017B0007A818B819C810E944EDA29853D85A10129
:1017C0000E9495D64B015C01E894B7F820E030E028
:1017D00040E85FE3C501B4010E9441DA18160CF439
:1017E000C3C32AE037ED43EA5BE3C501B4010E94BD
:1017F00041DA181694F42FE632E143E85AE369859A
:101800007D85C1010E94E3DA9B01AC01C501B401F1
:101810000E9441DA18160CF4A7C3A3019201505894
:10182000C701B60190580E9409D74B015C01609333
:1018300043587093445880934558909346588091EC
:10184000E533813039F4412C512C30E8632E3FEBE5
:10185000732E06C0412C512C20E8622E2FE3722EED
:1018600080915B588823D1F160915C5870915D58EC
:1018700080915E5890915F580E94DED86B017C0188
:101880002CEA35EC47E257E30E943ED887FD10C0B2
:1018900010919F332BED3FE049EC50E4C701B601B6
:1018A0000E94E3DA9B01AC01C12CD12C7601B9C0B6
:1018B00081E090E0A0E0B0E080935C5890935D58A8
:1018C000A0935E58B0935F5810919F332BED3FE08B
:1018D00049EC50E4C12CD12C7601A3C02D813E816E
:1018E0004F81588569817A818B819C810E9409D7BB
:1018F00069837A838B839C8360934758709348589D
:101900008093495890934A58A50194010E9495D616
:101910006B017C019F772CEA35EC47E257E30E948C
:101920003ED887FF18C010919F3360915C5870912A
:101930005D5880915E5890915F580E94DED82BEDE3
:101940003FE049EC50E40E94E3DA9B01AC01C12C7A
:10195000D12C760166C029813A814B815C81C50119
:10196000B4010E9441DA1816F4F42BED3FE049EC83
:1019700050E4C301B2010E94E3DA9B01AC0169812A
:101980007A818B819C810E9496D660934758709390
:1019900048588093495890934A58A50194010E9451
:1019A00095D66B017C0110919F33133099F06091B3
:1019B0005C5870915D5880915E5890915F580E947C
:1019C000DED82BED3FE049EC50E40E94E3DA9B01C6
:1019D000AC0127C02BED3FE049EC50E4C301B2015C
:1019E0000E94E3DA9B01AC01C701B6010E9495D6C3
:1019F0007B018C0160915C5870915D5880915E58BC
:101A000090915F580E94DED82BED3FE049EC50E406
:101A10000E94E3DA9B01AC01C701D8016C017D0192
:101A20000BC0123049F4C301B2010E94E3DAA701EE
:101A300096010E9496D60AC0C301B2010E94E3DA61
:101A40009B01AC01C701B6010E9495D67B01AB0199
:101A5000BC0140934F585093505860935158709325
:101A600052588C0150906258A52DB0E0FD01EE0F48
:101A7000FF1FEE0FFF1FEC57F74AAA0FBB1FAA0F5D
:101A8000BB1FA85EB74A13962D913D914D915C9175
:101A9000169760817181828193810E9495D64B0156
:101AA0005C016093535870935458809355589093A9
:101AB00056589701A80169857D85C1010E94E3DA26
:101AC0006B017C0160935758709358588093595814
:101AD00090935A58A50194010E944EDA69837A8343
:101AE0008B839C8360933F587093405880934158F8
:101AF000909342588091E433811117C0F091D8330C
:101B0000FD834090D9332091DA332E8B3091DB3333
:101B10003A8F1092D8331092D9331092DA33109250
:101B2000DB3381E08093E43312C02091D8333091CD
:101B3000D9334091DA335091DB3369817A818B81DB
:101B40009C810E9445D86D83472E8E8B9A8F598930
:101B500045E3549FF0011124E35DFD4C2081318168
:101B600042815381C701B6010E9445D8662E072FD6
:101B7000182F792E2D81342D4E895A8D0E943ED8F2
:101B800087FF04C06D80042D1E897A8C9A8985E3B5
:101B9000989FF0011124E35DFD4C20813181428149
:101BA0005381C701B6010E9445D86B017C019B019E
:101BB000AC01662D702F812F972D0E9441DA1816E7
:101BC00024F06C2C0D2D1E2D7F2C862D902FA12FF7
:101BD000B72D8093635890936458A0936558B09341
:101BE000665820E030E0A901C501B4019F770E944A
:101BF00041DA181684F5A5E35A9EF0011124E35D3D
:101C0000FD4C2081318142815381C501B4010E9484
